:100000004808002065A80108F1AF000805B0000805
:1000100019B000082DB0000841B000080000000031
:1000200000000000000000000000000055B00008C3
:1000300069B000080000000059740008BBCD00083A
:1000400091A8010895A8010899A80108A3D700085C
:100050009DA8010817B50008C5B00008A1A80108AF
:100060006FB200084FB30008A5A80108A9A80108AD
:10007000ADA80108B1A80108B5A80108B9A80108F0
:10008000BDA80108C1A80108C5A80108000000001A
:10009000000000000000000000000000C9A80108E6
:1000A000CDA8010881830108D1A80108D5A80108BD
:1000B000000000000000000000000000D9A80108B6
:1000C000DDA80108E1A80108E5A80108E9A80108E0
:1000D000EDA80108F1A80108F5A80108000000003A
:1000E000F9A801082BB4000800000000000000007F
:1000F000000000000000000000000000FDA8010852
:10010000000000000000000001A90108000000003C
:10011000000000000000000005A901080000000028
:1001200009A901080DA9010811A9010815A90108CB
:1001300019A90108000000000000000000000000F4
:1001400000000000000000000000000000000000AF
:100150002B8301081DA9010821A9010825A901086F
:10016000000000000000000000000000000000008F
:10017000000000000000000000000000000000007F
:1001800029A901082DA901080000000000000000B5
:100190000000000031A9010800000000000000007C
:1001A000000000000000000000000000000000004F
:1001B00000000000000000000000000035A9010858
:1001C00039A901083DA9010870B500224FF4126158
:1001D000DFF8140B02F002F9DFF8104B00221021B7
:1001E00004F11C0002F0FAF8DFF8045B0022182189
:1001F00005F10C0002F0F2F80022082104F12C00B5
:1002000002F0ECF80022082104F1340002F0E6F8D4
:100210000020E06320646064A0646862A862E86211
:10022000DFF8D06AB063F063E06428633064706420
:100230006863A863E863012028640020B064F06468
:100240004FF0FF306864A8640020E86430652065E2
:100250007065F06530667066B066F06202462C210B
:10026000304602F0BBF842F210707081B08100207D
:100270007060022030810020306002460C21204650
:1002800002F0ACF8DFF8700A6060DFF8700A2060F6
:10029000012020720020287028656880A880E880EE
:1002A0006065F0662881A06530636865A865606652
:1002B000A066E0667067306768662866E8650120BA
:1002C0002867E866A8660020E867A86768670620D0
:1002D000B0860020A082F067B0672067DFF8200AB0
:1002E000E065002020660120E082962068810620DB
:1002F000F0860C2020830020B06502464021DFF804
:100300005C0D02F06BF80022062104F10C00BDE840
:10031000704002F063B810B584B0DFF8D0490C2209
:10032000214600A802F098F8FFF74EFF0C2200A922
:10033000204602F091F81FBD2DE9F0472DED0C8B02
:1003400090B00024254600A821460A460B460EC060
:10035000302102F0B9F89FED9B8ADFF8906996EDA5
:100360001B0AD6ED140AC6ED1B0ADFF8887997ED53
:10037000149A86ED149ADFF8788998ED131AB8EE7E
:10038000411ADFED911AC1EE819AC7ED149AD8F89F
:100390004420D8F83490A9EB0200FA30FA21B0FBDF
:1003A000F1F1FA2303FB110080B2002800F0FE8374
:1003B0004C2880F28180D8F8401001297CD0D7F8F1
:1003C0004CA0BAF1040F21D3F4EE490AF1EE10FA71
:1003D0001CD5B4EE699AF1EE10FA17D59FED7B1A91
:1003E00020EE811AB4EE691AF1EE10FA0ED59FEDE7
:1003F000DB1AF4EE419AF1EE10FA07DB87ED149A5E
:10040000C6ED140A86ED1B0A00F009BC97ED0EAA92
:1004100087ED0FAAD7ED10AAC7ED11AA014600EE8D
:10042000101AB8EE400AD8ED0B8AC8EE800A98ED93
:100430000C1A81EE001A2146B963396420E0521C7F
:1004400092B2FA2A00D12246DFF89C3803EB8203ED
:10045000D3ED231A71EEE01AD3F8743402EE103A99
:1004600032EE412AD7ED0E2A41EEA12AC7ED0E2A1F
:10047000D7ED101A42EE021AC7ED101A491C89B2C4
:100480008142DCDBD7ED0E0A80EE80BA87ED0EBA32
:10049000D7ED100A80EE80CA87ED10CAD6ED1ABAE1
:1004A00098ED150AD8ED160A70EE60CAC6ED1ACAA4
:1004B00000F092FF012802D12046386376E3BAF1BA
:1004C000000F0BD1388E052802DB05462046388602
:1004D000788E052802DB4519204678861AFA85F0C1
:1004E000002824D1B6EE00DA3CEE2A0A20EE0D0AEE
:1004F000DFED9B0AB4EE600AF1EE10FA11D43BEE88
:100500000A0A20EE0D0ADFED970AB4EE600AF1EE5A
:1005100010FA06D4B3EE040AF4EE40CAF1EE10FA73
:1005200005D5388E401C3886C8F848903EE3388E92
:10053000002802D04519204638861AFA85F000288E
:1005400015D1B7EE000AF4EE409AF1EE10FA00F180
:100550002D839FED850AF4EE409AF1EE10FA03DB4D
:10056000788E401C788621E32046788603E0788EDA
:10057000451920467886284680B200F0C3FF01283E
:1005800008D187ED149AC7ED10AAC6ED1ABA87ED07
:100590000EAA0BE39FED750AF4EE409AF1EE10FA05
:1005A00002DBDFF8180C386520463886BAF1000FF8
:1005B0000ED1386D786586ED13BAC6ED19CA00F014
:1005C000A5FE3CE00000000000007A446666E63FBD
:1005D000B6EE00DA00F09AFE012816D197ED140A63
:1005E000F0EE000A20EE200A87ED140A6BEE0D0AE9
:1005F000C7ED0E0A2CEE0D1A87ED101AC7ED0F0A83
:1006000087ED111A86ED140A6D1C97ED140AD6EDCC
:10061000140A30EE200A20EE0D0A87ED150A97ED38
:100620000E0AD7ED0F0A30EE200A20EE0D0A86EDF5
:10063000130A3BEEAC0A20EE0D0A86ED190A98F873
:100640000100012840F0A782D8F80C00009000A813
:10065000D8F810104160D8F814108160214617E0D6
:1006600000AB03EB820393ED010A50F822C000EEC9
:1006700090CAB4EE600AF1EE10FA05D500EB820CD8
:100680008CED000AC3ED010A521C022AE8DB491C6A
:10069000022901DA2246F8E79DED000AB5EE400A8C
:1006A000F1EE10FA2AD5B5EE400AF1EE10FA01DCAF
:1006B000B1EE400AD0ED020A30EE800A80ED020A67
:1006C0009DED000AB5EE400AF1EE10FA01DCB1EE44
:1006D000400AD0ED010A30EE800A80ED010A9DED5E
:1006E000000AB5EE400AF1EE10FA01DCB1EE400A64
:1006F000DDED000A30EE800A8DED000A90ED010A72
:10070000D0ED020A30EEC01ADDED000A30EE600ACC
:10071000B4EE401AF1EE10FA05D5F0EE410AB0EE53
:10072000401AB0EE600AD6ED0B0AC6ED0C0A31EEA7
:10073000400A80EE010A9FED0E1A20EE010A86EDB6
:100740000B0A706BB063F4EE400AF1EE10FA11D5AB
:1007500070EE600AC6ED0D0A10E000BF01004040D7
:10076000000016430000A042666616400100A0404B
:100770000000C84270EEC00AC6ED0D0A386F796FEE
:10078000081800EBD070401002EE100A86ED0F2A18
:10079000C6ED108AD7ED100AC6ED110AD7ED141A6E
:1007A000DFF8300CC0EDC41A96ED121A31EE611A62
:1007B000D6ED122A72EEE12A21EE221A00F54471DA
:1007C00081ED011AC6ED121AD7ED1B1AC1ED021AFE
:1007D000D8F81810039103A9C1ED011AC1ED020A5E
:1007E000C1ED038AC1ED041AC1ED058AC1ED061AF7
:1007F000B8EEC22A81ED072AC1ED081A81ED090A77
:10080000C1ED0A1A81ED0B1ADDED032A9FEDD03AF6
:1008100062EE832A9FEDCF3A41EE832A9FEDCE3AD6
:1008200020EE833ADFEDCD3A08EEA33ADFEDCC3A85
:1008300061EEA33A9FEDCB4A48EE843A9FEDCA4A57
:1008400021EE844ADFEDC94A02EE244ADFEDC84AB0
:1008500061EEA44A9FEDC75A40EE054A9FEDC65A85
:1008600021EE855ADFEDC55A01EE255AF8EE085AF9
:10087000F4EE652AF1EE10FA00F18D81DFEDC05A39
:10088000B4EE653AF1EE10FA00F18581DFEDBD5A64
:10089000F4EE653AF1EE10FA00F17D81DFEDBA5A1F
:1008A000B4EE654AF1EE10FA00F175819FEDDF6A52
:1008B000F4EE464AF1EE10FA00F16D819FEDDC6A2C
:1008C000B4EE465AF1EE10FA00F16581DFEDD96A17
:1008D000F4EE662AF1EE10FAC0F25D81DFEDD62A61
:1008E000B4EE623AF1EE10FAC0F25581F4EE653AD8
:1008F000F1EE10FAC0F24F81B4EE464AF1EE10FA72
:10090000C0F24981F4EE654AF1EE10FAC0F243817B
:10091000DFEDCA2AB4EE625AF1EE10FAC0F23B8162
:10092000DFEDC72A9DED033AB4EE623AF1EE10FA1C
:1009300001D5CDED032ADDED032A9FEDD83AF4EE83
:10094000432AF1EE10FA02DBDFF8AC2B0392DFED65
:10095000D42AF4EE621AF1EE10FA01D5C1ED012AA3
:100960009FEDB83ADFEDB83A91ED014AB4EE634A33
:10097000F1EE10FA01DB81ED013A9FEDB44AF4EE9D
:10098000440AF1EE10FA01D581ED024AD1ED020AD6
:100990009FEDAF4AF4EE440AF1EE10FA02DBDFF805
:1009A0005C2B8A60DFEDBF0AF4EE608AF1EE10FA8C
:1009B00001D5C1ED030A9FEDBC4AD1ED034AF4EE27
:1009C000444AF1EE10FA02DBDFF8342BCA60F4EE91
:1009D000621AF1EE10FA01D5C1ED042AD1ED044AF4
:1009E000F4EE634AF1EE10FA01DB81ED043AF4EE25
:1009F000608AF1EE10FA01D5C1ED050AD1ED050AC4
:100A0000F4EE440AF1EE10FA02DBDFF8F42A4A6150
:100A1000F4EE621AF1EE10FA01D5C1ED062AD1ED1D
:100A2000060AF4EE630AF1EE10FA01DB81ED063AF4
:100A3000F1EE000AB4EE602AF1EE10FA02D54FF0A2
:100A40008142CA61D1ED070A9FEDA12AF4EE420A64
:100A5000F1EE10FA02DBDFF82C2CCA61F4EE621A18
:100A6000F1EE10FA01D5C1ED082AD1ED080AF4EE35
:100A7000630AF1EE10FA01DB81ED083ADFED950A29
:100A8000B4EE600AF1EE10FA01D5C1ED090A91ED5C
:100A9000090ADFED910AB4EE600AF1EE10FA02DB0A
:100AA000DFF8E42B4A62F4EE621AF1EE10FA01D597
:100AB000C1ED0A2A91ED0A0AB4EE630AF1EE10FACA
:100AC00001DB81ED0A3AB5EE401AF1EE10FA01D5DC
:100AD0002246CA6291ED0B0ADFED800AB4EE600A8D
:100AE000F1EE10FA02DBDFF8A42BCA62214612E015
:100AF0001B1FD3ED000A92ED031AF4EE410AF1EE4A
:100B000010FA01D59FED760AB8EEC00AD2ED020ABE
:100B100000EE208A491C312938DA9FED720A0B0158
:100B20001A18D2F804C0BCF1010F0DF10C0C1B58BF
:100B30000CEB8303DCD11B1FD3ED000A92ED031AEB
:100B4000F4EE410AF1EE10FADEDB9FED650ADBE719
:100B5000168733BDB0568DBD03275BB9E23C9CB907
:100B6000983115BEBF49D3B97061FDBD55C128BCD0
:100B700036CB05BE3D7FDABBDDED0ABEE4BE353EB9
:100B80006666A6BF3333F3BFCDCC4CBFB5EE408A0B
:100B9000F1EE10FA0ADC97ED150A284680B200F053
:100BA000B1F800F057F80446C8F84890C8F84490E7
:100BB0000020C8F84C00C8F82C00C8F83000C8F86D
:100BC00040000246102106F11C0001F007FC002243
:100BD0000C2108F10C0001F07FFC4948F065002071
:100BE0003066F88800281AD1F86F00280CD0B86C4D
:100BF0003969401AB98EB0EB510F02DB0020388101
:100C00000DE0012038810AE0388E798E11FA80F0EB
:100C1000032802DB0120388101E0022038812046D0
:100C200010B0BDEC0C8BBDE8F08700BFCDCC8CBF05
:100C3000333333BFCDCC0CC09A9919BFCDCC4CBE49
:100C40005017C93F15E6684016E668407D90A341FD
:100C5000A2F2924438B50025DFF8BC4B0120E067D2
:100C600000F0F0FC2060E06CA18E884214D3A06CF0
:100C70002061A08DA080E08DE080A06DA061E06D7E
:100C8000E061206E2062606E6062A06EA062012052
:100C9000A0672846E0670125284632BDC9AC454219
:100CA000A9F56E3EBA9F17443564EC4411480169BA
:100CB00081640021C1644160022101810021C1627F
:100CC000016A0166816A81660021C1677047000080
:100CD000010058427B4D4F3D47FFC742BEBA984185
:100CE00001000000FFFFFFFFD4250020341D00207D
:100CF000341C0020B41C002000002F430000704270
:100D000000007A442DE9F84F2DED048B82B0834624
:100D1000F0EE400A00239E461846DFF8FC4AE56CD8
:100D200005F10F0101F00F01EA1D02F00702009228
:100D3000CA4A02EB8106C6ED000ABBF1000F15D0CE
:100D4000064611E04F1EBF1B10374FEAE70C07EBBA
:100D50001C7C4FEA2C1CB7EB0C1703D402EB870763
:100D6000C7ED000A761C36B25E45EBDB102D02D2D1
:100D7000294609B200E00F219FEDB68A9FEDB51A12
:100D8000DFEDB51A06461BE052F8217000EE107A2E
:100D9000B5EE400AF1EE10FA10DD38EE008AB4EE3E
:100DA000401AF1EE10FA01D5B0EE401AB4EE610A25
:100DB000F1EE10FA01D5F0EE401A761C491E09B288
:100DC0000029E1D536B2314603290BDB38EE410A62
:100DD00030EE610A891E01EE101AB8EEC11A80EEDB
:100DE000018A07E0012905DB00EE106AB8EEC00AAF
:100DF00088EE008AB5EE408AF1EE10FA01D0002E9E
:100E000001D1B0EE608A84ED168A9FED950AB4EEAA
:100E1000408AF1EE10FA02D5B0EE408A08E09FED6C
:100E2000910AB4EE408AF1EE10FA01DBB1EE028ACB
:100E3000B0EE040AB4EE408AF1EE10FA08D494ED54
:100E40001B0AF0EE080AB4EE600AF1EE10FA02D5C1
:100E50000321A18501E00421A185A66C06F0070805
:100E6000DFF8BC7908EB070CA18D8CF8B818BBF142
:100E7000000F0AD0721E02F00702D21906F007090D
:100E8000B94499F8B89882F8B89808220EE0B9F1F8
:100E9000040F00D1401CA8F101080FFA88F8B8F13E
:100EA000000F01D508F10808521E12B2012A16DB04
:100EB0000FFA88F808EB070999F9B898B9F1030F08
:100EC00002D10EF1010E03E0B9F1040F00D15B1C59
:100ED000062AE0DBB9F1030FD9D1401EDBE7E28D32
:100EE0009BB21FFA8EFE734507D39E4502D20420A3
:100EF000E0850DE000B2002802D50320E08507E080
:100F0000012802DB0420E08502E09CF9B808E085B6
:100F1000B4F82E80B8F1040F01D1184600E07046F5
:100F2000424509D000202081E088002820D1042DEE
:100F30001ED3012020811BE013FA8EF2012A15DB5B
:100F4000052A10DB00EE102AB8EEC00AF6EE080AF9
:100F500020EE200A00EE900AF8EE600AF4EE400A55
:100F6000F1EE10FA02D50120208101E0022020815B
:100F7000DFF8B09849B2B0EE480A484600F020F9D0
:100F8000DFED8D0AB4EE600AF1EE10FA01D5B0EE95
:100F9000600A84ED170A584600F1010A00EE90AA93
:100FA000F8EEE08AD4ED180A48EE800AC4ED180A7B
:100FB0009FEDCB9A20EE080A20EE090A009907EB74
:100FC000810101F65C0181ED000ABBF1000F16D032
:100FD000002212E00099491E891A08318B1001EB9A
:100FE0005373DB10B1EBC30105D407EB810101F6AC
:100FF0005C0181ED000A521C12B28242EADB082D2C
:1010000002D2284600B203E0072001E0401E00B2F1
:101010000028FBD584ED190A414649B2484600F044
:1010200047F968EE090AB7EE001AC1EE200A20EE71
:10103000800AD4ED1A0A48EE800AC4ED1A0A0AEBB7
:101040000600A0640AEB0500E06402B0BDEC048B6E
:10105000BDE8F18F000000000000C842E46F0020EE
:101060006666A63F0100904049B2032944D1DFEDF6
:101070009D0AB4EE600AF1EE10FA01DBB0EE600AF0
:101080009FED991ADFED990A40EE010A90ED011AE1
:101090009FED970AB4EE401AF1EE10FA43DADFED55
:1010A000951AB4EE611AF1EE10FA74DBB4EE401A40
:1010B000F1EE10FA6FD59FED900A31EE000ADFEDE8
:1010C0008F1A60EE211A9FED8E0A9FED8E2A01EE97
:1010D000002A22EE200A20EE210A9FEDB72ADFED3A
:1010E000B72A41EE022A62EEA00AB7EE001A31EEEC
:1010F000611A00EE810A56E0DFED830A60EE200AF5
:1011000060EE800A9FEDAE1A40EE410A9FEDAD0AF7
:1011100070EE800A90ED011A9FED750AB4EE401A48
:10112000F1EE10FA0ADB90ED010A9FED751ADFED82
:10113000751A40EE011A21EEA00A34E0DFED6D1AB7
:10114000B4EE611AF1EE10FA25DBB4EE401AF1EEBE
:1011500010FA20D59FED680A31EE000ADFED671A1C
:1011600060EE211A9FED660A9FED662A01EE002AC5
:1011700022EE200A20EE210A9FED8F2ADFED8F2A32
:1011800041EE022A62EEA00AB7EE001A31EE611AB1
:1011900000EE810A07E090ED010A20EE800ADFED03
:1011A0008A0A20EE200A007A022803D1DFEDCA0A5B
:1011B00020EE200A70470000CDCC4C3E0000A0403D
:1011C00010B52DED028BB0EE408A0C46DFED7F8A24
:1011D00049B2FFF749FF64B2042C31D1DFED7C0A3C
:1011E000B4EE608AF1EE10FA16DBB1EE021AB4EE3C
:1011F000418AF1EE10FA0FD5DFEDB80A78EE200A39
:10120000B1EE041A60EE810AFCEEE00A10EE900ADC
:10121000C01D08EE900A3DE0B4EE608AF1EE10FACF
:1012200003D5072008EE900A34E0F1EE020AB4EE8E
:10123000608AF1EE10FA2DDB122008EE900A29E008
:10124000F7EE080AB4EE608AF1EE10FA11DBDFED7A
:10125000A40AB4EE608AF1EE10FA0AD5FFEE080A8D
:1012600078EE200AB1EE041A60EE810AFCEEE08A04
:1012700010E0F7EE080AB4EE608AF1EE10FA09D435
:10128000DFED970AB4EE608AF1EE10FA02DB062079
:1012900008EE900ADFF8580D18EE901A00EB810066
:1012A000D0ED000A20EE200ABDEC028B10BD00003C
:1012B000F0EE0C0A49B2042904D19FED8A1A40EEDF
:1012C000010A03E09FED881A40EE010A9FEDDB0A58
:1012D00020EE800AD0ED000A20EE200A70470000C0
:1012E000000070429A9919406ADEF13D8638163F37
:1012F00000002A4300001643000016C3CDCC4C3D2D
:101300004260E53A6666263F2575C23E0020DFF85A
:10131000081591ED140AF7EE040AB4EE600AF1EE36
:1013200010FA47DADFF8CC2CD288042A42DAD1ED61
:10133000150A9FED6E1A60EE810AB4EE600AF1EEB6
:1013400010FA03D5022A01DB012012E0DFF8D414E1
:1013500091ED0A0ADFED660AB4EE600AF1EE10FACA
:1013600007DBDFED640AB4EE600AF1EE10FA00D597
:10137000012001281ED1DFF8AC1491ED170AD1ED40
:10138000180A70EEC00A9FEDAE1AF4EE410AF1EEB3
:1013900010FA07DBF7EE080AB4EE600AF1EE10FA75
:1013A00000D50020DFEDB30AB4EE600AF1EE10FACA
:1013B00000D500207047000052491D3BB81E053F74
:1013C0007593E83F24975340C1C0C03B0000000024
:1013D00066660640481800200021DFF83C24D38DC3
:1013E000032B1BDA92ED140ADFEDA30AB4EE600AB8
:1013F000F1EE10FA12DB92ED0E0AF2EE040AB4EEF0
:10140000600AF1EE10FA09D592ED100ADFED9B0AA1
:10141000B4EE600AF1EE10FA00D5012192ED100A47
:10142000F6EE000A92ED111A30EE011A21EE201AA2
:10143000F3EE0E1AB4EE611AF1EE10FA1CD492ED2E
:101440000E1AD2ED0F1A71EE211A61EEA01AB2EE49
:10145000042AF4EE421AF1EE10FA0DD4F3EE041A57
:10146000B4EE610AF1EE10FA06D4B1EE040AB4EE5D
:10147000401AF1EE10FA00D5012192ED140A9FED09
:10148000801AB4EE410AF1EE10FA23DBDFF8942360
:1014900092ED090A92ED0A1A80EE010A9FEDA51A53
:1014A000B4EE410AF1EE10FA14DB00EE100AB8EEC9
:1014B000400A20EE200AD2ED070AF4EE400AF1EECF
:1014C00010FA07D5D2ED080AF4EE400AF1EE10FA50
:1014D00000D50121084670473333733F666606C066
:1014E0009A993940CDCC4C3ECDCCCC3D3333333FB3
:1014F000010020420000C842C8AC4542A1F292441B
:101500003464EC440021C44AD36C13FA80F00228FE
:1015100016D392ED140ADFED880AB4EE600AF1EEFC
:1015200010FA0DDB92ED110AD2ED100A80EE200ABE
:10153000DFED820AB4EE600AF1EE10FA00DB012161
:10154000022818D39FED7E0AD2ED110A92ED101AEF
:10155000C0EE810AF4EE400AF1EE10FA0BDBD2ED98
:101560000F0A92ED0E1AC0EE810AF4EE400AF1EE77
:1015700010FA00DB012100280ED0AA4890ED190ACC
:10158000DFED9E0A20EE200AD0ED1A0AF4EE400AA2
:10159000F1EE10FA00D5012192ED140ADFED980A60
:1015A000B4EE600AF1EE10FA08DA92ED150ADFEDFA
:1015B000950AB4EE600AF1EE10FA1ADB92ED100A09
:1015C000DFED910AB4EE600AF1EE10FA0DD492ED5F
:1015D0000E0ADFED8E0AB4EE600AF1EE10FA04D4C2
:1015E000DFF8100AC088022803DBD08D032800DB57
:1015F00001218C4890ED130ADFED830AB4EE600AF6
:10160000F1EE10FA08D492ED1B0AF1EE040AB4EEE2
:10161000600AF1EE10FA0ED5106F526F101800EE3E
:10162000100ABAEEEF0ADFED7A0AB4EE600AF1EEC4
:1016300010FA00DB01210846704700000AD7A33BDF
:101640000100C03F002074498A6C12F10A0F0FD2CA
:101650009FED700AD1ED180AF4EE400AF1EE10FA8F
:1016600006DAD1ED1A0AF4EE400AF1EE10FA00DBC8
:101670000120704785EB113F01000040000020422F
:10168000010040400000584246FFC742BDBA9841A1
:1016900010B401460020634A614BD3F8144900EEB0
:1016A000104AD1ED000AB4EE600AF1EE10FA08D14A
:1016B000147B641C1473E4B2FE2C04DB3224147318
:1016C00001E00446147303F6141393ED010AD1EDFF
:1016D000010AB4EE600AF1EE10FA08D1547B641CE2
:1016E0005473E4B2FE2C04DB3224547301E004464C
:1016F000547393ED020AD1ED020AB4EE600AF1EEE2
:1017000010FA08D1917B491C9173C9B2FE2904DB00
:101710003221917301E001469173117B322905DA80
:10172000517B322902DA917B322900DB012010BC87
:10173000704700003433333F010060400100A04097
:10174000010070410146002091ED000AB5EE400A0B
:10175000F1EE10FA01DCB1EE400A324ADFED2F0A59
:10176000B4EE600AF1EE10FA08DBD37B5B1CD37396
:10177000DBB2FE2B04DB3223D37301E00346D373C9
:1017800091ED010AB5EE400AF1EE10FA01DCB1EE7E
:10179000400AB4EE600AF1EE10FA08DB137C5B1C21
:1017A0001374DBB2FE2B04DB3223137401E0034617
:1017B000137491ED020AB5EE400AF1EE10FA01DC65
:1017C000B1EE400AB4EE600AF1EE10FA08DB517C8B
:1017D000491C5174C9B2FE2904DB3221517401E065
:1017E00001465174D17B322905DA117C322902DAA3
:1017F000517C322900DB0120704700009A99993E04
:1018000001009040010080400000C84300001643E2
:1018100001005C428096184BB41C002035336B41AC
:10182000D4250020341D00202DE9F24F2DED048B2E
:1018300084B004469FEDE58ADFEDE48A9FEDE39AEC
:10184000DFF8405BE888ADF80800A888ADF8020032
:1018500028898DF8000000273E462046FFF718FF34
:1018600001902046FFF76EFF8246DFF888873046FA
:10187000C8F85400C8F85800D8F86800DFF8089B8A
:10188000D9F8141900EE101AD4ED000A30EEC01A7F
:1018900001EE900AF8EEE11A21EE211AB5EE401A97
:1018A000F1EE10FA1ED598ED1D1A70EE411AF5EE04
:1018B000401AF1EE10FA01DC71EE401A9FEDC41AE5
:1018C000F4EE411AF1EE10FA07DB296F491C296783
:1018D000D8F85C10491CC8F85C1088ED1D0A40421D
:1018E000C8F8680009F6141090ED010AD8F86C10D9
:1018F00094ED011A31EE401A01EE901AF8EEE11A59
:1019000021EE211AB5EE401AF1EE10FA1ED598ED2F
:101910001E1A70EE411AF5EE401AF1EE10FA01DCD3
:1019200071EE401A9FEDAA1AF4EE411AF1EE10FA88
:1019300007DB2A6F521C2A67D8F86020521CC8F8AF
:10194000602088ED1E0A4942C8F86C1090ED020A2A
:10195000D8F8700094ED021A31EE401A01EE900AA8
:10196000F8EEE11A21EE211AB5EE401AF1EE10FA66
:101970001ED598ED1F1A70EE411AF5EE401AF1EEE1
:1019800010FA01DC71EE401A9FED911AF4EE411A43
:10199000F1EE10FA07DB296F491C2967D8F86410AB
:1019A000491CC8F8641088ED1F0A4042C8F870004E
:1019B00098F80000052809D10120C8F840003046F9
:1019C00088F80000A8F80200A8F80400D8F84C0035
:1019D00008990818C8F84C00D8F83400D8F8441012
:1019E000884202D10120C8F84000D8F8380000EB46
:1019F000400109EB810B0BF6C000C0ED000A6168E5
:101A00004160A16881600899204600F029FA686168
:101A10000198012802D0BAF1010F32D19FED6B0A73
:101A2000DBF8C00800EE900A60EEA00ADBF8C408FC
:101A300001EE100A21EE011ADBF8C80801EE900A47
:101A400061EEA11ADFF84409017B322904DAC17B77
:101A5000322901DA30EE800A417B322904DA017C36
:101A6000322901DA30EE010A817B322904DA407C26
:101A7000322801DA30EE210A00F094FCF0EE409AB0
:101A800037E00BF50C60D0ED020A90ED011ADBF89F
:101A9000C00800EE100A20EE000A01EE010A00EE76
:101AA000A00A00F07FFCF0EE409AD4ED010A94ED1C
:101AB000000A20EE000A00EEA00A00F073FCB0EE6F
:101AC000408AD4ED020A94ED010A20EE000A00EEED
:101AD000A00A00F067FCF0EE408AD4ED020A94ED13
:101AE000000A20EE000A00EEA00A00F05BFCB0EE57
:101AF000409AD8F83C0000282ED130460CE009EB83
:101B00008001C1ED159A09EB800282ED008AC1EDDA
:101B1000078A81ED0E9A401C0728F0DBB1EE0C0A13
:101B200069EE800AC8ED090AD8F80C00C8F8180058
:101B3000D8F81000C8F81C00D8F81400C8F8200025
:101B400068EE000AC8ED030A68EE800AC8ED040AD0
:101B500029EE000A88ED050AD8F8380009EB800163
:101B600091ED150A39EEC00AD8ED090A30EE200AC7
:101B700088ED090AC1ED159AD8F8340009EB800008
:101B800080ED230AD8ED0B0A70EE800AC8ED0B0A2F
:101B9000D8F80C20C8F81820D8F81020C8F81C2055
:101BA000D8F81420C8F82020D8F8382009EB820291
:101BB00082ED008AC1ED078A81ED0E9A3246DFED93
:101BC000030A9FED021ADFED011A12E00000000087
:101BD000CECC4C3E09EB820393ED002A70EE820AD4
:101BE00093ED072A31EE021A93ED0E2A71EE821A56
:101BF000521C072AEEDBC8ED030A88ED041AC8ED73
:101C0000051AD1ED1C0A70EE600A00F27442C2EDB2
:101C1000000A81ED1C0A98ED0C0AD0F8741400EE4D
:101C2000901A30EE200A88ED0C0A09F6141194EC93
:101C3000030A81EC030ADFF85417096F01290AD15E
:101C40000120C8F84000304688F80000A8F80200DB
:101C5000A8F804007EE0D8F85010491CC8F85010CD
:101C600098F80020012A01D0032A3AD102292BD268
:101C7000EA8D042A28DAE96C00296BD198ED0A0A6A
:101C8000DFEDDA0AB4EE600AF1EE10FA08D5D0F80A
:101C9000741401EE101AB4EE601AF1EE10FA0FDAB5
:101CA000F9EE0C0AB4EE600AF1EE10FA52DBD0F84D
:101CB000740400EE100AB4EE600AF1EE10FA49D591
:101CC0000120C8F8400045E027290AD3B8F80220CF
:101CD000002A03D011FA82F14B2902D30121C8F85E
:101CE0004010D0F8740400EE900A98ED0A0A00F053
:101CF00083F998F8000001282CD1B8F802000028D8
:101D000028D0B8F80410002924D0032211FA80F05A
:101D10003D2802DB0120C8F84000E88D042800DBE4
:101D20000222B8F80600824202D20120C8F8400020
:101D30003046C8F86400C8F86000C8F85C00FEF7D8
:101D4000FBFA0746286F686730462867A8F8040042
:101D5000A8F80600D8F83400D8F84810401AFA302D
:101D6000FA242146B0FBF1F104FB1100B8F80A1087
:101D7000884201D100F031FAD8F83400D8F8481080
:101D8000401AFA302146B0FBF1F104FB110064283F
:101D900001D100F063FAE888BDF80810814204D14F
:101DA000BDF80210AA88914200D00126002814D064
:101DB000D8F83400D8F84810401AFA302146B0FB61
:101DC000F1F104FB1101322902D10120288116E032
:101DD0004B2914D10020288111E0A88800280ED0BA
:101DE000D8F83400D8F84810401AFA302146B0FB31
:101DF000F1F104FB11007D2801D1012028819DF81B
:101E000000002989884200D00126D8F8340009EB67
:101E10008001D1F87414C8F82810401CC8F83400A8
:101E2000FA2802D10020C8F83400D8F83800401C45
:101E3000C8F83800072802D10020C8F83800D8F8C0
:101E40003C00401CC8F83C0047EA0600401E8041A8
:101E5000C043C00F04B0BDEC048BBDE8F28F00009E
:101E600030B4DFF8243590ED000AD3F8142900EEE1
:101E7000902A30EE600A03F61412D0ED010A92EDBA
:101E8000011A70EEC10A90ED021AD2ED021A31EE7B
:101E9000611AB5EE400AF1EE10FA02DDF0EE401ADA
:101EA00001E0F1EE401AF5EE400AF1EE10FA02DD23
:101EB000B0EE602A01E0B1EE602AB5EE401AF1EE14
:101EC00010FA02DDF0EE412A01E0F1EE412A71EE56
:101ED000821A71EEA21AB5EE400AF1EE10FA01DC98
:101EE000B1EE400ADFF8A40490ED072A32EE000AB2
:101EF00080ED070AF5EE400AF1EE10FA01DCF1EE92
:101F0000600A90ED080A30EE200A80ED080AB5EE6E
:101F1000401AF1EE10FA01DCB1EE411A90ED090A17
:101F200030EE010A80ED090A90ED0A0A30EE210A2E
:101F300080ED0A0A2F4AD46B002C12D1002406E04F
:101F400003EB850505F67C05C5ED001A641CA4B2FB
:101F500025460F2DF4DBB2EE0E0A21EE800A80ED4D
:101F6000150A148903EB8403D3F87C5800EE105A49
:101F700031EEC00AD0ED150A30EE200A80ED150AC8
:101F800003F67C03C3ED001AF2EE0E0A80EE200A7F
:101F9000DFF8F03383ED1B0AD0ED170AB4EE600AC8
:101FA000F1EE10FA01D580ED170AD0ED180AF4EE23
:101FB000400AF1EE10FA01D580ED180ADFEDA50A0E
:101FC000B4EE600AF1EE10FA03D5836DC91881658D
:101FD00001E000218165611C118189B20F2901D1C5
:101FE00000211181806D30BC704700000100E0408D
:101FF000681E0020341C00209FED971ADFF8840330
:10200000C08D042801DBB0EE001ADFF88403B5EEC2
:10201000400AF1EE10FA07DBF5EE400AF1EE10FA95
:1020200002D5C188491CC1800178002905D0022948
:1020300060D02DD3032976D0B0E0F1EE0C1A31EE4A
:10204000211AB4EE401AF1EE10FA0BDBB4EE601A6E
:10205000F1EE10FA06D5016D1029C0F08F80002135
:1020600001658BE0416BDFF8202302EB8101D1F8A1
:10207000741401EE901ADFF81C1391ED010AF4EECE
:10208000401AF1EE10FA40F18980C1ED011A85E0A5
:10209000416BDFF8F42202EB8101D1F8741401EEF8
:1020A000901ADFF8F01291ED002AB4EE612AF1EEF9
:1020B00010FA01D5C1ED001AF7EE001AB4EE610A6C
:1020C000F1EE10FA6ADBB7EE000AF4EE400AF1EE28
:1020D00010FA63D5016D418000210165B9EE0C0A4B
:1020E00030EE410AF4EE400AF1EE10FA10D402216B
:1020F000017053E0F9EE0C1A31EEC11AB4EE410A48
:10210000F1EE10FA4ADBF4EE410AF1EE10FA45D591
:10211000032101709C49426B01EB8201D1F87414D8
:102120009C4A51603AE0416B974A02EB8101D1F839
:10213000741401EE901A974991ED012AF4EE421AB7
:10214000F1EE10FA01D5C1ED011ADFED7B1AB4EE04
:10215000610AF1EE10FA21D5F4EE610AF1EE10FAFF
:102160001CDB016D818000210165B1EE0C0A31EEAE
:10217000000AB4EE600AF1EE10FA0ED501210170EA
:1021800084490A6842654A6882657F4A436B02EB6C
:102190008302D2F874240A6000E00170007870476E
:1021A000002803D077492C2200F056B97047002848
:1021B00006D0764942684A6002680A60007A08726E
:1021C000704780B5002801D1002002BD542201468D
:1021D000714800F041F9012002BD10B5694CE08D55
:1021E000A18D002904D0002802D00020208106E023
:1021F000084302D00120208101E00220208100203C
:10220000E0646062A061A080A08520636065A06535
:1022100002464021614800F0E1F8E06F012801D159
:10222000FEF744FD5948818A002909D0E28E8A428E
:1022300001D2A18600E0A286002181820846A06723
:10224000A06F012801D1E08EA0860020A06710BDFC
:1022500000000000EC51383E0000000010B5494C71
:10226000E08DA18D002904D0002802D0002020811B
:1022700006E0084302D00120208101E002202081F5
:1022800000206062A061E085E080024608214448A9
:1022900000F0A4F800202063E06F012801D1FEF7D0
:1022A00005FDA06F012801D1E08EA08610BD80B58C
:1022B000012036490867FFF7D1FFFFF78EFFBDE821
:1022C000014003E000203149086770472F48008B28
:1022D0002C49898E814200D200E070472949CA6C9E
:1022E0008B8E9A4203D288860020886770472749E0
:1022F000888270472348C16C002904D1018E408E2A
:1023000010FA81F070470020704701460020002934
:1023100002D0012901D0704702E01A48C06C704712
:102320001848818EC26C891A028E891A408E081A4A
:1023300000D5002070470000FEFF7FBF38B504467F
:102340001348124D0F49012C06D10622CA860C22D1
:102350002A839622428105E00722CA860F222A8319
:1023600064224281E88AA04209D0888E082803DAD4
:10237000C88EFFF7B3FF02E0288BFFF7AFFFEC82B8
:1023800031BD0000B41C0020D4250020341D0020E5
:10239000341C00209C710020681E0020E46F002087
:1023A0008C2E002081B08DED000A0098401000F1C5
:1023B000FE500090DDED000AC0EE200A9DED001AEF
:1023C00070EE810ACDED000AB5EE001ADDED001ABF
:1023D00080EE210A00EE810A01B0704762F30F22FD
:1023E00062F31F4200B500BF1300964694461039B1
:1023F00028BFA0E80C50FAD85FEA417C28BF0CC087
:1024000048BF40F8042BC90728BF20F8022B48BF5B
:1024100000F8012B00BD50F8041B61B150F8042BEB
:10242000D30744BFA9F101039A180023091F42F8FA
:10243000043BFAD1EFE7704762B38B0708D0521E16
:1024400011F8013B00F8013B00F024808B07F6D126
:10245000830740F0208000BF103A07D330B4B1E8C2
:102460003810103AA0E83810F9D230BC530724BF16
:10247000B1E80810A0E8081044BF51F8043B40F848
:10248000043BD20724BF31F8022B20F8022B44BFB3
:102490000B7803707047083A07D3B1E80810083A80
:1024A00040F8043B40F804CBF7D25307E4E78268D6
:1024B000521C8260426832B10268531C0360117082
:1024C0004168491E416070470022FFF78BBF0268D8
:1024D000531C03601170704762F30F2262F31F42B6
:1024E000401810F0030308D0C91A1FD3DB0748BFF8
:1024F00000F8012D28BF20F8022D130030B4144637
:102500001546103928BF20E93C00FAD8490728BFF2
:1025100020E90C0048BF40F8042D890028BF20F8AE
:10252000022D48BF00F8012D30BC7047C91818BFF4
:1025300000F8012DCB0728BF00F8012D70470000DF
:1025400010B5DFF8044D04F1AC01012001F0A4FB4B
:10255000002805D00FF2480002F0A0F8032010BDBB
:102560000FF2500002F09AF8002060732087E064B8
:1025700002464421DFF8E80CFFF730FF01223C213E
:10258000AA2002F0A8FA00202074A073E063A065DE
:10259000A4F84000A07400F0B9FD002010BD0000B8
:1025A00050443A204641494C20524547494C494203
:1025B0005648000050443A20537461727450656468
:1025C0006F2D30383232000080B5DFF8BC1C01209E
:1025D00001F0A3FB002801D0032002BD002002BDB2
:1025E000F0B587B003A80FF24C1191EC030A80EC10
:1025F000030A0FF24C100068029003A9012001F0B9
:10260000ECFC02A9062001F0E8FC02F050FE441E9A
:10261000A441E40F02F045FE012801D1012000E0B1
:102620000020DFF8685C6978A14200D06C702978DE
:10263000814200D02870DFF8106C05200020C046D1
:10264000002816D1DFF8480C02900020F063B6F89D
:102650004000401CA6F8400080B240F2EF218842C2
:102660004BDB0FF2E00002F019F80020A6F8400062
:1026700043E096F90800022838D19DED020AD6ED14
:10268000160AB4EE600AF1EE10FA03D1B08F401CC6
:10269000B08701E00020B0879DED020ADFED890AD6
:1026A000B4EE600AF1EE10FA06D4DFED870AB4EE5C
:1026B000600AF1EE10FA03DBF08F401CF08701E0B6
:1026C0000020F087F78FB48F972C01DA972F0FDB5C
:1026D000029802F019FFCDE900013A4621460FF2B7
:1026E000780001F0DBFF0020F06301E00020F063E0
:1026F0000020A6F840000298B065706C006AC468BB
:1027000002F077F930722046DDED021A03A991EC50
:10271000030A02F09FF8B06C2018B06495F901002C
:1027200000F03CFB002801D000F0D0F8002007B0FA
:10273000F0BD0000000000000000000000000000EC
:102740000000000050443A204261726F4469736196
:10275000626C65640000000050443A204241524FD0
:1027600020256420256420256600000010B5DFF8D0
:10277000D84A94F9000000283AD494F90A0094F950
:102780000110814228D1217B0818A07240B23D2857
:1027900001DB3C38A07294F90A100FF2700001F0CE
:1027A0007DFF0020A064DFF87C0C90F9010010F19F
:1027B000010F01D1012010BD94F90110081A02F097
:1027C000CBFE21F0004102F0DFFE40B2012801DB28
:1027D000012010BD002010BDDFF8DC0C90F90120B5
:1027E000914203D0D4E90023C0E90023002010BDAA
:1027F000A06CDFF8581D884205DB0FF21C0001F0C9
:102800004DFF012010BD002010BD000050443A20B3
:102810004E5420256400000050443A204E6F546905
:102820006D6500002DE9F8430026DFF81C4A02E040
:10283000207B4019A07294F90A50002E1DD46078B4
:10284000461B76B2012EF3DA002E16D094F90C70E6
:10285000304602F081FE21F0004102460B469046D0
:102860009946384602F078FE42464B4602F0B8FEE2
:10287000E1D2E81BA0720026DDE73C2D02DBA5F1CA
:102880003C00A072BDE8F18380B5DFF8BC090021EF
:10289000817301210172002141724FF0FF310170FB
:1028A0000F21C17214210173002141730187C1649A
:1028B0004174016541650A4624211430FFF78EFDFD
:1028C000002002BD0000FA430180BB4430B5A5B032
:1028D0000AA85821FFF7F8FD00A82821FFF7F4FD0A
:1028E00020A81421FFF7F0FD0AA800F037FEDFF85A
:1028F000604C0320A4F864009DF8290020709DF826
:1029000029000146C02906D113A9C88DA4F8660084
:10291000086BA066E9E0E02953D100203FE00AA956
:1029200001EB8001D1F80220130223F0FF13120AF9
:1029300002F0FF121A43C1F802204FEA3242C1F8F6
:102940000220D1F80620130223F0FF13120A02F02E
:10295000FF121A43C1F806204FEA3242C1F806209E
:10296000D1F80A20130223F0FF13120A02F0FF121B
:102970001A43C1F80A204FEA3242C1F80A20D1F8BE
:102980000E20130223F0FF13120A02F0FF121A4363
:10299000C1F80E204FEA3242C1F80E20001D142863
:1029A000BDDB50210FF2781001F078FE50220DF1BE
:1029B0002A01601CFFF740FD5120A4F86600A466C0
:1029C00093E0000633D49DF82A008DF8800020A8FB
:1029D0009DF82B104170002181709DF82C10C17062
:1029E000BDF833100A0A027141710DF133018A7882
:1029F0008271C978C1719DF8371001729DF8381045
:102A000041729DF82D1081729DF82E10C1729DF8B3
:102A10002F1001739DF8301041730E2220A9601C05
:102A2000FFF70AFD0F20A4F86600A4665DE0DDF85C
:102A30002A10080C8DF8000000A80A0A4270817064
:102A4000DDF82E100A0CC2700A0A02714171DDF81D
:102A500032100A0C82710A0AC2710172DDF8361056
:102A60000A0C42720A0A8272C17213990A0C02732A
:102A70000A0A4273817313A90A79C2734A790274EC
:102A8000CA88130A8DF811308274097A8DF81310F0
:102A9000DDF83A100A0C02750A0A8DF815208175C6
:102AA000DDF83E100A0C8DF817200A0A8DF8182060
:102AB0008DF81910DDF842100A0C82760A0A8DF89A
:102AC0001B208DF81C10DDF846100A0C8DF81D2017
:102AD0000A0A82778DF81F10202200A9601CFFF7D8
:102AE000ABFC2120A4F86600A466DFF85C07406C0C
:102AF000B4F86620D11C418200218182C182DFF8B6
:102B0000585A0120287068700320A870A16EE81C34
:102B1000FFF792FC2946242001F0B4F925B030BD1E
:102B200050442053462053656E7425640000000015
:102B300038B5DFF814374FF46164C1EB0115AD000F
:102B400014FB005414194FF47A756C43DC611B7C40
:102B5000009313460A4601460FF2080001F09EFD5D
:102B600031BD000050443A204254202564202564A1
:102B70002025642025640000F8B52DED028BA0B05F
:102B8000DFF8DC66314684B068464422FFF764FC17
:102B90000FBC00F093FC10EE100A02F0B5FC41EC03
:102BA000100B9FED7C8BDFF8A046256A53EC102BB1
:102BB00051EC180B02F02CFD02F0E6FC15FA80F047
:102BC00020624FF6FF75A84200D32562314684B0DB
:102BD00068464422FFF740FC0FBC00F025FC10EED5
:102BE000100A02F091FC41EC100B676A53EC102BB9
:102BF00051EC180B02F00CFD02F0C6FC17FA80F045
:102C00006062A84200D3656200200E9002200D9001
:102C1000314684B068464422FFF71EFC0FBC00F02A
:102C20008BFAE18A4018E08280B2FF2801DBFF20A6
:102C3000E08200200E9003200D90314684B068465B
:102C40004422FFF709FC0FBC00F076FAA16A401895
:102C5000A062A84200D3A56200200E9006200D902D
:102C6000314684B068464422FFF7F6FB0FBC00F003
:102C700063FA218B4018208380B2FF2801DBFF20FC
:102C8000208300200E9007200D90314684B06846C6
:102C90004422FFF7E1FB0FBC00F04EFA618B4018B5
:102CA000608380B2FF2801DBFF20608300200E904C
:102CB00008200D90314684B068464422FFF7CCFBD3
:102CC0000FBC00F039FAE16A4018E062A84200D374
:102CD000E56200200E9009200D90314684B06846D0
:102CE0004422FFF7B9FB0FBC00F026FA216B401815
:102CF0002063A84200D325630FA801F07EFE276D54
:102D00001E9802F001FC0022DFF8003D02F080FC7A
:102D100002F03AFC57FA80F02065616D491C61654C
:102D2000B0FBF1F0207500200E9001200D9031468F
:102D300084B068464422FFF78FFB0FBC00F0FCF91B
:102D4000616B40186063A84200D36563E07B00F0CC
:102D5000EAFA20B0BDEC028BF1BDDFF8EC04C18AC9
:102D6000002914D1816A002911D1018B00290ED1CB
:102D7000418B00290BD1C16A002908D1016B0029C0
:102D800005D1406B401E8041C043C00F70470120F9
:102D90007047000000000000000059402DE9F04F8E
:102DA000A1B006460025B246DFF89C44A07B314620
:102DB000884205D0BAF1010F78D1284602F0C2F955
:102DC0000FA801F01AFEDFF8989428460E90012013
:102DD0000D90494684B068464422FFF73DFB0FBC86
:102DE00000F0AAF907469DED1E0AD9ED0F0A30EE54
:102DF000600A10EE100A02F087FB2A46DFF80C3C4E
:102E000002F006FC02F0C0FB80461FFA88F8B9F811
:102E10000200BDF83E10A1EB000B5FFA8BFBD9F866
:102E20001020139B9A4207D1884205D1B9F80A00B5
:102E3000BDF84610884210D00FF27022D2E900018E
:102E4000CDE90001139800901398D9F81010401A9A
:102E5000019000A9452001F015F8002E36D1002F71
:102E600002D15BEA080000D001250020A0644FF0E9
:102E7000FF302070D4E90001DFF83C26C2E90001F0
:102E8000DFF8782CC2E90001DFF89825C2E90001DB
:102E9000E07AA072A07B002851D00020A073207C93
:102EA00000284CD001206074054648E0002E07D170
:102EB0000FF2002001F0F2FB012002F043F97FE75E
:102EC0000FF2FC1001F0EAFB2846EBE00FF20C22B7
:102ED000D2E90001CDE9000100A802F0FEF900F0FE
:102EE000BAF9002817D0DDE90001C4E9000128463D
:102EF0006072D4E90001DFF8C025C2E9000194F94D
:102F0000023094F9012094F900100FF2D81001F06A
:102F1000C5FBFFF787FCDDE90001C4E90001FFF70D
:102F200025FC00280BD0D4E90001DFF8F824C2E921
:102F30000001207C002801D0012060740125BAF135
:102F4000010F06D1A07B3146884202D000F058FA2A
:102F5000A673BAF1010F56D1002F54D0DFF89C6B45
:102F6000E07B217C08430AD101202074D4E90001D0
:102F7000C6E90201A27861782078FFF7D9FD94F9BB
:102F8000010096F90910401A411E222901D20120A0
:102F900005E010F1230F01DA012000E000200128F4
:102FA0002AD1FFF7DAFE002826D0E07B401CE07330
:102FB000C0B2152809D10FF2441001F06FFB0120B7
:102FC00060741420E073012516E000202065606520
:102FD0000246242104F11400FFF700FA207C401C73
:102FE0002074A27861782078FFF7A2FD062221469E
:102FF00006F10800FFF730FAFFF7BEFD44220FA9E3
:103000004846FFF729FA607B012834D1208F002839
:1030100005D10FF6443001F041FB012523E0E16CBE
:10302000814218D2002F02D15BEA080000D00125AE
:10303000DFF8C86A96F9020094F90220904212D093
:10304000491CE1640FF6243001F028FBD4E90001AB
:10305000C6E9000107E0002060732087E0640FF6F6
:103060001C3001F01BFBBAF1010F04D1207C0028B9
:1030700001D0012060742846012801D10021A164FB
:10308000616C496A002906D10021A164012801D19F
:1030900000F0B6F90025002D03D1A07C012800D155
:1030A0000125284621B0BDE8F08F00000000000097
:1030B0000000000050443A206C63646F6E00000012
:1030C00050443A206249734150536C656570696E93
:1030D000672077726F6E6720256400000000000093
:1030E0000000000050443A2054696D654E6F7469C9
:1030F00020256420256420256400000050443A20E7
:1031000042542042462046554C4C000080B50020D9
:103110004D49886400F002F8002002BD00B591B06E
:1031200000A801F06AFC442200A94D48FFF794F979
:10313000012011B000BD00000FB410B592B0002402
:103140009DF9980001280BD101F040FD18998842A3
:1031500002D3441AE4B271E08038441AE4B26DE05C
:1031600000A801F04AFC9DF99400401E082865D88B
:10317000DFE800F02905111D2935414D590005985A
:103180001999884201D3441A58E0DFF878291018B9
:10319000401A441C52E006981A99884201D3441AF6
:1031A0004CE0DFF860291018401A441C46E00798EC
:1031B0001B99884201D3441A40E0DFF848291018CF
:1031C000401A441C3AE004981899884201D3441AE2
:1031D00034E0DFF830291018401A441C2EE008981B
:1031E0001C99884201D3441A28E0DFF818291018E6
:1031F000401A441C22E009981D99884201D3441AC0
:103200001CE0DFF800291018401A441C16E00A9848
:103210001E99884201D3441A10E0DFF8E8281018FC
:10322000401A441C0AE00B981F99884201D3441AA3
:1032300004E0DFF8D0281018401A441C204612B0D1
:1032400010BC5DF814FB0000641B00200120DFF8B7
:10325000B81848727047DFF8B008407A704700002D
:10326000A06F002001F0D3BB0146DFF89C2879292C
:1032700002DB7820108700E01087012050730FF6E2
:10328000101001F00BBA0000101C0020F07100209B
:1032900000007A4410B5040001D1012402E0072C9B
:1032A00000DB062421460FF6FC0001F0F7F9641E4E
:1032B000052C2DD8DFE804F0030A11181F26DFF8CB
:1032C00048083721C1723C21017321E0DFF838083A
:1032D0001921C1721E2101731AE0DFF82C080F2199
:1032E000C1721421017313E0DFF81C080A21C172B6
:1032F0000F2101730CE0DFF810080721C1720C21C7
:10330000017305E0DFF800080521C1720A2101738D
:10331000DFF8F407C17A8172BDE81040FFF782BA86
:10332000DFF8E807704700EB80018800821CDFF8B7
:10333000DC07DFF8D417CB691B0E92B21354521C72
:10334000CB691B0C92B21354521CCB691B0A92B26C
:103350001354521CCB6992B21354521C0B6A1B0AB1
:1033600092B21354521C0B6A92B21354521C4B6A01
:103370001B0A92B21354521C4B6A92B21354521C41
:10338000CB8A92B21354521C8B6A1B0A92B213540A
:10339000521C8B6A92B21354521C0B8B92B2135470
:1033A000521C4B8B92B21354521CCB6A1B0A92B222
:1033B0001354521CCB6A92B21354521C0B6B1B0A4F
:1033C00092B21354521C0B6B92B21354521C0B7DCD
:1033D00092B21354521C4B6B1B0A92B21354521CE0
:1033E0004B6B92B21354501C4887704710B5DFF8EE
:1033F0001847618F0FF2B87001F050F9608F10BD5F
:1034000010B5DFF804470022242104F11400FEF770
:10341000E5FF0020E0730120608700202074206514
:10342000606510BD947100200FB400B591B000A884
:1034300001F0E3FA9DED0C0ADDED1E0AB4EE600A20
:10344000F1EE10FA02DB30EE600A05E09FED411A62
:1034500071EE600A30EE800A10EE100A02F054F8A5
:10346000DFF8AC26DFF8AC3602F0A4F902F016FA69
:1034700002F04AF80022DFF8A03602F0C9F802F0A4
:1034800083F800EE100AB8EEC00A10EE100A02F03F
:103490003BF8DFF87C26DFF8843602F0B9F8DFF875
:1034A0008026DFF8803602F085F902F0F7F900EEA9
:1034B000100A11B05DF814FB8C7100200FB400B538
:1034C00091B000A801F099FA9DED0E0ADDED200AF9
:1034D000B4EE600AF1EE10FA02DB30EE600A05E0AD
:1034E0009FED1C1A71EE600A30EE800A10EE100A91
:1034F00002F00AF8DFF81826DFF8183602F05AF959
:1035000002F0CCF902F000F80022DFF80C3602F0ED
:103510007FF802F039F800EE100AB8EEC00A10EE9B
:10352000100A01F0F1FFDFF8E825DFF8F03502F0CE
:103530006FF8DFF8EC25DFF8EC3502F03BF902F02C
:10354000ADF900EE100A11B05DF814FB40771B00D6
:10355000946E0020002474496C62002070B52DED3B
:10356000068BA0B004460FA801F047FADFF8985583
:10357000687B012804D1288F002801D100206873BE
:10358000A87C01280AD1E0206070502205F15C017E
:10359000A01CFEF751FF0020A874C2E1687C01283E
:1035A00016D1287C002813D0C0216170DFF85C158B
:1035B000C0220A70487004F12406FFF717FFF08557
:1035C000FFF7AEFE3063FFF71BFF00206874A8E131
:1035D0009FEDD68B9FEDD79BDFF84C5500200E90CA
:1035E00001200D90294684B068464422FEF734FF3E
:1035F0000FBCFFF7A1FD0A2880F0BE80002060709C
:103600000E9002200D90294684B068464422FEF7B1
:1036100023FF0FBCFFF790FD617808436070002026
:103620000E9003200D90294684B068464422FEF790
:1036300013FF0FBCFFF780FDA07000200E90042048
:103640000D90294684B068464422FEF705FF0FBC62
:10365000FFF772FDE07000200E9005200D902946C6
:1036600084B068464422FEF7F7FE0FBCFFF764FD06
:103670002071294684B068464422FEF7EDFE0FBC57
:10368000FFF71CFF10EE100A01F03EFF41EC100B9B
:1036900053EC102B51EC190B01F0BAFF01F074FF41
:1036A000A4F80B0004F10B061E9801F02DFF53EC5B
:1036B000182B01F0ADFF01F067FFB070BDF83E00C0
:1036C000F070294684B068464422FEF7C5FE0FBC60
:1036D000FFF7AAFE10EE100A01F016FF41EC1A0BDC
:1036E00053EC1A2B51EC190B01F092FF01F04CFF37
:1036F000E0731F9801F008FF53EC182B01F088FFCE
:1037000001F042FF207400200E9006200D90294603
:1037100084B068464422FEF79FFE0FBCFFF70CFD05
:10372000607100200E9007200D90294684B06846F5
:103730004422FEF791FE0FBCFFF7FEFCA0710020B3
:103740000E9008200D90294684B068464422FEF76A
:1037500083FE0FBCFFF7F0FCE07100200E90092003
:103760000D90294684B068464422FEF775FE0FBCD2
:10377000FFF7E2FC2072D2E08020607000200E9003
:1037800002200D90294684B068464422FEF764FE6C
:103790000FBCFFF7D1FCC4F8020000200E900320FC
:1037A0000D90294684B068464422FEF755FE0FBCB2
:1037B000FFF7C2FCC4F8060000200E9004200D9014
:1037C000294684B068464422FEF746FE0FBCFFF748
:1037D000B3FCC4F80A0000200E9005200D90294685
:1037E00084B068464422FEF737FE0FBCFFF7A4FC06
:1037F000C4F80E00294684B068464422FEF72CFE29
:103800000FBCFFF75BFE10EE100A01F07DFE41ECED
:10381000100B53EC102B51EC190B01F0F9FE01F0D9
:10382000C9FE606204F124061E9801F06DFE53EC9F
:10383000182B01F0EDFE01F0A7FE3071BDF83E003F
:103840007071294684B068464422FEF705FE0FBC1D
:10385000FFF7EAFD10EE100A01F056FE41EC1A0BDC
:10386000DFF8C822DFF8C83202F060F808D8DFF8C5
:10387000C422DFF8C43201F0B3FE01D29FED64AB85
:1038800053EC1A2B51EC180B01F0C2FE01F07CFE38
:10389000F0801F9801F038FE53EC182B01F0B8FEB1
:1038A00001F072FE307200200E9006200D90294625
:1038B00084B068464422FEF7CFFD0FBCFFF73CFC06
:1038C000C4F8120000200E9007200D90294684B005
:1038D00068464422FEF7C0FD0FBCFFF72DFCC4F87C
:1038E000160000200E9008200D90294684B06846EE
:1038F0004422FEF7B1FD0FBCFFF71EFCC4F81A000E
:1039000000200E9009200D90294684B0684644227C
:10391000FEF7A2FD0FBCFFF70FFCC4F81E00FFF777
:10392000FDFB20B0BDEC068B70BD00000000000068
:1039300000002440000000000000594070B582B033
:1039400004460020002C05D10FF2782000F0A6FEDE
:10395000002076BD04F150014978012948D10FF2C9
:10396000782000F09BFE0020ADF80000734D664EFD
:1039700017E0BDF8000006EB8000C26500EE102ADB
:10398000B8EE400ADFED5E0A20EE200ABDF8000026
:1039900005EB800080ED000ABDF80000401CADF88A
:1039A0000000BDF8000014281CDABDF8000054F82F
:1039B0002020A2F52F70B0F5167FDAD9BDF80010DF
:1039C0000FF2202000F06AFEBDF800004FF07E519B
:1039D00045F820104FF47A70BDF8001006EB810115
:1039E000C865D9E701202865284601F0ADFB0BE04A
:1039F000022909D194F850100FF2FC1000F04EFE8D
:103A000094F850000120C046C0B276BD00002440AA
:103A10009A9999999999B93F80B5112802D110784E
:103A2000FFF722FC002002BD30B595B014461028E7
:103A30001FD014280AD015280DD0162810D017280A
:103A400013D0292843D1FFF701FC40E02178002062
:103A5000FFF708FC3BE021780120FFF703FC36E08C
:103A600021780220FFF7FEFB31E02078FFF712FCFF
:103A70002DE000A85421FEF727FD217814AD6970D0
:103A80000FF2C00000F00AFE6878012817D100206C
:103A90000FE004EB80014A788B781B0403EB026291
:103AA000CB7802EB03220979511800AA42F82010C2
:103AB000401C1428EDDB00A8FFF740FF07E00228B8
:103AC00005D160788DF8500000A8FFF737FF00207F
:103AD00015B030BD0C494864B831C1612421017072
:103AE00014218160012101730182002141828182C0
:103AF000C182134981610020704700004871002095
:103B00006F12833A80969800641B0020A860002002
:103B10007B14AE47E17A743F00005940E17A843F5C
:103B20002D431CEBE2361A3FA06F0020B81E85EB38
:103B300051B89E3F9A9999999999B93F141E0020BE
:103B40006C62002050443A2050726F706572747934
:103B5000205346202564000050443A2052657120CD
:103B60005065646F496E666F3100000050443A2022
:103B70007574696D657220256400000050443A2018
:103B8000526571205065646F496E666F32000000A7
:103B900050443A205374617274204461746120254A
:103BA0006400000050443A20555420256400000071
:103BB00050443A204241544C454E475448202564D5
:103BC0000000000050443A20534620505452332005
:103BD0006E756C6C0000000050443A205346205330
:103BE0004554310050443A205346204552525B25FB
:103BF000645D20256400000050443A205346205361
:103C0000455432202564000070B5002420E02C20AB
:103C100001F0A4FE054600222C21FEF7DFFB28461A
:103C20000FF2AC6151F826108847DFF84866287813
:103C300046F820500020E96909688847002806D026
:103C40000020297846F82100284601F09FFE641CD8
:103C5000E4B22646172EDADB002070BD10B46FF0F8
:103C600000410846002210E0DFF8083653F8223001
:103C7000002B09D01C6A002C06D0DB78002B03D166
:103C8000E368984200DD1846521C602AECDB88424B
:103C900000D1002010BC7047F8B506460F4600F072
:103CA000E4F8040001D10320F2BD251D6868002856
:103CB00001D0B8607860786801F04CFB7860B96832
:103CC000002902D0084601F045FBB860394604F1EE
:103CD000200001F063FF94F82800012807D100209C
:103CE000A9694968884701F0E9FF606008E0E07869
:103CF000012805D13878002802D1304602F058F862
:103D0000002211462E20AB691B699847DFF8681521
:103D1000022002F077F80020F2BD70B50D4600F0E9
:103D2000A4F8060007D006F11C04287800280AD160
:103D3000A068002801D1032070BDC0686860A06839
:103D40000069A86007E0686801F004FB6860A86883
:103D500001F000FBA860294606F1200001F03EFFBB
:103D6000F369207B002803D10020D968884704E04C
:103D7000002211462E201B699847DFF8FC14022010
:103D800002F040F8002070BD38B50C4600F06DF828
:103D90000546606801F0DEFA6060A168002902D083
:103DA000084601F0D7FAA060002D02D0686A00280A
:103DB00001D1032032BDC1686268914205D1016919
:103DC000A268914201D1002032BD00F1080105F145
:103DD000200001F003FF002811D1214605F1200049
:103DE00001F0DCFE002211462E20EB691B6998478A
:103DF000DFF88414022002F005F8002032BD032011
:103E000032BDF8B504460D4616461F4600F02DF8A3
:103E1000002801D10120F2BD3A4631462846DFF89C
:103E2000543453F82430DB691B6998470020F2BDF5
:103E3000F8B504460D4616461F46192D03D101213B
:103E400002F012F80FE000F010F8002801D1012074
:103E5000F2BD3A4631462846DFF8183453F824308C
:103E6000DB695B6998470020F2BD0146602901DAF1
:103E7000002801D100207047DFF8F80350F8210036
:103E80007047000070B52DED028B0C46DFF8E4138F
:103E900051F8205001280FD0042845D0052868D0BB
:103EA00008287AD01D2800F08A80422800F07F8000
:103EB000452800F0898021E09FED5E0ADFF8BC63B1
:103EC000B4F9000000EE900AF8EEE00A60EE800A15
:103ED000C6ED000AB4F9020000EE900AF8EEE00A1E
:103EE00060EE800AC6ED010AB4F9040000EE900A03
:103EF000F8EEE00A20EE800A86ED020A002D10D0CE
:103F0000686A00280DD04069DC49896C401A012894
:103F100007DA214605F1100002F008F801F0D0F9A7
:103F20006860BDEC028B70BD9FED438BD34EB4F93E
:103F3000000001F011FB53EC182B01F069FB01F0BC
:103F4000ADFCF060B4F9020001F006FB53EC182B55
:103F500001F05EFB01F0A2FC3061B4F9040001F055
:103F6000FBFA53EC182B01F053FB01F097FC706146
:103F7000C4E7C24E206870626068B0622089B08574
:103F80006089F085A0893086E0897086207C86F87B
:103F90003400607C86F83500B0E7B84E207886F8AB
:103FA0003800607886F8390060887087A6E7B34EDD
:103FB0002068B0616068F061A06830629EE7207898
:103FC000AE4981F83C0099E708222146AC48BDEC97
:103FD000028BBDE87040FEF72FBA02460846012A60
:103FE0000CD0042A0ED0052A10D0082A12D01D2A7F
:103FF00018D0422A12D0452A18D070470C229F4967
:10400000FEF71ABA0C229F49FEF716BA14229E49EF
:10401000FEF712BA04229D49FEF70EBA0C229C4903
:10402000FEF70ABA01229B49FEF706BA0822944914
:10403000FEF702BAFDF61C3B0597A11D4F04443F55
:1040400010B5082802D0102823D010BD0FF24C2044
:1040500000F024FB0120FFF708FF03460022114671
:104060002F20DB691B6998472920FFF7FEFE90F897
:104070002800002801D002F06EFA1120FFF7F5FEAB
:10408000044694F82800002827D0BDE8104002F02C
:1040900096BB0820FFF7E9FE044601F011F96168BC
:1040A000401AE16989688847002816D1606A0028AB
:1040B00007D0C1680069814203D10021082001F0C6
:1040C000D3FE5920FFF7D1FE044694F828000028BB
:1040D00003D0BDE8104002F0CFBC10BD2DE9F04385
:1040E00085B0044601A80FF244212CC92CC001F070
:1040F000E7F8054601F0CFF8012801D1012600E0DC
:1041000000265E4884640027DFF8688129E0602F7C
:1041100020DADFF884910120BDF8071001F80900CA
:10412000022200A9BDF807004844401CFEF784F9AC
:1041300058F8270000F11001BDF807004844C01CE2
:1041400001F01FFFBDF80700BDF80010C91C0818DA
:10415000ADF80700214658F82700203001F05BFD3C
:104160007F1C602F79DA58F827000028F8D090F8E3
:1041700028100029F4D0C1780029F1D1011DCA69A5
:104180005269121B012A05DA4068281A401C896905
:104190008968884758F82700416A0029DAD0896978
:1041A000091B0129D6DA002E02D0017B0029D1D0CB
:1041B000103001F032FFADF8000058F82700103041
:1041C00001F04CFFADF80200BDF800000028C1D09E
:1041D000BDF802000028BDD0BDF80700BDF80010F2
:1041E00011FA80F2101DB0F5007F0CDD0FF2B40162
:1041F0000FF2C40000F052FA274901A802F041FF73
:104200000020ADF80700212FBFF681AFDFF88890BE
:104210003720BDF8071001F80900BDF80700484431
:10422000477002220DF10201BDF807004844801CCE
:10423000FEF702F958F8270000F11001BDF8070059
:104240004844001D01F09DFEBDF80700BDF80010B8
:10425000091D0818ADF807007CE7BDF80700002825
:1042600003D00D4901A802F00CFF002005B0BDE805
:10427000F08300003064002030370020546F0020AD
:10428000946F0020606F0020786F00208C6F0020FA
:104290006C6F0020906F0020245900204143432080
:1042A000494E5400636F6C6C6563745F73656E7325
:1042B0006F725F646174610025733A2074785F6483
:1042C0006174612069732066756C6C28256429000F
:1042D00035A30108959501080DA40108CF9A01089E
:1042E00021A70108236F00086B920108CBA40108E5
:1042F000A97F01088F6500089FA50108D53A00082D
:10430000296800089B9E010843A2010855940108F2
:10431000CF9F0108EF960108A1760108AF8F010831
:104320006DA60108A5E700080F9D01080500000023
:104330000000000000000000EFF3038070474FF022
:10434000AC3000787047F8B507460C460025DFF81A
:1043500090646FF01E01401A27D0083825D0001F46
:1043600010D0001F1AD0083818D0001F24D104F133
:1043700020003062EFF3148040F00200F062306AF7
:10438000B06219E004F164003062EFF3148040F091
:104390000200F062306AB06201250DE004F12000F5
:1043A0003062EFF31480F06206E004F164003062E2
:1043B000EFF31480F0620125EFF308807062EFF3F1
:1043C0001080F063EFF311803064EFF313807064BA
:1043D000F1EE100AB064EFF305803063EFF3008074
:1043E0007063FFF7A9FFB063F764002004E054F89E
:1043F000201046F82010401C0828F8D3012D0AD1BF
:10440000002006E004EB8001096A06EB80021165DA
:10441000401C1128F6D3F1BDDFF8C803DFF8C8133C
:104420000A6802604A6842608A688260CA68C2603C
:104430000A6902614A6942610A7E8261097F81617B
:10444000DFF8A8130A7882614A6842628A68826249
:10445000CA68C2620A6902634A6942638A698263FE
:10446000CA69C2638A6EC0F88820DFF88423936922
:10447000C0F89830D368C0F88C301369C0F8903019
:104480005369C0F894300B6FC0F89C304B6FC0F884
:10449000A0308B6FC0F8A430C96FC0F8A810DFF847
:1044A00054130968C0F8AC10DFF84C130B68C0F85F
:1044B000CC304B68C0F8D0308B68C0F8D430CB68B3
:1044C000C0F8D8300969C0F8DC105168C0F8E810AD
:1044D0001168C0F8E410704710B582B0044640F28D
:1044E0000240ADF800000520207000206070A07030
:1044F000022200A9E01CFDF79FFFDD20607113BDC3
:1045000002F032BFA0F10060B0F5003F01D80120F9
:10451000704700207047F8B505460E4614461F4602
:104520002868FFF7EFFF002801D10020F2BD2868BE
:1045300040084000009004203060024600A93888FE
:104540000019FDF779FF0120F2BD2DE9F04182B09D
:1045500080460C4615461E46002738460090B8F1A6
:10456000000F19D0002C01D116E07F1C0C2F12D2A5
:1045700033462A4600A94046FFF7CDFF002803D066
:1045800030880099081830803088142803DA08F140
:1045900004084445E9D20120BDE8F681F8B50C468F
:1045A000154610F1030F02D010F1130F09D1934EED
:1045B000B06802F0E1FE0746B06802F0E9FEC119FA
:1045C00005E002F0F3FE064602F0F2FE81192B46EA
:1045D00022468348806AFFF7B8FF0120F2BD80B50C
:1045E0000021ADF8001000AA01467D48C06CFFF71D
:1045F000D5FF01BD10B582B004461620ADF800000D
:104600000520207000206070A070022200A9E01C2C
:10461000FDF712FF0F2060711420A07113BD70B55B
:1046200088B0724601461046FFF78DFEFFF7F4FE94
:1046300000A81C21FDF748FF00A8FFF7DBFF0DF1E4
:104640000700FFF7CCFF1B2100A802F00AFE0024A0
:104650006B4D2846FFF740FF40F207460CE0AC7177
:104660000A46A00200F10051E81DFDF7E5FE3146C3
:10467000284602F0F6FD641C4FF48061202CEED336
:104680000022E81DFDF728FFDD20A87131462846ED
:1046900002F0E7FDFFF734FF08B070BD0EB470B54F
:1046A000C1B0044600A84FF48071FDF70DFF45AB83
:1046B00022464FF4807100A802F082FE00A802F0AA
:1046C0009DFE441C002000A9611801F8010C4B4D0F
:1046D0002878401C28706878F021084202D0992080
:1046E00002F0A8FE02F01CFF6878401C6870454E7E
:1046F000317808462218FA2A0DDA434A8018002930
:1047000002D00A2100F8011C224600A9FDF794FE00
:104710003078201830706878F021084202D0992053
:1047200002F088FE6878401E6870C0B2002801D18F
:1047300002F0F0FE03F0DEF941B070BC5DF810FB52
:10474000FEB52E4C2078401C20706078F021084285
:1047500002D0992002F06EFE02F0E2FE6078401C6A
:104760006070284D2E78002E28D005208DF800008E
:10477000B01CADF8030080B201F0F0F8CDF80500F0
:1047800000282CD003210170DDF8050046701E4F73
:1047900032463946DDF80500801CFDF74DFE00A9C4
:1047A0001A4803F0CBFA1A49042001F02BFB00222F
:1047B000FA213846FDF712FE002028706078F021BB
:1047C000084202D0992002F035FE6078401E6070E9
:1047D000C0B2002801D102F09DFE03F08BF9F7BDB5
:1047E000106D0020FC68002000ED00E020ED00E0EE
:1047F00004E000E0A0ED00E034EF00E0501F0020F6
:10480000B8520020F3710020006800206C4E002098
:10481000584A0020DFF81809C17B00EB810181EDC7
:10482000050AC17B00EB8101C1ED090AC17B00EBE8
:10483000810181ED0D1A017C042901DA491C017402
:10484000C17B491CC173C9B2042901DB0021C173BA
:1048500070470000F8B52DED068B88B0B0EE408AA9
:10486000F0EE608AB0EE419AF0EE619A04468DED6A
:10487000040AB0EE68AA8DED05AAF0EE49AACDEDC6
:1048800006AA0A26DFF8A858B5F9660010FB06F05C
:10489000B5F96810471A05F1440003F085FA95F858
:1048A000440010FB06F095F845104618B6B22A2EC3
:1048B0000FD13FB2002F0CD56868002806D1012027
:1048C000FDF723FDFDF7F3FC01206860012028605F
:1048D00015E06868012807D1FDF7F4FC0020686046
:1048E0000FF66800FFF7DAFE2868282E3BDA012869
:1048F00003D10FF68400FFF7D1FE0020286095ED6C
:10490000150AF0EE480AB4EE600AF1EE10FA37D15B
:1049100095ED160AB4EE4A0AF1EE10FA30D195ED93
:10492000170AB4EE6A0AF1EE10FA29D1DFF804682A
:104930003068401C306015282CD3E86D00F0E4FD91
:10494000CDE90201A86D00F0DFFDCDE90001686D41
:1049500000F0DAFD02460B460FF62800FFF79EFE38
:104960000020306016E0002805D1002231460FF209
:10497000E870FFF793FE01202860FDF7A7FCBEE773
:10498000049868650598A8650698E8650020DFF832
:10499000A417086004A890EC030AFFF73BFF204629
:1049A00080B2B0EE690A03F017FA214604A8FCF7BA
:1049B0003BFF05F16000FDF7F3FB286E012811D1E4
:1049C000FBF7A9FC05F16000FDF7EAFB2C2205F1DD
:1049D000600105F18C00FDF73FFD0FF2BC70FFF7A1
:1049E0005DFE01E000F000F9002008B0BDEC068B90
:1049F000F2BDDFF83C07807B7047002806D0DFF867
:104A00003017D1F8B8104422FDF726BD704710B515
:104A100000281CD1DFF81847483400EE101AB8EE11
:104A2000400A84ED010A2046FDF7C1FB94ED010A1E
:104A3000F2EE0A0A20EE200A10EE100A00F064FDE1
:104A400002460B460FF25870FFF728FE2FE00128B0
:104A50001CD1DFF8DC4600EE101AB8EE400A84EDF7
:104A6000120A04F14800FDF7A2FB94ED120AF2EEDF
:104A70000A0A20EE200A10EE100A00F045FD024658
:104A80000B460FF22870FFF709FE10E002280ED146
:104A9000DFF89C46483421722046FDF788FB207AD7
:104AA0000D2111FB00F10FF21070FFF7F7FD0FF26F
:104AB0001470FFF7F3FD42F26A7001460FF21070B6
:104AC000FFF7ECFD40F2EE7001460FF21070BDE80A
:104AD0001040FFF7E3BD2DE9F0412DED028B84B0CE
:104AE00006460F4690460FF2DC60FFF7D7FD42F214
:104AF0006A7001460FF2D860FFF7D0FD40F2EE7009
:104B000001460FF2D860FFF7C9FDDFF82446002206
:104B10004FF4E6712046FDF761FC04F58075C4F89A
:104B2000B85000EE106AB8EE408A84ED138A00EEA9
:104B3000107AB8EE400A84ED120A84F85080F2EE42
:104B40000A8A40460D2111FB00F0029020EE280A4F
:104B500010EE100A00F0D8FCCDE9000128EE280A7A
:104B600010EE100A00F0D0FC02460B460FF27C60FB
:104B7000FFF794FDFBF728FB04F14800FDF717FB56
:104B800042F21070A4F8C200A4F8C4000020A4F8F7
:104B9000BC00A4F8BE000220A4F8C6002C2204F138
:104BA000BC012846FDF758FC0220A07303F006F96B
:104BB0000120607304F1440003F0F6F80020606007
:104BC000206004B0BDEC028BBDE8F08110B592B05E
:104BD000FDF790FB044600A8FFF70FFF04980019AB
:104BE00012B010BD000000002DE9F0412DED028B48
:104BF000DFF83C4504F17005E86A216F814205D178
:104C0000B4F866206B8C9A4200F08880B1EB000803
:104C100002D5DFF82405804495ED060AD5ED110A8A
:104C200070EE608AF5EE408AF1EE10FA03D59FED42
:104C3000950A78EE808A95ED040AD5ED0F0A30EEDC
:104C4000608AB5EE408AF1EE10FA03D59FED8D0A29
:104C500038EE008AB4F86600C0B295ED050A03F09C
:104C6000B7F9B0EE401A04F10C067078012802D0B2
:104C700002282BD033E004F5A27739469FED821A43
:104C8000F0EE480AB0EE680A404600F057F8207B84
:104C900040442073C0B2062821DB04F5AA7004F159
:104CA000BC019FED791AD0ED0A0A90ED080AD4F8FC
:104CB000540100F043F8207B401C20730022442163
:104CC0003846FDF78BFB0220707008E004F1BC0150
:104CD000F0EE480AB0EE680A404600F02FF8B4F84B
:104CE0006600002809D10022442104F5A270FDF7D6
:104CF00075FB00202073012070702C2204F16001EC
:104D000004F18C00FDF7A8FB04F1BC01A96404F5D3
:104D1000807644223046FDF79FFBAE6404F16600C6
:104D20004088B4F80A11884203D0A4F8C600A4F859
:104D30000A01BDEC028BBDE8F08100002DE9F041D5
:104D40002DED048B8AB0B0EE409AB0EE608AF0EEA2
:104D5000418A0C46DFF8D87307F164056E88B7F80E
:104D60006480A680B0EE680A00F0BDF8B86800283C
:104D700019D194ED0C0A30EE090A84ED0C0A00F00A
:104D8000AFF984ED0C0A6680A4F80080A86960631E
:104D900094ED0E0A30EE080A84ED0E0A00F094F944
:104DA00084ED0E0A4AE007F1480007AA0AC80AC2C1
:104DB0000368136007F1600184B068462C22FDF798
:104DC0004BFB0FBCB0EE680A00F030F9D4ED0C0AD2
:104DD00030EE800A84ED0C0A00F082F984ED0C0AB2
:104DE000F5EE408AF1EE10FA0BDD032E03D106201A
:104DF0006080208010E0042E0ED10820608020808A
:104E00000AE0032E03D107206080208004E0042EF6
:104E100002D1092060802080F6EE000A95ED060A96
:104E200020EE200A84ED0D0A94ED0E0A08EE200A09
:104E300084ED0E0A00F048F984ED0E0A95ED080A9B
:104E4000DFEDB00A20EE200A84ED0F0ADFEDAE0A96
:104E5000B4EE600AF1EE10FA01DBB848E06368696D
:104E600020646088002801D1002020642869E06067
:104E700028892081A88860810AB0BDEC048BBDE838
:104E8000F0810000002474490000000010B50C46B9
:104E9000A188032912D1B5EE400AF1EE10FA06DD21
:104EA000216A4018206200F027F9206210BD616A73
:104EB0004018606200F020F9606210BD042911D131
:104EC000B5EE400AF1EE10FA06DDA16A4018A062C4
:104ED00000F012F9A06210BDE16A4018E06200F033
:104EE0000BF9E06210BDF8B52DED028B0546B0EE72
:104EF000408A0C4620692818206100F0FDF82061E6
:104F0000B5EE408AF1EE10FA02DDB0EE480A01E09B
:104F1000B1EE480AB5EE400AF1EE10FA43DD844ED8
:104F2000B068002830D106F5CE77B86806280ED2D2
:104F30006188042903D179686918796004E0D6F89A
:104F40009C116918C6F89C112818B86051E0E169F5
:104F50004018E06100F0D0F8E0612146B0EE480A68
:104F6000B868FFF793FFE0692818E06100F0C4F823
:104F7000E0612146B0EE480A2846FFF787FF00F0BF
:104F80003BF80120B06034E0E0692818E06100F0EF
:104F9000B3F8E0612146B0EE480A2846BDEC028B2A
:104FA000BDE8F44072E76088032802D0042807D0E7
:104FB0000DE060692818606100F09EF860610CE007
:104FC000A0692818A06100F097F8A06105E0606969
:104FD0002818606100F090F86061554E06F5CE70BB
:104FE0008068002801D000F010F800F005F80020DB
:104FF000B060BDEC028BF1BD4D480021C0F89C11A2
:1050000000F5CE704160816070474948D0F8D010FB
:10501000D0F89C215118C0F8D01000F1D0014A6896
:10502000D0F8A00180184860704700000FB4DFED91
:10503000370A9FED361AF0EE0C1A9DED092ABDF8DD
:10504000060004280FD1DFED322A42EE221AB5EE17
:10505000400AF1EE10FA15D49FED2E1A22EE011A35
:1050600021EE001A0EE0DFED2C2A42EE221AB5EEF8
:10507000400AF1EE10FA05D49FED281A22EE011A2B
:1050800021EE001AB5EE402AF1EE10FA0ED09DED99
:10509000060AB5EE400AF1EE10FA07D0DFED200A5D
:1050A00020EE200AF7EE000AC0EE800A31EE810AF7
:1050B0009FED1C1A20EE010A9DED0B1A20EE010A4D
:1050C00020EE200A04B07047DFED170AB4EE600A44
:1050D000F1EE10FA03DBDFED150A30EE200A70471F
:1050E000DFED110AB4EE600AF1EE10FA03DBDFED3A
:1050F0000F0A30EE200A70470F49884201D3104949
:10510000081870478FC2753D0100C84100000000BB
:10511000CDCC4C3E6666663FCDCCCC3D6666E63F68
:10512000000070420AD7A33B01247449002474C9CB
:10513000DC5E0020C8710020819698000000C84104
:10514000806967FFFDF7FAB8FDF73BB850443A2095
:1051500042505F4F4646000050443A2053746570F9
:10516000436E7455702056482825642920435943BE
:10517000282564290000000050443A20455849542D
:105180002056480050443A204E41432025662025B1
:10519000662025660000000050443A204F46520029
:1051A00050443A20312025660000000050443A2047
:1051B000322025660000000050443A203320256448
:1051C0000000000050443A2030324645423135005C
:1051D00050443A204D50445F7625640050443A20B4
:1051E00050524950445F76256400000050443A20F4
:1051F00031202566203220256620332025640000DA
:105200005148006870471FB5044601A800210A46AE
:105210000B460EC0FFF7F4FF00900522214601A8BF
:10522000FDF70AF90420ADF8070000A901A801F074
:1052300028FF1FBDF0B587B0044602A800210A462A
:105240000B460EC00846CDE90001012510E02846B6
:10525000FEF70BFE00280AD0DDE9006701200021DF
:105260002A4603F085F830433943CDE900016D1C2F
:10527000212DECDB0522214602A8FDF7DDF80820F0
:10528000ADF80B0000A902A801F0FBFE07B0F0BDCD
:105290002E49087070472D48007870472B49487098
:1052A00070472A48407870472849887070472748D7
:1052B000807870472549C87070472449C860704796
:1052C0002248C0687047214902780A7142784A71C1
:1052D0008078887100200881704706221C49FDF7FC
:1052E000ABB81A4A1369002B01D0CB1A00E0034671
:1052F000B3F57A7F00D3034610891818108100B2E5
:10530000B0F57A7F05DBA0F57A7010819079401CAA
:10531000907192F906003C2804DB3C38907150797A
:10532000401C507192F905003C2804DB3C38507158
:105330001079401C107192F90400182801DB00203C
:105340001071116170470000D025002010710020FD
:1053500014710020B0F5A07F02DB4FF4A0707047FD
:10536000A02801DBA0207047502801DB50207047A7
:10537000282801DB28207047142801DB14207047FF
:105380000A2801DB0A2070470520704710B586B057
:1053900002A80FF25C111CC91CC000A800210A461B
:1053A00006C003F001F801788DF8001000A9C2785A
:1053B0004A7042798DF802208079C87001208DF8FA
:1053C00004000520ADF80B0002A801F05AFE06B05B
:1053D00010BD30B59DB003A86421FDF775F800A895
:1053E0000FF218111CC91CC00024FF226421FCF715
:1053F000F5FF012515E02846C0B2FEF736FD00286E
:105400000ED02946491E012904D9C91E022901D9F5
:10541000091F05D103A964B26554408A401C0419D0
:105420006D1C092DE7DB64B2ADF8034003A900A8A9
:1054300001F027FE00201DB030BD10B50446A07855
:105440000146491E01290FD9091F012914D9891EB6
:10545000012919D9891E01291ED9203923D1D4F84F
:105460000500FFF730FF1EE0012801D1002000E019
:105470000120FFF70DFF16E0052801D1012000E013
:105480000020FFF711FF0EE0072801D1012000E006
:105490000020FFF70FFF06E0092801D1002000E0FF
:1054A0000120FFF7FBFEA0781438032801D9153836
:1054B0000ED12420FEF7D9FC030009D0D4F8052032
:1054C000B4F80310A078DB691B69BDE810401847E9
:1054D00010BD81780C2906D0182906D01B2903D0CD
:1054E0002C2903D070478EE6A4E64FE771E7000051
:1054F00004FF1800000000000000000004FF2C0062
:1055000000000000000000005FF0FF0C1CEAD0511A
:1055100014BF614506E0C110400721F0E04101F1F0
:105520006051704779B900F0004100020AD0B0FA2A
:1055300080FC00FA0CF001F16051A1EB0C5101EB81
:10554000D0214005704741020CBF40F4E0016FF0EC
:105550000001002070470000010040F10980F4467E
:10556000404200F005F851F000416047010000BFE3
:1055700009D0B0FA80F18840C91CC1F584610905E1
:1055800001EBD02140057047F446400D40EAC120B0
:10559000490006D200F014F8004248BF6FF0004006
:1055A000604700F00DF84FF0004188428CBF08467C
:1055B00040426047400D40EAC120490080F00D8024
:1055C00040F00040490DA1F58061491C05D4D1F19E
:1055D0001F0154BFC840C01770474FF0000070470C
:1055E0004FF4001C1CEB410F94BF1CEB430F09E070
:1055F00041EA030C50EA4C0C52EA0C0C03D29942DB
:1056000008BF9042704714BF8B428242704700002F
:10561000B0B581EA030C0CF0004C40F2FF7515EABE
:1056200011541DBF15EA1357AC42AF4239E0E419DB
:1056300023EA455343F48013C90241F0004141EA93
:10564000505EC7021100A7FB020200284FF00000C5
:10565000EEFB01204FF00001E3FB072118BF42F0F1
:105660000102401800214941E3FB0E01A4F58064CA
:105670000F0302D252004041494154F101046CDD54
:10568000470872F1004250F1000051EB0451A1F5BE
:1056900080115CBF41EA0C01B0BD4CEA055100200D
:1056A000B0BD05EA1357AC4214BFAF4241E050EA27
:1056B000410E1CBF52EA430E02E061460020B0BD1D
:1056C00024423C441BD15FEA070EF6D0090302BF17
:1056D00001460020AEF1140EB1FA81F7AEEB0704DB
:1056E00001FA07FE0C37C7F1200100FA07F7C8409E
:1056F0004EEA000E23EA455343F48013A2E733F049
:105700000043B3FA83F704BFB2FA82FE77440B3F3B
:10571000E41BB7F1200E2FBF02FA0EF3BB40C7F116
:10572000200E22FA0EFE38BF43EA0E03BA40641C74
:1057300082E750EA410E14BF52EA430E6FF00001B7
:105740004FF4001717EB430F8ABF194617EB410FB1
:10575000B5E74CEA05510020B0BDD4F10104B4F125
:1057600020070FDAC4F12007520828BF42F00102D7
:1057700010FA07F501FA07F7E1BF2A43E040384382
:10578000E1400FE0352C98DCC7F1200452EA4002DA
:1057900020FA07F218BF42F0010231FA07F0A140E7
:1057A0000A43002172F1004250F1000051EB0C015C
:1057B000B0BD000070B44FF0004591EA030C44BF47
:1057C0006B4002F09BBE00BF841A71EB030603D24C
:1057D000001BB141121973414FF4001C1CEB410F27
:1057E00034BF7CEB430443E00C0DA4EB1356352E81
:1057F00050DC45EAC323DB0A45EAC121C912B6F1F0
:1058000020050DDD63FA05F6EB4086EA030512423A
:1058100018BF45F00105C01851F100010CD213E08A
:1058200062FA06F5F2405540F3415A40B340F34066
:105830005A408018594107D349085FEA30005FEAAF
:10584000350528BF45F0010501F58011420875F1C5
:10585000004250F1000041EB045170BC4FF4001CB9
:105860001CEB410F38BF70470020090D0905704738
:105870001CEB410F10D252EA43060BD0BCEB410F98
:1058800005D80C0DAB43661E342EB5DD02E0AB43EC
:105890008018594170BC704770BC70474FEAF17C6A
:1058A000BCF1E04C2CBFBCF5001F11E05FEA4C0CD2
:1058B00034BFBCF17F5F2EE05FEA9C0C4FEA0C1C0A
:1058C0004FEA3C0CC10071F100414CEB5070704745
:1058D000C90241EA5051C00218BF41F0010141F034
:1058E00000414FEA6C50C0F10900212810D240EA73
:1058F000CC7CCCF1200C11FA0CF070F10040CCF112
:10590000200C21FA0CF00CF0004C40EB0C0070471E
:105910004FEACC707047490011F5001F04D84FEAD8
:10592000CC10FF30C0057047C81770474FF4001CFB
:105930001CEB410F94BF1CEB430F09E041EA030C41
:1059400050EA4C0C52EA0C0C03D28B4208BF824244
:10595000704714BF994290427047000010B5040090
:1059600010480078002805D10F4802F0A2FE0D482B
:10597000012101700C4802F0D6FE200003F0D3FD97
:105980000400094802F003FF200010BD10B5040018
:10599000054802F0C8FE200003F025FF024802F08F
:1059A000F6FE10BDFD7100202471002038B50446BC
:1059B000002500E06468002C0CD0207A0A78904220
:1059C000F8D1E0684A689042F4D120698A68904230
:1059D000F0D101252A460FF2C8210FF2D020FEF7A0
:1059E0005DFE002D00D10024204632BD38B50446AE
:1059F0002020FFF7B3FF054600222021FCF7EEFC34
:105A00000C22214605F10800FCF726FD606868615C
:105A1000A068A86101202877284632BD2DE9F84307
:105A200005460E460027B84606F108099B4C20782B
:105A3000401C20706078F021084202D0992001F0CB
:105A4000F9FC01F06DFD6078401C60702868D9F8A1
:105A5000041001E080464068002803D0C2689142EB
:105A6000F8DA0127002F0AD0016831607060016800
:105A7000002901D04E6000E02E60066008E0B8F119
:105A8000000F04D0C8F80460C6F8008000E02E6063
:105A90006078F021084202D0992001F0CBFC6078B8
:105AA000401E6070C0B2002801D101F033FD02F049
:105AB00021F80020BDE8F28370B506460D46774C0C
:105AC0002078401C20706078F021084202D0992094
:105AD00001F0B0FC01F024FD6078401C6070686843
:105AE0002968002901D0486000E03060686800281B
:105AF00001D0296801602846FFF748FF6078F0214F
:105B0000084202D0992001F095FC6078401E607038
:105B1000C0B2002801D101F0FDFC01F0EBFF002034
:105B200070BD70B505462E68002E00D16E68002E3F
:105B300033D05A4C2078401C20706078F021084205
:105B400002D0992001F076FC01F0EAFC6078401C5C
:105B50006070F0687169401AE9680A1A90FBF1F305
:105B600001FB0321696129690A1A90FBF1F001FB2D
:105B70000020A8616078F021084202D0992001F04D
:105B800059FC6078401E6070C0B2002801D101F05D
:105B9000C1FCBDE8704001F0ADBF70BD70B50446FA
:105BA0000D462068FFF702FF06000BD12846FFF7DD
:105BB0001DFF064631462046FFF730FF3046FFF70F
:105BC000B0FF02E0307F401C3077207A401C20720A
:105BD000307A002800D16660002070BD10B5044600
:105BE0002068FFF7E3FE002801D1032010BD017FEC
:105BF000491E0177217A491E2172017A002901D1BB
:105C000000216160017F002903D101462046FFF792
:105C100053FF002010BD70B506460D461F4C20787E
:105C2000401C20706078F021084202D0992001F0D9
:105C300001FC01F075FC6078401C6070306801E088
:105C400081614068002815D041694A1B8169491B60
:105C5000012A05DAC368D61892FBF3F203FB12623D
:105C600042610129ECDA02698B1891FBF2F102FB27
:105C70001131E5E76078F021084202D0992001F067
:105C8000D9FB6078401E6070C0B2002801D101F0DD
:105C900041FC01F02FFF002070BD0000501F0020CC
:105CA00066696E645F636C69656E740025733A2083
:105CB00066696E6428256429000000002DE9F04D16
:105CC0008EB0394E7078F021084202D0992001F050
:105CD000B1FB01F025FC7078401C707004F0F2F804
:105CE000074601A9002004F043F900A9002004F0B0
:105CF000C4F8DFF8B880D8F80800B84203D2811C95
:105D0000B94200D307469DF8020002909DF80100B9
:105D100003909DF8000004909DF8060005909DF802
:105D20000500401E06909DF80700463007900020B1
:105D30000A90DFF870A0834602A804F00DFAAAFBCF
:105D4000004543F6FF70C01B4EF66B614843594651
:105D50004FF47A720B4604F089FA24184D41D8E9C1
:105D600000018D4206D801D3844203D214EB0A0409
:105D700045EB0B05C8E90045C8F808707078F021BC
:105D8000084202D0992001F055FB7078401E7070D7
:105D9000C0B2002801D101F0BDFB204629460EB05B
:105DA000BDE8F08D40420F00501F002070710020B0
:105DB0007FB50446FEF759F801A9114A68CA68C1BF
:105DC000458A0120ADF80000281DFFF7C7FD0646F3
:105DD000372030707470022200A9B01CFCF72CFB35
:105DE000311D2046FEF7F9F8281DADF807003146B1
:105DF00001A801F046F93046FFF7C8FD7FBD00BF9E
:105E00004CA8010838B505000C0094F8500064282F
:105E100002D0802001F00EFB01F003FE802080F311
:105E2000118800BF00BFA0692843A061207C10F04A
:105E3000F800082806D1E069A169084202D02000D4
:105E400001F098FE07484078F021084202D09920DE
:105E500001F0F0FA03484078002802D1002080F3D6
:105E6000118831BD501F00202DE9FF4104460D4629
:105E7000FDF7FBFF064600A829498CC98CC006F136
:105E8000100000F0CAF8074606F1100000F0E6F82E
:105E9000ADF80C00002F01D1002D3FD0002D01D016
:105EA000032000E00020002F01D0391D00E0002178
:105EB0000818FFF753FD8046002F13D0372088F8CD
:105EC000000088F80140022203A908F10200FCF753
:105ED000B3FA06F1100108F1040000F052F8381D81
:105EE000ADF80300002D12D00520BDF8031001F815
:105EF00008000120BDF8031041444870BDF80300BC
:105F000040448470BDF80300C01CADF80300414656
:105F100000A801F0B6F84046FFF738FDBDE8FF8164
:105F200058A8010800218180C180704738B5044617
:105F3000E088401C2288A38890FBF2F502FB150044
:105F400093FBF2F502FB1535A84205D1581C90FBD6
:105F5000F2F302FB1300A080E088401C90FBF2F3F8
:105F600002FB1300E08060880246A368E58800FB1E
:105F70000530FCF761FA2088012801D10120E0807A
:105F800031BDF8B504460D0046D0002C44D0A98898
:105F900008462B88012B01D1002604E0421C92FB0D
:105FA000F3F603FB1626EA88571C97FBF3FC03FB6A
:105FB0001C7C90FBF3FE03FB1E0EF44518D1022B54
:105FC00016DB8A4208D26E8806FB07F2A968181A07
:105FD00006FB0040FCF730FA6888A9882A88521A24
:105FE0004243AB6800FB01312046FCF725FA10E084
:105FF000284600F012F800280BD0284600F00DF8D3
:106000000246A868B6B2698801FB06012046FCF783
:1060100013FA0020A880E880F1BD70B481880A4698
:10602000C3881C46A51A01D5C91A00E0591A631C79
:106030000488254693FBF5F605FB163392FBF5F62F
:1060400005FB1622934202D1022D00DB2146C9B284
:10605000408811FB00F080B270BC704730B481887A
:106060000A46C3881C46A51A01D5C91A00E0591A68
:10607000631C0088044693FBF4F504FB153392FB84
:10608000F4F504FB1522934202D1022C00DB0146F9
:10609000C9B2084630BC70470020704710B5DFF821
:1060A00014450020A08104F114010120FDF7F4FD46
:1060B000002803D00FF21050FEF7F0FA0120A07173
:1060C0000020E071207020816070E0811E206071EE
:1060D00000202061A070E070207110BD80B501210A
:1060E0008DF800108DF8011008218DF802108DF840
:1060F000030000A92920FDF7C5FE01BD70B52DEDF7
:10610000048B84B0002400A90120FDF766FFDFF8AE
:10611000A45495F90160002E05D0022E37D00FD37C
:10612000032E5DD086E09DED000AB0EE408A9DED25
:10613000010AF0EE408A9DED020AB0EE409A79E045
:106140009DED010AF0EE408ADDED020AB0EE609AA4
:106150009FEDCC1A00EE401A00EEE01AB5EE401AA0
:10616000F1EE10FA10DD11EE100AFFF7CDF941EC57
:10617000100B04F0F3F851EC100BFFF78FFB00EE5F
:10618000100AB0EE408A55E09FEDD08A52E09DEDB6
:10619000000AB0EE408ADDED020AB0EE609ADDED55
:1061A000001A9FEDB81A00EE611A00EEE01AB5EE83
:1061B000401AF1EE10FA10DD11EE100AFFF7A4F903
:1061C00041EC100B04F0CAF851EC100BFFF766FB22
:1061D00000EE100AF0EE408A2CE0DFEDBC8A29E0E8
:1061E0009DED000AB0EE408A9DED010AF0EE408A76
:1061F0009FEDA41A00EE401A9DED000ADDED000AA5
:1062000000EE601AB5EE401AF1EE10FA10DD11EE54
:10621000100AFFF779F941EC100B04F09FF851ECEC
:10622000100BFFF73BFB00EE100AB0EE409A01E0C6
:106230009FEDA69AB5F90C00012801D101201DE1BE
:1062400095F90000002860D16889411C698195F9A1
:106250000500421C09B28A4233DB0098FFF754F96B
:1062600021F000414FF02042D34BFFF75FFB03D8F2
:10627000A878401CA87001E02046A8700198FFF79C
:1062800043F921F000414FF02042CB4BFFF74EFB8A
:1062900003D8E878401CE87001E02046E8700298D6
:1062A000FFF732F921F000414FF02042C24BFFF7D7
:1062B0003DFB03D82879401C2871DEE02046287178
:1062C000DBE095F90210814202DB012068700FE0EB
:1062D00095F90310814202DB0220687008E095F90D
:1062E0000410814202DB0320687001E020466870E0
:1062F00095F901100FF2DC20FEF7D0F9012028708B
:106300002046688104F0AAF8B7E0012864D1288902
:10631000401C28813046B0EE491AF0EE680AB0EE13
:10632000480A04F09FF8002847D0F0EE680AB0EE63
:10633000480A20EE000A00EEA00A09EE090A04F05D
:1063400053F989EE000A10EE100AFFF7DDF841EC70
:10635000100B04F0E9F953EC102B98489849FFF71B
:1063600057F9FFF711F9286195F90100002821D1AB
:10637000A879012809D105F114010120FDF7CDFC10
:10638000002800D003240020A871E87900280AD151
:1063900005F120011C20FDF77FFC002801D003201F
:1063A0006CE00120E8710FF23C20FEF777F9022043
:1063B000287062E0032028705FE0B5F908006428C7
:1063C0005BDB2046288100F0A5F8052028700FF23D
:1063D0002820FEF763F950E003284ED1F0EE680A5A
:1063E000B0EE480A20EE000A00EEA00A09EE090A03
:1063F00004F0FAF889EE000A10EE100AFFF784F8AC
:1064000041EC100B04F090F953EC102B6B486C49E5
:10641000FFF7FEF8FFF7B8F82969081A04F08CF9BD
:10642000002E19D16989491C698109B2652908DAE8
:10643000242803DBE889401CE88115E02046E88138
:1064400012E020466881012028702046E8810FF282
:10645000B410FEF723F910E0242803DBE889401C80
:10646000E88101E02046E881B5F90E00052804DB4B
:10647000042028700120FFF731FE204604B0BDEC57
:10648000048B70BD3D57C04210B54A4C00202070AF
:10649000A081E079012808D104F120011C20FDF73A
:1064A0003CFC00280BD10020E071A07901280AD122
:1064B00004F114010120FDF730FC002801D0032075
:1064C00010BD0020A071002010BD000000000000E1
:1064D000002070470020704710B5364CE079012845
:1064E00008D104F120011C20FDF717FC00280BD176
:1064F0000020E071A07900280AD104F114010120E4
:10650000FDF7CAFB002801D0032010BD0120A071B7
:10651000002010BD10B5274C002060812081A0799B
:10652000012808D104F114010120FDF7F6FB002831
:106530000BD10020A071E07901280AD104F12001DB
:106540001C20FDF7EAFB002801D0032010BD00202D
:10655000E071002010BD10B50FF2DC00FEF79EF8D0
:10656000144C94F9000002280FD1FFF7B5FF03285F
:1065700005D10FF2D000FEF791F8032010BD0320E3
:1065800020700FF2CC00FEF789F8002010BD0D49F5
:106590000A1DC26129220270142282600122027344
:1065A00002820422428200228282C28281611046DB
:1065B000704700002C2100209999274046DF617E1A
:1065C000DCA54C400C240020736D20414343206621
:1065D00061696C0053535020534D41204D6F6465E9
:1065E0002025640053535020534D41204144442002
:1065F000414343494E54000053535020534D4120D2
:106600004E46000053535020534D4120556E736148
:1066100074697366696564204D6F76696E672041A1
:106620006E676C6520647572696E6720322D7365C4
:10663000632021212100000053535020534D41205D
:10664000494E5400534D20414420464C0000000068
:1066500053535020534D4120494E56205341490039
:106660000020704710B5794C04F108010120FDF7B6
:1066700013FB002801D0032010BD04F061F80020B6
:106680002070012060700020A07060600120E07028
:10669000002010BD3EB500A90120FDF79EFC6B4C0B
:1066A0002078012818D16078012808D104F1080168
:1066B0000120FDF732FB00281BD100206070A0787C
:1066C00001284FD104F114011C20FDF726FB0028FE
:1066D0000FD10020A07045E0E078002824D1607838
:1066E00001280AD104F108010120FDF716FB00285A
:1066F00001D003203EBD00206070A078002831D179
:1067000004F114011C20FDF7C7FA002805D00FF290
:106710004410FDF7C3FF03203EBD0120A0700FF21F
:106720004810FDF7BBFF1DE000A890EC030A04F041
:1067300029F8054604F09FF9002803D16068401C41
:10674000606001E0002060606068332803DB0020A7
:10675000E07003F0F5FF012D04D1012000F027F8CF
:106760000120207000203EBD10B5384C6078012813
:1067700008D104F108010120FDF7CFFA00280BD160
:1067800000206070A07801280AD104F114011C20B7
:10679000FDF7C3FA002801D0032010BD0020A0702F
:1067A0000020207010BD002070470020704780B589
:1067B0008DF8000000A91120FDF764FB01BD10B5A4
:1067C0000FF2B400FDF76AFF204CE078002829D1D1
:1067D000A07801280ED104F114011C20FDF79DFAC8
:1067E000002805D00FF29C00FDF758FF032010BDD4
:1067F0000020A070607800280ED104F1080101206B
:10680000FDF74AFA002805D00FF29400FDF746FF85
:10681000032010BD012060700120E0700FF2940091
:10682000FDF73CFF002010BD09490A1DC26111227D
:1068300002701422826001220273028242820022CC
:106840008282C2828161104670470000742300205A
:10685000F023002053535020534D4420494E5420E0
:106860004641494C0000000053535020534D4420F2
:10687000494E54204144440053535020534D44202A
:10688000494E540053535020534D4420414343201C
:10689000494E542052656D6F7665204661696C00E3
:1068A00053535020534D4420414343204F6E2046C4
:1068B00061696C0053535020534D4420494E54207D
:1068C0004F4343000020704710B5DFF8804604F1C5
:1068D00038010120FDF7E0F9002805D00FF28060B3
:1068E000FDF7DCFE032010BD04F138010520FDF7A3
:1068F000D3F9002805D00FF27860FDF7CFFE032012
:1069000010BD00F081F9002010BD1CB50446012027
:106910008DF800008DF8010038208DF8020001206C
:106920008DF803008DF804008DF805108DF8062011
:1069300000A95920FDF7A6FA204600F04EF813BD35
:1069400080B500F0F0F8DFF80406C07A052813D807
:10695000DFE800F003060C09120F00F0A1F90EE0C9
:1069600000F0DAF90BE000F010FA08E000F047FA66
:1069700005E000F082FA02E0012000F0F8F800F0F3
:1069800067F900F01AF9002002BD10B500F0B7F861
:10699000DFF8B84504F138010120FDF7BEF9002801
:1069A00001D0032010BD04F138010520FDF7B5F931
:1069B000002801D0032010BD002010BD80B5112893
:1069C00001D100F081F8002002BD80B5102802D16D
:1069D000104600F01EF8002002BD012811D1DFF89A
:1069E0006C054179017100210172C171417902295F
:1069F0000DD18179082901D0092908D10021C1626E
:106A000005E0022803D1DFF844054178C170012078
:106A1000704738B5017803292CD144788178C07843
:106A200010EB0125ADB22A4621460FF25450FDF776
:106A300035FE012C06D01DD3032C0ED006D3042C1A
:106A400012D017E0DFF80805857713E04FF47A706D
:106A50006843DFF8FC1488600CE04FF47A706843F8
:106A6000DFF8E814486105E04FF47A706843DFF816
:106A7000E0144860012032BD70B582B000A9082042
:106A8000FDF7ABFA9DF80050BDF90260DFF8BC4499
:106A9000B4F93030324629460FF2F440FDF7FEFDDE
:106AA000B4F93000864200DA2686002D04D1B4F90C
:106AB0003000301A322802DB0120A07202E00020F0
:106AC000A0722062002076BD0120DFF880140872D9
:106AD000704710B5DFF87444607A002801D00020B8
:106AE00010BD04F138010820FDF7D6F8002801D0C8
:106AF000032010BD012060720020206210BD10B57F
:106B0000DFF84844607A002801D1002010BD04F16C
:106B100038010820FDF701F9002801D0032010BD3D
:106B20000020607210BD00B589B000A90120FDF7FA
:106B300054FA03A90520FDF750FA039900A803F0C1
:106B4000BDFFDFF80804417A002907D090F90A1048
:106B5000012903D1016A826A51180162816AC26AFD
:106B60008A18C262426A8918416209B000BD38B50C
:106B70000446DFF8D8532246E97A0FF24040FDF789
:106B80008DFDEC7200206862BDE83140B7E770B55A
:106B900004460D46164633462A4621460FF230403B
:106BA000FDF77CFDDFF8A403047021464171857177
:106BB000002E01D00121C17170BD10B5DFF88C43EA
:106BC000207A002806D021786171A2790120BDE8E1
:106BD00010409AE6E07900280BD061792079814253
:106BE00004D0A2790120BDE810408EE60020E071BB
:106BF00010BD207B002806D0A27861780220FFF724
:106C000084FE0020207310BD10B503F047FFCF4C69
:106C1000002234212046FBF7E1FB5020A062002037
:106C2000E07240F6B830206147F230516161A061F6
:106C300001206073E1614FF4FA60E062012020708E
:106C40006071A07147F6FF7020866420E07010BD6F
:106C500038B5BE4C94F8320001280ED104F06AF920
:106C600000280AD0022084F83200651C0120E87256
:106C7000032060700B20687031BD94F83200032847
:106C80000DD1651CE87A002809D104F0F5F8A9783F
:106C9000814204D00121E97260700C20687031BD1E
:106CA00080B503F083FF00280AD0002201210846A6
:106CB000FFF76DFF0120FFF75AFF0120A34948733A
:106CC00001BD000038B5A14C606BA16A0818606373
:106CD0000025FFF7FEFEA069616B88421AD200EE24
:106CE000100AB8EE400ADFED980A20EE200ABCEE4A
:106CF000C00A10EE100A216A884206D20225E17A03
:106D00000FF2E820FDF7CAFC00E0012500206063D7
:106D1000FFF7F5FE284632BD10B58C4C00F01DF88B
:106D2000002805D00320FFF722FF0120607310BD6B
:106D3000606900F021F800280ED0FFF7C3FF022899
:106D400005D1002060730220BDE810400FE7012844
:106D500002D100206073606210BD80B504F063F85A
:106D6000002807D07948006903F026FF022801D1E6
:106D7000012002BD002002BD74494A6A904201D23E
:106D80000120487391F90D00704710B56F4C00F069
:106D900023F800280AD0012202211046FFF7F7FE4F
:106DA0000120FFF7E4FE0120607310BD607B002826
:106DB00011D0FFF787FF022807D100220821022007
:106DC000FFF7E5FE0020607310BD012803D100200D
:106DD00060730520A07110BD10B55C4CE06AB0F581
:106DE000FA6F0AD304F02BF8002806D0E16A0FF2FC
:106DF0001020FDF753FC012010BD002010BD70B520
:106E00000026524C534DFFF7A8FF002807D030460C
:106E10002870012060730320FFF7A9FE18E0E069E5
:106E2000FFF7AAFF002813D0FFF74CFF02280CD170
:106E30002878411C2970304660626073E27AC9B2DA
:106E40000FF2D010FDF72AFC02E0012800D1012644
:106E50002878032807DB012209210220FFF797FE8B
:106E600003F006FF0526002E06D000202870607370
:106E70003046BDE870407AE670BD3448C06AB0F56F
:106E8000FA6F00D2704780B500F010F8002803D1E7
:106E900000F01AF8002808D0012204211046FFF75C
:106EA00076FE0120BDE8024061E601BD00B585B077
:106EB00000A90520FDF791F8009815288041C043EE
:106EC000C00F40B205B000BD38B50024224D95F981
:106ED0000000002805D103F0D7FE002801D00120D2
:106EE000287095F90000002819D0FFF7F2FD174827
:106EF0006968826A51186960B1F5967F0FDB90F975
:106F00000A00002804D10FF22410FDF7C7FB01246A
:106F1000002068602870FFF7F2FD03F0A9FE20460C
:106F200032BD0E4901F10802C2615922027050229D
:106F30008260012202730282072242820022828240
:106F4000C282816110467047CDCCCC3E981F002094
:106F5000AC1F0020F47100207C710020142300205D
:106F60004450434D20414343206661696C0000005A
:106F70004450434D204C49474854206661696C0099
:106F80004450434D2053657420256420256400003F
:106F90004450434D2050726F7820537461746520C3
:106FA0005B25645D206F6666736574205B25645D98
:106FB000206D696E205B25645D0000004450434DE8
:106FC000205354205B25645D2D3E5B25645D0000ED
:106FD0004450434D2053455420524554205B256472
:106FE0005D5B25645D5B25645D0000004450434D9E
:106FF00020434C4F534544205B25645D0000000056
:107000004450434D20484F4C442054494D45202581
:10701000640000004450434D204F464620434E54E8
:10702000205B25645D5B25645D0000004450434D9A
:107030002050726F7869204F70656E0010B5684CF3
:1070400068488089C0464021674804F019F801F07B
:107050002AFA4FF48051654804F008FC00280FD14B
:107060002046441E0128F4DA0021614804F0D8FCCF
:107070000021604804F0D4FCBDE8104001F010BAD3
:1070800010BD38B504460D46B4F80300FEF766FCA3
:10709000C4F80500002807D10FF26810FDF7FEFACA
:1070A000BDE83140FDF74CBBB4F803202946FBF79F
:1070B000C3F9514D214605F2144000F03FFE294628
:1070C0000420BDE83440FEF79DBE38B50446B4F850
:1070D0000300401DFEF742FC050007D10FF23C10F3
:1070E000FDF7DCFABDE83140FDF72ABB0522214659
:1070F000FBF7A2F9B4F80320D4F80510681DFBF7DC
:107100009BF9B4F80300411D89B2284600F0A9F8A4
:10711000002D02D02846FEF739FCD4F805000028DF
:1071200004D0FEF733FC0020C4F8050031BD10B5D3
:1071300084B00120ADF8030005208DF80000BDF8F3
:107140000300FEF70BFCCDF8050000280FD0072147
:1071500001700FF2E000FDF7A1FA274C00A904F23C
:10716000144000F0EBFD21460420FEF74BFE1FBD4E
:1071700010B584B000A800210A460B460EC0FFF7E8
:10718000D6FF062004F00CFD0446A00701D5FFF74A
:1071900055FF600706D500A9184804F047FD00A870
:1071A000FFF793FFFDF7CCFAEBE710B584B0124C74
:1071B00004F586630422092104F2144004F06AFDF8
:1071C000022002904FF47070019004F1540000907E
:1071D0000B4B64220FF26401204604F0AFFD1FBD8B
:1071E000404B4C0000300140146F0020000402406E
:1071F0005864024010640240584A00206C4E00203F
:10720000717100083D3D3D3D3D3D3D3D20616C6C53
:107210006F63206661696C20310000003D3D3D3D9B
:107220003D3D3D3D20616C6C6F63206661696C2063
:10723000320000005245534554000000636F6D6DED
:107240005F7461736B000000BFF34F8F40480168AB
:1072500001F4E0613F4A11430160BFF34F8F00BF6B
:10726000FDE7F0B583B00E460021009103210191A6
:10727000394CA16CC90706D5A16C49084900A16425
:10728000A16CC907FCD4354D00220146284604F004
:10729000DDFB4FF0C051284604F0F5FB314628468F
:1072A0004160C0460121284604F0BAFB2C4E0096EE
:1072B00001F0F3F80FF2B4070BE0009601F0EAF8E2
:1072C000052001F0A7F801993846FDF7E7F901F02C
:1072D000E4F84FF0C051284604F0C2FB002816D154
:1072E0000098411E00910128F3DA0198401E019098
:1072F000E3D50021284604F093FB0021204604F04A
:107300008FFB01993846FDF7C9F9FFF79DFF49F654
:1073100040400090134C0221204604F02DFE00282E
:1073200004D10098411E00910128F4DA42F2107055
:1073300000908021204604F01FFE012804D100980F
:10734000411E00910128F4DABDE8F74001F0A2B82F
:107350000CED00E00400FA0510640240586402409D
:1073600080841E00003001406EE7000054785265B2
:107370007472792025640000002801D10A488068D1
:1073800090F85010642901D0002000E0C06A7047D6
:10739000002801D10448806890F85010642901D079
:1073A000002000E0806A7047501F002002487047AC
:1073B00002480149401A7047480000204808002050
:1073C00008B584B00023029311B90093019302E041
:1073D0000090481E019004AB00A90748784418307B
:1073E00004F0D2FD009911B1009A0021117000281B
:1073F00058BF029805B000BDB7B0FFFF00F1010310
:10740000810704D010F8011B89B18107FAD1026805
:10741000B2F10131914311F0803F04BF50F8042FC5
:10742000F6E710F8011B11B110F8011BFBE7C01AB9
:107430007047000000B585B002460FF2140100A8A5
:1074400005F078FC00A8FCF77AFF05B000BD00004D
:107450004F4525640000000034488168002904BFBE
:1074600008B008E0EFF30982A2F12802036882E87D
:10747000F84F83685A6000F056F9816859B14A683C
:1074800092E8F84F036002F1280282F3098813F4AE
:107490007F4F3FD07047264826490968401A80F33D
:1074A00008884FF08071C161234981617FF0060E29
:1074B000704701BC2046DFF884E000BDFEE72048AD
:1074C00000681C490968401A203820F0070080F342
:1074D00008884FF000011548417081F3118862B6A9
:1074E00000F014F8FEE703680CB44FF0000141709F
:1074F0004FF0000181F311881249134A0A604FF0DE
:10750000800181F311880CBC036070470D490E4A5D
:107510000A6070474FF0000181F31188704700BF87
:107520004FF0800181F31188704700BF501F002089
:107530002808002088A8010895CE0008BD7400081E
:107540000000000804ED00E00000001010B48020EE
:1075500080F3118800BF00BFDFF8C0078068DFF844
:10756000BC1700220A71002181F3118800282ED057
:10757000016800292BD0426901684969914226D1EE
:10758000016800E019000B68002B02D05C6994428E
:10759000F8D0802282F3118800BF00BFDFF87C277B
:1075A0001269824203D1DFF8742703681361026A0B
:1075B000036813601A6201620B6803600268002AA4
:1075C00000D01862086091F8450081F8440000205E
:1075D00080F3118810BC7047802080F3118800BFB1
:1075E00000BFDFF83C070068DFF83017096A401A6F
:1075F00001283ADADFF82407006A05E0DFF81C17F3
:107600000862002181F31188DFF818170978C9078B
:1076100026D5802181F3118800BF00BFDFF8041751
:1076200009788907EAD5DFF8FC16097811F0FD0121
:10763000DFF8F0261170002181F31188DFF8DC16E5
:10764000096A8842FAD0DFF8D4160862DFF8D0065B
:107650000068401CDFF8C8160860DFF8C0164862F2
:10766000802080F3118800BF00BF704710B5DFF89D
:10767000AC0600214171DFF8A406006A10F18040D9
:10768000DFF898164862DFF89406C069002805D034
:10769000DFF88806DFF88416C9698847002080F380
:1076A0001188DFF87806C4680EE0E068DFF86C1631
:1076B000496A401A002803D5DFF86006E168416294
:1076C000002080F311882468002C26D0802080F3CD
:1076D000118800BF00BFDFF844060069002806D00B
:1076E0006069DFF838160969496988421AD3207C35
:1076F0004007E5D5E068DFF82416096A401A01283A
:10770000D3DA200000F036FA802080F3118800BF21
:1077100000BF207C0028C8D104E0802080F31188BD
:1077200000BF00BF10BD38B5DFF8F0050021417083
:10773000DFF8E80501210170DFF8E005C06B0028E3
:1077400018D0802080F3118800BF00BFDFF8CC057F
:10775000C06B8047002080F31188DFF8C00500214E
:10776000C163DFF8B80500214163DFF8B0050021EF
:1077700080F83810FFF71AFE0078C0B2CD2802D08A
:107780007D20FFF757FEDFF894058068002812D0AF
:10779000DFF888058068806C00280CD0DFF87C0555
:1077A0008068806C01680800002804D0DFF86C0550
:1077B000806840688847DFF8640590F83100002849
:1077C0000FD0DFF858058068DFF8501591F83010B9
:1077D00080F84410DFF844050079002801D0FFF755
:1077E000B5FEDFF8380590F8400000283DD0DFF8FE
:1077F0002C0590F84000C00718D5DFF82C0500686C
:10780000DFF81815096A401A00280FD5DFF80C05B3
:1078100090F8400010F0FE00DFF8001581F84000FD
:10782000DFF8F80490F8400000281ED0802080F394
:10783000118800BF00BF05F03BFB002181F31188D8
:10784000DFF8D814896800290CD0DFF8D0148968D3
:10785000896B4118DFF8D4241268891ADFF8BC2438
:1078600092689163DFF8C4140860DFF8B0048068A0
:1078700000280ED0DFF8A4048068007C002808D11E
:10788000DFF898048068406B401CDFF8901489682A
:107890004863DFF888040069002839D006E0DFF883
:1078A0007C0421680161002080F31188802080F32E
:1078B000118800BF00BFDFF864040469002C2FD0DA
:1078C000257CEDB2002D2BD0680716D5E068DFF8D7
:1078D0004C14096A411A012906DA200000F04AF91D
:1078E000207C002809D113E0DFF83014496A411ADE
:1078F000002902D5DFF824144862EDB215F0FB0030
:107900001028CCD1A06880684068007C0028C6D1CF
:10791000802080F3118800BF00BF01E0FFF7A6FEC2
:10792000DFF8F80340790028F8D1DFF8F803007891
:10793000C00701D5FFF750FEDFF8E00300214171D9
:10794000DFF8D8030069002853D0DFF8D0030069BE
:10795000007C002809D0DFF8C403006980688068D3
:10796000DFF8B8134068886005E0DFF8B003DFF89F
:10797000AC1309698160DFF8A403806890F85000B7
:10798000642802D08020FFF755FDDFF8900380685F
:10799000C06A0078CD2802D07820FFF74BFDDFF8D1
:1079A0007C038068806C00280CD0DFF8700380684E
:1079B000806C41680800002804D0DFF8600380680C
:1079C00040688847DFF85403806890F84400DFF887
:1079D0004C1381F83000DFF8441381F83100DFF8F0
:1079E0003C038068006B401CDFF830138968086333
:1079F00014E0DFF82803002180F83110DFF81C03C1
:107A0000002180F83010DFF8140300218160DFF8D6
:107A10000C0300210170002080F31188DFF8FC02C4
:107A200032BD80B505F07EFADFF80413097800282E
:107A300006D0022810D009D3042815D010D314E0A2
:107A4000002902D0A320FFF7F5FC11E0002902D1A4
:107A5000A420FFF7EFFC0BE0A620FFF7EBFC07E00C
:107A6000A720FFF7E7FC03E002E0A820FFF7E2FC15
:107A700001BD10B505F056FA0400DFF8B402007835
:107A8000002802D0A020FFF7D5FC002C05D0022C46
:107A900008D003D3032C09D00CE00EE0A420FFF79C
:107AA000C9FC0AE0A620FFF7C5FC06E0A720FFF707
:107AB000C1FC02E0A820FFF7BDFC10BD80B505F0B9
:107AC00031FA002805D0022808D006D3032809D0AF
:107AD0000CE0A320FFF7AEFC0BE00AE0A620FFF7C6
:107AE000A9FC06E0A720FFF7A5FC02E0A820FFF70D
:107AF000A1FC01BD80B5DFF824020078002802D186
:107B00009720FFF797FCDFF814020078401EDFF89B
:107B10000C120870C0B200282BD1DFF800024068B8
:107B2000002826D0802080F3118800BF00BFDFF836
:107B3000EC01406800280BD0DFF8E0010121017062
:107B4000DFF8D801FFF7CFFCDFF8D001002101708A
:107B5000DFF8C8014078F021084202D09920FFF7F1
:107B600069FCDFF8B8014078002802D1002080F3DA
:107B7000118801BD10B5816800290CD0DFF89C1177
:107B8000096AC16081680A684968002A00D05160AA
:107B90000A6000218160017C11F003010174C9B207
:107BA000002943D1DFF87411096900292AD1DFF8CF
:107BB0006C110861DFF86401007800280CD1DFF84F
:107BC0005C0101210170DFF85401FFF78CFCDFF844
:107BD0004C010021017003E0DFF8400101214171F7
:107BE000DFF838014078F021084202D09920FFF7F1
:107BF00021FCDFF828014078002802D1002080F322
:107C0000118813E042694B699342D0D38142D1D0AD
:107C10004B699A420AD10300FFE71B68002BDFD0B3
:107C20005C69A242DCD18B42F7D1C0E710BD10B530
:107C300004006069002802D1CB20FFF7FBFB6269DA
:107C400036480078401C354908703A4800E0080082
:107C50000168002902D04B699A42F8D32160206262
:107C60000460002909D00C624869904202D194F85E
:107C7000450000E0002084F84400207C002816D154
:107C8000802080F3118800BF00BF2000FFF772FF43
:107C900022484078F021084202D09920FFF7CAFB21
:107CA0001E484078002802D1002080F31188FFF799
:107CB00021FF10BD10B51948047818480078401C01
:107CC000164908701548FFF70EFC14480470134855
:107CD0004078F021084202D09920FFF7ABFB0F4813
:107CE0004078002802D1002080F3118810BD10B523
:107CF00005F01EF9094801210170FFF757FB040048
:107D00006846C046021B203A012A03DBCD21200031
:107D100005F032F908480121017010BD501F002004
:107D2000CC710020FA710020E4710020D071002095
:107D3000F97100205C1F0020FC71002038B50400A0
:107D40000D0017480078401C154908701548007848
:107D5000002802D0A120FFF76DFBFFF78AFEA07E6E
:107D6000662802D08220FFF765FB802080F311880F
:107D700000BF00BF08E03821200005F007F980208F
:107D800080F3118800BF00BFE06821698842F2D00B
:107D90002900200005F01EF9FFF7ACFE31BD00BF41
:107DA000501F0020FB710020002803D00249B1F8C9
:107DB0009A170180704700008437002010B5DFF863
:107DC000A84500224FF4F0712046FAF707FBDFF8D0
:107DD0009C05606410BD000010B5DFF88C45A189DA
:107DE0004118A181E2898018E081207A192803DAFC
:107DF000401C207284ED110ADFED700AB4EE600AB7
:107E0000F1EE10FAC0F2958094ED111AB4EE601AFA
:107E1000F1EE10FAC0F28D80207A1928C0F2898024
:107E200089B2C329C0F28580207904EB800080EDFF
:107E3000280A84ED110AE079002804D184ED120AA1
:107E400084ED130A17E0D4ED120A9FED5D1A60EE7F
:107E5000810A9FED5C1A40EE010AC4ED120A94ED0E
:107E6000130A9FED591A20EE010A9FED581A00EEF1
:107E7000810A84ED130AE089B0F57A7F14DDA079D8
:107E800004EB8000E16CC0F84011A079401CA071A7
:107E9000C0B2142801D10020A071607A142801DA40
:107EA000401C60720020E0812279E17914290DD113
:107EB000501C142800D1002094ED0F0A04EB800020
:107EC000D0ED3C0A30EE600A84ED0F0A04F1A00008
:107ED00000F086F9207904EB800080ED3C0AD4EDB7
:107EE0000F0A30EE800A84ED0F0A207904EB80003F
:107EF000E16C0165207904EB4000A1890182E07901
:107F0000142801DA401CE071E07900EE100AB8EEA6
:107F1000400AD4ED0F0A80EE800A84ED100A207921
:107F2000401C2071C0B2142801D100202071002013
:107F3000A08110BDDFF8300481794A1E00D51432CB
:107F4000891F00D5143100EB810191ED500A00EB3F
:107F50008200D0ED500A91ED501A70EEC10AF5EE94
:107F6000400AF1EE10FAD0ED500A02DD30EEC00A00
:107F7000704730EE600A7047DFF8EC0381794A1EE3
:107F800000D51432891F00D5143100EB810191ED29
:107F90003C0A00EB8200D0ED3C0A91ED3C1A70EEF9
:107FA000C10AF5EE400AF1EE10FAD0ED3C0A02DD0E
:107FB00030EEC00A704730EE600A70470100FA43A5
:107FC0006666663FD0CCCC3DCDCC4C3FCCCC4C3E55
:107FD0002DE9F84F2DED088BF0EE409A07468846C4
:107FE0004FF000094C469FED798ADFED788A9FEDCE
:107FF000779A9FED76AAA246FFB2042F04D1DFED57
:1080000074AA9FED74BA03E0DFED73AA9FED73BA13
:10801000DFF8545395F807B05E46142E40F0CF8039
:10802000687A0728C0F2CB80F5EE409AF1EE10FA9C
:1080300040F3C580FFF77EFFF0EE40BAFFF79CFFEC
:10804000F4EE6BAAF1EE10FA34D5D5ED100AF5EE88
:10805000400AF1EE10FA02DDB0EE601A01E0B1EE76
:10806000601AB4EE41BAF1EE10FA23D5F5EE400AEB
:10807000F1EE10FA01DCF1EE600A9FED7B1AF4EEEE
:10808000410AF1EE10FA15D5DFED780AB4EE600A78
:10809000F1EE10FA0ED52868002802D0A86BA8EBE4
:1080A000000A3B46524659462879401E00F0E4F843
:1080B000814602E020462860A863B9F1000F7BD01A
:1080C0002868002803D1C5F83880012028602046A0
:1080D00005E005EB4101098A0C19A4B2401C80B2ED
:1080E00001461429F5DB00EE104AB8EE400ADFED38
:1080F000970A20EE200ADFED5F0A69EEA00A20EE63
:10810000200A2879411E00D51431801B00D5143077
:1081100005EB8101D1ED140A05EB800090ED141AF6
:1081200070EEC10A9FED521AC0EE819AF4EE409AA9
:10813000F1EE10FA02DBDFED259A07E020EE000AEF
:1081400009EEE90AFAF72EF9B0EE408AB5EE408A58
:10815000F1EE10FA01D0C9EE888A687905EB80004B
:10816000C0ED648A6879401C6871C0B2142801D1DE
:1081700000206871A87A142801DA401CA872002037
:1081800006E005EB800191ED640A39EE009A401C8F
:10819000A97A0A4680B29042F3D3B2EE040A29EEDD
:1081A000000A00EE901AF8EE600A80EE200ADFED79
:1081B000680A20EE20AA02E020466871A872B0EE9C
:1081C0004A0ABDEC088BBDE8F18F000000000000FA
:1081D000CDCC4C3EA69B443BCDCC4C3D6F12033BDB
:1081E00010B49FED5C0ADFED5B0A9FED5A1ADFEDDC
:1081F000591A00231AE0142C00DB143C02EE103A4A
:10820000B8EEC22A32EE000A50F8244002EE904A3C
:1082100070EEA20A02EE221A13FB03F402EE104AD9
:10822000B8EEC22A72EE211A5B1CDBB20C46A342E6
:1082300005DA141B1C19641CDDD51434DEE702EECC
:10824000101AB8EE422A22EE011A00EE601A62EE0F
:10825000210A40EE400A9FED400A30EE800A81EE8E
:10826000000A10BC704700000AD7233C0AD7A33C81
:108270008FC2F5BD3B89883CF0B51C460023002821
:1082800001D5143002E0142800DB14381D461E46C8
:10829000042C04D19FED310ADFED310A03E09FED9C
:1082A0002B0ADFED300A1C460CE0B4EE410AF1EE79
:1082B00010FA06D5B4EE601AF1EE10FA01D5761C6C
:1082C000B6B2641C0F46E4B2A446A7F1010EF44511
:1082D0002EDAC71B67447F1C01D5143702E0142F28
:1082E00000DB143F07F1010CBCF1140F01DBACF112
:1082F000140CDFF874E00EEB8C0C9CED141A0EEBF2
:108300008707D7ED141A31EE611AFFEE001A20EE3E
:10831000212AB4EE421AF1EE10FAC6D560EEA11A87
:10832000F4EE411AF1EE10FABFD56D1CADB2C8E7FC
:10833000072A01D20C2000E00A20B04201D201231A
:1083400002E0A84200D202231846F0BD6F12833A21
:10835000CDCCCC3D00000000BD3786356F12033B0D
:108360008FC2F53C8FC2753C245B002000407E44E8
:10837000D2B2203A22BF00FA02F1002070475242E6
:10838000D041D2F1200291404140D0409040414044
:108390007047000010B5354C00224FF49071204614
:1083A000FAF71CF8204610BD3048704710B5044657
:1083B0002F4804F0A2FF2F4804F09FFF01206071B6
:1083C00010BD10B5044604F0D8FF0120A07110BD07
:1083D00038B50446012505F086F8012804D1284661
:1083E000E0700020A0700AE0022804D10020E070B4
:1083F0002846A07003E00020E070A07005462846E3
:1084000032BD10B50446E07905F036FB012121703C
:1084100010BD000018490A6A0B6A00BF00BF00BF08
:1084200000BF00BF9B1A8342F6DB704705F016BA07
:1084300005F018BA70B504460025E679E171FFF73A
:10844000E0FF00280BD00D480078002802D020461D
:10845000FFF7ACFF2046FFF7B4FF012503E0E6710C
:108460002046FFF7CEFF284670BD0000E0660020E2
:108470000058004000540040501F0020F7710020B9
:1084800005F0A5BD05F008BE05F0B2BD05F06EBE55
:1084900005F076BE012004F02DBE002004F02ABEB7
:1084A000012004F033BE002004F030BE05F072BE9F
:1084B00010B5FFF76FFF044604F057FE0B2120466E
:1084C000FFF7B8FF05F09FF82046FFF7D9FF2046D9
:1084D000FFF77EFF002201210846FFF7E7FFFFF7C5
:1084E000D9FFBDE81040DBE770B44FF0004591EADA
:1084F000030F44BF6B40FDF767B900BF841A71EBEF
:10850000030604D26E40001BB141121973414FF4AF
:10851000001C1CEB410F34BF7CEB430684E00C0DC8
:10852000A4EB1356362E7DDC012E43DC45EAC32333
:1085300043EA525312BFD20292025B08240545EA75
:10854000C12141EA5051D2EBC020994125D407D135
:10855000B0FA80F610FA06F164D00020203608E068
:10856000B1FA81F6B140C6F1200220FA02F21143BD
:10857000B0404FEAF474B4EB465434F001064FEACD
:1085800074040AD8D6F50016760D04F00044F040C5
:1085900061FA06F25040F1404840C00A40EA4150BA
:1085A00021F0004128BF5FEA500550F1000044EB84
:1085B000D12137E045EAC323DB0A45EAC121C90AD4
:1085C000B6F120050EDD42EA0242120CC5F120068A
:1085D00003FA06F6EB4042EA06056D42984161F166
:1085E00000010DE062FA06F5F240554063FA06FC20
:1085F00082EA0C02F3405A406D42904161EB030164
:1086000011F4801F05D1641E620502D06D00404147
:10861000494121F48011430875F1004350F10000F5
:1086200041EB045170BC70471CEB410F15D223F095
:10863000004352EA43060BD04FEA4C0CBCEB410F0F
:1086400004D80C0D661E342EB7DDEBE7801A994175
:1086500050EA410608BF0021E4E708BF1CEB430FC6
:1086600028BF6FF00001DDE780B55A490978491C41
:10867000584A1170017A491E0172C9B2002901D10C
:1086800005F0F2FDFFF736FA01BD38B50400524897
:1086900005680BE0287A002807D06868A04204D15A
:1086A000012028722800FFF7DFFFED68002DF1D1CF
:1086B00031BD38B5040049480078002802D0A12017
:1086C000FEF7B8FEFFF7D5F94348056805E0A54277
:1086D00002D1AF20FEF7AEFEED68002DF7D1404885
:1086E0004049016014220021200004F045FC69206B
:1086F0002074802080F3118800BF00BF36480068D6
:10870000E0603548046033484078F021084202D0E8
:108710009920FEF78FFE2F484078002802D10020D4
:1087200080F3118831BD38B504002C48007800284A
:1087300002D0A120FEF77EFEFFF79BF9207C69287E
:1087400002D08520FEF776FE22480078401C2149A1
:108750000870207A002804D11E48806860600125D6
:1087600010E060681B498968884209D01021200008
:1087700004F00CFC207A0028F8D11648806860606C
:10878000207A451C2572FFF7B5F9280032BD10B5D7
:10879000040012480078002802D0A120FEF74AFE0B
:1087A000FFF767F9207C692802D08520FEF742FE9A
:1087B000207A002802D19620FEF73CFE6068054929
:1087C0008968884202D09C20FEF734FE2000FFF723
:1087D0004BFF10BD501F0020D4710020FB71002002
:1087E000E87100208B86000800F5E0700268914275
:1087F00003D343689A18914202D380680028F5D1C8
:108800007047DFF86007016891B94FF480318160EB
:108810004FF4805141604FF0FF31C160016104218C
:10882000DFF844274161C2F8BC11DFF8401701604E
:108830000120704701F1080313F0070305D001F18F
:108840000803C3F1080303F007035918D21A816122
:10885000C26042F001034B60511828234B60DFF8DF
:1088600004170969C16170472DE9F04F064601F10F
:10887000080010F0070083B008BF884607D001F158
:108880000800C0F1080000F0070000EB010802F149
:10889000080010F0070006D002F10800C0F108003F
:1088A00000F0070082181546A5EB0800A0EB0309AD
:1088B00043F0030003EB080BC8F80400AB4528BFE6
:1088C00005F0F4FC2879C00758BF05F0EFFCB9F1BA
:1088D000100F38BF05F0EAFCB069854209D1F06895
:1088E0004844F060C6F818B040F00100CBF804002E
:1088F0006DE1706985420BD1B0684844B060C6F83C
:1089000014B040F00101CBF8041040F80B005EE118
:10891000686800F00301012940F0AD80C008C00084
:108920000190C00820283AD2D5F808A0EF6800903E
:10893000BD4208BF05F0BAFC554508BF05F0B6FCBE
:1089400068680099C008C000B0EBC10F18BF05F0FF
:10895000ADFC009806EBC00000F128018A4507D065
:1089600031698A45C0F08280DAF80C10A9427DD1C5
:10897000574506D1009A3068012191408843306004
:1089800076E02830874205D0306987426ED3B868D8
:10899000A8426BD1CAF80C70C7F808A068E0EF686D
:1089A000D5F818A0AF420CD0A8683169884223D30B
:1089B000C168A94204BFB968A9421DD1C760B860A7
:1089C0001CE005F11400076837B905F110000768CD
:1089D000A7B101E00846076807F114010A68002AF8
:1089E00002BF07F110010A68002AF3D131698842F9
:1089F00002D30021016001E005F058FCBAF1000F3C
:108A000036D0E86906EB800000F5987001688D4269
:108A100008D10760A7B9EA697068012191408843CD
:108A2000706025E03069824508D3DAF81000A8426A
:108A300014BFCAF81470CAF8107001E005F036FCD3
:108A4000B7B13069874211D3C7F818A0296929B195
:108A5000814226BF39618F6105F028FC686938B111
:108A60003169884202D37861876101E005F01EFC1C
:108A700001984519814468684008400068604FEAE1
:108A8000D90549F00100CBF8040049F80B90202DDE
:108A900023D206EBC50000F12807B9F1100F38BF4B
:108AA00005F004FC306820FA05F1C907BA4604D481
:108AB0000121A9400843306006E0B8683169884266
:108AC0002CBF824605F0F2FBC7F808B0CAF80CB01C
:108AD000CBF808A0CBF80C7079E05FEA192108BF49
:108AE000002023D0B1F5803F28BF1F201ED2A1F562
:108AF0008070000C00F008008140A1F58052120C3B
:108B000002F004029140A1F580431B0CC0F10E005D
:108B100003F00203801AC01A994000EBD130C11D46
:108B200029FA01F202F0010101EB4000CBF81C0030
:108B30000022CBF81420CBF8102006EB80017268DD
:108B400022FA00F3DB0701F5987107D4012303FA39
:108B500000F010437060C1F800B01DE01F280968E4
:108B60000EBF00204008C0F1190009FA00F000E033
:108B700011464A68D208D2004A4514D0C20F01EB10
:108B8000820202F1100340001A68002AF0D1306915
:108B900083421AD3C3F800B0CBF81810CBF80CB04E
:108BA000CBF808B013E032698868914228BF904240
:108BB0000BD3C0F80CB0C1F808B0CBF80800CBF864
:108BC0000C100020CBF8180001E005F06FFB08F155
:108BD000080000F005BE2DE9FA4D0546DFF88403D4
:108BE000006884B008B9FFF70CFEDFF87803049939
:108BF000806841182F31401E21EA0000049981420B
:108C000080F0AB8105F5D876B16841B1D5F8B021D7
:108C10008018824280F0A1818142C0F09E8105F0DF
:108C200049FB00281EBF0446D0F8008014F1010F54
:108C300000F09381D5F8B0014044C5F8B0017168E7
:108C4000814238BF01467160A86980BB286908B1BC
:108C5000844200D22C613461C6F814800020F06197
:108C600005F12801BF48006868624FF0FF302862B4
:108C70000020C960896001F10802801C1031D260B7
:108C800020289260F5D3B848854203D1A8F1280284
:108C9000214629E055F8040CC00805EBC000A0F1FE
:108CA000080108EB0400401AA0F128021CE005F5B9
:108CB000E071084600E08068D0B1026843689A1805
:108CC0009442F8D1027B120712D4AA6903689A422F
:108CD0000ED347683B449A420AD208EB0701416031
:108CE000E868A96908EB00022846FFF7A3FD1EE12A
:108CF00028698442084638BF2C6108EB040100E073
:108D0000806880B102688A42FAD1017B09070AD4DF
:108D100004604168414441602146049B284606B0F6
:108D2000BDE8F04DA0E5AF6939462846FFF75CFD88
:108D300001684068401802902F3800F1080111F0D6
:108D4000070105D000F10801C1F1080101F0070198
:108D5000081807F11001884234BF0097009000986E
:108D60000830019004F10801009800F1180A11F090
:108D700007014FF0000BA8F1280005D004F108010D
:108D8000C1F1080101F007010A19401AAA61E8605F
:108D900040F001015160801828214160714800694C
:108DA000E861019810F0070018BF05F07FFA0099FC
:108DB0001B20486005F5E071B1E80C500198A0E86F
:108DC0000C503461C6F81480C6F81CB00198B0612C
:108DD000029800E08A460722CAF804200AF104013A
:108DE0000A1D82420BF1010BF4D3BBF1020FB8BF95
:108DF00005F05CFA0098B84200F09980C01BC119D8
:108E0000C4084A68520852004A6040F00101796083
:108E1000C051202C20D205EBC40101F128061028F6
:108E200038BF05F043FA286820FA04F1C907B046B4
:108E300004D40121A1400843286006E0B0682969F4
:108E400088422CBF804605F031FAB760C8F80C7034
:108E5000C7F80880FE606AE0010A08BF002223D03C
:108E6000B1F5803F28BF1F221ED2A1F58072120CDF
:108E700002F008029140A1F580531B0C03F004039B
:108E80009940A1F58044240CC2F10E0204F00204C2
:108E9000D21A121BA14002EBD131CA1D20FA02F3F3
:108EA00003F0010202EB4102FA6100237B613B61A6
:108EB00005EB82016B6823FA02F4E40701F598716F
:108EC00005D401209040184368600F601CE01F2A01
:108ED00009680EBF00225208C2F1190200FA02F21C
:108EE00000E019464B68DB08DB00834210D0D30F4B
:108EF00001EB830303F1100452002368002BF0D12F
:108F00002869844211D32760B961FF60BF600EE019
:108F10002A698868914228BF904206D3C7608F6053
:108F2000B860F9600020B86101E005F0BFF9E868B9
:108F30000499814211D2401AE860A969049A521832
:108F4000AA6140F001005060049840F003004860BE
:108F500006B001F10800BDE8F08D002006B0BDE8C4
:108F6000F08D0000F8700020045D00206859883CF6
:108F70002DE9F04D0446884600265FEA1820C8F126
:108F8000000B08BF002123D0B0F5803F28BF1F2170
:108F90001ED2A0F58071090C01F008018840A0F5EF
:108FA0008052120C02F004029040A0F580431B0C8A
:108FB000C1F10E0103F00203891AC91A984001EBAE
:108FC000D030C11D28FA01F202F0010101EB40018D
:108FD00004EB8100D0F8300128B31F290EBF002216
:108FE0004A08C2F1190208FA02F2002300E0520016
:108FF0004768FF08FF00A7EB08075F4503D25FEA59
:10900000070B06460BD04769D50F00EB8500002FF4
:1090100000691CBF87423B460028E8D1184600285B
:109020003CD1002E3CD10120884040004142084301
:109030006168084000F0678141420840411E080B0A
:1090400000F0100021FA00F2510901F0080122FAA3
:1090500001F39A0802F00407FB405A0802F00205E7
:10906000081823FA05F23844C2F3400328181818E8
:1090700022FA03F1081804EB8000D0F830010DE06B
:1090800008464168C908C900A1EB080159453CBF21
:109090008B46064601690029F2D140690028F0D1CB
:1090A000002E00F03081A068A0EB0800834580F01E
:1090B0002A8120698642C0F024817068C008C000FF
:1090C00008EB0B01884208EB060518BF05F0EEF827
:1090D000AE4280F01681F768D6F818A0B7420CD0DF
:1090E000B0682169884223D3C168B14204BFB9681E
:1090F000B1421DD1C760B8601CE006F114000768DA
:1091000037B906F110000768A7B101E00846076803
:1091100007F114010A68002A02BF07F110010A686A
:10912000002AF3D12169884202D30021016001E0C5
:1091300005F0BCF8BAF1000F38D0F06904EB8000FC
:1091400000F5987001688E4209D10760380014D18B
:10915000F2696068012191408843606026E02069DF
:10916000824508D3DAF81000B04214BFCAF8147070
:10917000CAF8107001E005F099F8BFB12069874284
:1091800012D3C7F818A0306930B12169884226BFD0
:109190003861876105F08AF8706938B121698842C1
:1091A00002D37861876101E005F080F8BBF1100F10
:1091B0000CD208EB0B0040F00300706008EB0B00D2
:1091C0008019416841F00101416096E048F00300D8
:1091D00070604BF0010068604FEADB004BF805B0AF
:1091E00020281DD204EBC00101F12807216821FAD3
:1091F00000F2D207BB4605D4012202FA00F0084370
:10920000206006E0B868216988422CBF834605F0DB
:109210004DF8BD60CBF80C50C5F808B0EF606CE0BD
:109220005FEA1B2108BF002023D0B1F5803F28BF93
:109230001F201ED2A1F58070000C00F008008140B4
:10924000A1F58052120C02F004029140A1F5804376
:109250001B0CC0F10E0003F00203801AC01A9940E3
:1092600000EBD130C11D2BFA01F202F0010101EB3C
:109270004000E86100226A612A6104EB80016268B3
:1092800022FA00F3DB0701F5987106D4012303FAF3
:1092900000F0104360600D601CE01F2809680EBFDD
:1092A00000204008C0F119000BFA00F000E0114660
:1092B0004A68D208D2005A4510D0C20F01EB820290
:1092C00002F1100340001A68002AF0D1206983429D
:1092D00011D31D60A961ED60AD600EE02269886860
:1092E000914228BF904206D3C5608D60A860E960B6
:1092F0000020A86101E004F0D9FF06F10800BDE8F4
:10930000F08D04F0D3FF0020BDE8F08D2DE9F84F7B
:1093100004468846606841420840411E080B00F040
:10932000100021FA00F2510901F0080122FA01F3BC
:109330009A0802F0040223FA02F56B0803F0020314
:10934000081825FA03F61018C6F340051818284423
:1093500026FA05F1081804EB8000D0F830014168C6
:10936000C908C9000646A1EB080A09E00846416899
:10937000C908C900A1EB080151453CBF8A46064611
:1093800001690029F2D140690028F0D120698642A4
:10939000C0F0C4807068C00808EB0A09C0004845E6
:1093A00008EB060B18BF04F081FF5E4580F0B68025
:1093B000F768B569B7420CD0B0682169884223D3F9
:1093C000C168B14204BFB968B1421DD1C760B8607D
:1093D0001CE006F11400076837B906F110000768B1
:1093E000A7B101E00846076807F114010A68002ADE
:1093F00002BF07F110010A68002AF3D121698842EF
:1094000002D30021016001E004F050FF002D34D0B0
:10941000F06904EB800000F5987001688E4209D174
:109420000760380011D1F2696068012191408843DA
:10943000606022E02069854205D32869B04214BFEC
:109440006F612F6101E004F031FFB7B120698742FD
:1094500011D3BD61306930B12169884226BF3861BE
:10946000876104F023FF706938B12169884202D313
:109470007861876101E004F019FFBAF1100F09D299
:1094800049F00300706009EB0600416841F00101FA
:1094900041603FE048F0030070604AF00100CBF803
:1094A00004004AF80BA0D4F808804FEAD805202D14
:1094B00028BF04F0FBFEB8F1000F27D0D4F81490B9
:1094C000009504EBC50000F12805B8F1100F38BF76
:1094D00004F0ECFE2068009920FA01F2D1072F4633
:1094E00005D4009A012191400843206006E0A86855
:1094F000216988422CBF074604F0D8FEC5F80890C1
:10950000C7F80C90C9F80870C9F80C50C4F808A046
:10951000C4F814B006F10800BDE8F28F04F0C6FEEE
:109520000020BDE8F28F2DE9F04F83B00546C0461C
:10953000C046F52DDFF8C04780F007810B2D31BF05
:10954000102705F10B00C008C7002168FE0821FAAA
:1095500006F010F0030F42D0C04300F0010086195E
:1095600004EBC60000F12808F700D8F80850686836
:10957000C008C000B84218BF04F098FED5F80890A3
:10958000454508BF04F092FE4D4508BF04F08EFE2D
:109590006868C008C000B84218BF04F087FEC8451C
:1095A00005D120680121B140884320600DE0206989
:1095B000814508D3D9F80C00A84204D1C8F8089016
:1095C000C9F80C8001E004F071FE47F00300686008
:1095D00078190835416841F001014160FDE0A1685A
:1095E000B94280F0C480002800F0A680012505FA69
:1095F00006F149004A42B040114308404142084048
:10960000411E080B00F0100021FA00F2510901F090
:10961000080322FA03F18A0802F0040221FA02F692
:10962000710801F00208181826FA08F11018C1F3A1
:1096300040064044301821FA06F202EB000804EB21
:10964000C80000F128094FEAC80AD9F80860706814
:10965000C008C000504518BF04F028FED6F808B076
:109660004E4508BF04F022FE5E4508BF04F01EFE12
:109670007068C008C000504518BF04F017FED945F7
:1096800005D1206805FA08F1884320600DE02069C3
:10969000834508D3DBF80C00B04204D1C9F808B008
:1096A000CBF80C9001E004F001FE47F0030070607D
:1096B000AAEB0708B819019048F001000199486029
:1096C000019848F80080A7684FEAD70ABAF1200F3E
:1096D00028BF04F0EBFD47B3CDF800A004EBCA00AF
:1096E000D4F8149000F1280A102F38BF04F0DEFDE2
:1096F0002068009920FA01F2D107D34605D40099D9
:1097000005FA01F10843206007E0DAF80800216952
:1097100088422CBF834604F0C9FDCAF80890CBF8F4
:109720000C90C9F808B0C9F80CA0C4F8088006F17C
:1097300008050198606150E06068C0B33946204672
:10974000FFF7E4FD050012D047E015F1400F28BFF8
:109750004FF0FF370BD205F10B00C008C70060685F
:1097600028B139462046FFF703FC050035D1A06833
:10977000B8421CD3C11B626910290AD3B8186061B2
:10978000A16041F001034360095047F003005060BD
:109790000AE00021A160616140F00301516080187E
:1097A000416841F00101416002F1080515E0E068FF
:1097B00087420DD2C01BA169E0607A18A26140F017
:1097C0000100506001F1080547F00300486004E023
:1097D00039462046FFF7FFF90546C046C0462846F1
:1097E00003B0BDE8F08F00B970472DE9F047A0F154
:1097F0000804C046C046DFF8005528698442C0F01E
:109800007482616801F00302012A00F06E82CA08C6
:109810004FEAC208CA0708EB040936D4226811F0DF
:10982000030F00F06482A41A84429044C0F05D8269
:1098300069698C4200F0D880D608202E70D2D4F806
:109840000CA0A768544508BF04F030FDBC4208BF17
:1098500004F02CFD6068C008C000B0EBC60F18BF54
:1098600004F024FD05EBC60000F128018F4205D06D
:1098700029698F4251D3F968A1424ED1BA453DD1F1
:1098800028680121B140884328604C4580F02D8232
:10989000D9F80400C10740F12882810700F17A81DC
:1098A000A969894540F0B580E868AC614044E8604A
:1098B00040F00101616069698C4202D10021696157
:1098C000A960E969814280F01282DFF83004006803
:1098D00008B9FEF796FFA969002900F00882E86838
:1098E000292824BF2846FEF77FFFE869E9688842F7
:1098F00080F0FD814FF0FF30E861F8E128308245CB
:1099000006D02869824508D3DAF80800A04204D1BD
:10991000C7F80CA0CAF80870B7E704F0C7FCB4E7B2
:10992000E768A669A7420BD0A168814222D3C86824
:10993000A04204BFB868A0421CD1CF60B9601BE050
:1099400004F114010F6837B904F110010F689FB1D9
:1099500001E011460F6807F114021368002B02BFE3
:1099600007F110021368002BF3D1814202D30020CB
:10997000086001E004F09AFC002E86D0E06905EB57
:10998000800000F5987001688C4209D107603800AA
:1099900011D1E2696868012191408843686074E7E9
:1099A0002869864205D33069A04214BF77613761C8
:1099B00001E004F07BFC002F3FF467AF2869874289
:1099C000ABD3BE61216929B1814226BF39618F6164
:1099D00004F06CFC606900283FF457AF29698842A5
:1099E0009BD37861876150E799F8040000F0030089
:1099F00003287FF44AAFC5F80880D9F8040040086E
:109A00004000C9F8040048F00100606048F8048094
:109A10006DE16969894508D1A8686C614044A86016
:109A200040F001016160005161E1C008C0004FEAEF
:109A3000D00ABAF1200F804436D2D9F80C70D9F888
:109A40000860B94508BF04F031FCB14508BF04F017
:109A50002DFCD9F80400C008C000B0EBCA0F18BF35
:109A600004F024FC05EBCA0000F128018E4206D068
:109A700029698E42C0F08180F16849457DD1B742A5
:109A800006D12868012101FA0AF18843286076E0AE
:109A90002830874205D0286987426ED3B868484588
:109AA0006BD1F760BE606AE0D9F80C70D9F8186025
:109AB0004F450DD0D9F808002969884223D3C168E1
:109AC000494504BFB96849451DD1C760B8601CE06D
:109AD00009F11400076837B909F110000768A7B148
:109AE00001E00846076807F114010A68002A02BF6E
:109AF00007F110010A68002AF3D12969884202D3CC
:109B00000021016001E004F0D1FB002E37D0D9F82C
:109B10001C0005EB800000F59870016889450AD1AA
:109B20000760380012D1D9F81C20686801219140E3
:109B30008843686023E02869864205D33069484538
:109B400014BF7761376101E004F0B0FBBFB1286951
:109B5000874212D3BE61D9F8101029B1814226BFC5
:109B600039618F6104F0A2FBD9F8140038B129697A
:109B7000884202D37861876101E004F097FB48F0E6
:109B80000100606048F80480686984420BD1C5F820
:109B90000880ACE040084000C9F8040048F001002B
:109BA000606048F804804FEAD807202F22D205EBE6
:109BB000C70000F12809B8F1100F38BF04F076FB98
:109BC000286820FA07F1C9074E4604D40121B9409C
:109BD0000843286007E0D9F80800296988422CBFAB
:109BE000064604F063FBC9F80840F460A660C4F8B8
:109BF0000C907CE05FEA182008BF002123D0B0F56C
:109C0000803F28BF1F211ED2A0F58071090C01F0F2
:109C100008018840A0F58052120C02F00402904026
:109C2000A0F580431B0CC1F10E0103F00203891A59
:109C3000C91A984001EBD030C11D28FA01F202F098
:109C4000010101EB4001E16100226261226105EB4B
:109C500081006A6822FA01F3DB0700F5987006D4E8
:109C6000012303FA01F11143696004601CE01F291C
:109C700000680EBF00214908C1F1190108FA01F17D
:109C800000E010464268D208D200424510D0CA0F08
:109C900000EB820202F1100349001A68002AF0D199
:109CA00029698B4211D31C60A061E460A4600EE0BE
:109CB0002A698168904228BF914206D3CC608460B3
:109CC000A160E0600020A06101E004F0EFFA286AE2
:109CD000401E28620BD1D5F8C80100E0806800283A
:109CE000FCD14FF0FF30286201E004F0DFFAC046FB
:109CF000C046BDE8F0870000045D0020F870002039
:109D000070B504460026DFF80854CA20E8615320E5
:109D1000E86100F018F8002811D0286820F0400011
:109D200028602868216808432860A068A860A8689F
:109D3000616840EA0140A86000F024F80126FF2095
:109D4000E861304670BD81B000200090DFF8C403A8
:109D50000168490613D44FF0FF310160016801F03A
:109D60004001009A521C0092009AB2F5803F01D047
:109D70000029F3D00068800900F0010000E0012014
:109D800001B07047DFF88C03016821F080010160A9
:109D9000704781B000200090DFF87813CA208861F6
:109DA00053208861086820F0A0000860086800F06F
:109DB0002000009A521C0092009AB2F5003F01D098
:109DC0000028F3D00868400900F00100FF228A61F2
:109DD00001B070472DE9F04107460E460024DFF838
:109DE0002C53002FA86804D140060AD42046F070F6
:109DF00007E0400603D5307800F0A5F901E02046E1
:109E0000F0703078002F09D07178090241EA0040E3
:109E1000B1780843F17840EA014611E000F088F992
:109E20000746707800F084F98046B07800F080F939
:109E30004FEA082141EA07410843F17840EA014628
:109E4000CA20686253206862FFF77DFF00280FD0A8
:109E5000DFF8C40230402860FFF794FFA86880064E
:109E600005D4FFF796FF002802D0012400E001246A
:109E7000FF2068622046BDE8F08110B50C46DFF88F
:109E80008C120968DFF8902211400A0C02F03F039F
:109E900023700B0A03F07F03637001F07F01A17050
:109EA00002F04001E17000280BD1207800F04BF95E
:109EB0002070607800F047F96070A07800F043F9F6
:109EC000A07010BDDFF85412486A09687047F8B5F1
:109ED00006460D460024002E06D16878C10603D53B
:109EE00000F0EF000A306870002E05D0687800F0AE
:109EF0002AF9A87800F027F9E878002E09D06978C7
:109F0000090241EA0040A9780843297840EA41362D
:109F100010E000F00DF90646687800F009F90746F0
:109F2000A87800F005F9390241EA0641084329788A
:109F300040EA4136DFF8E451CA2028625320286203
:109F4000FFF701FF00280FD0DFF8D4013040286070
:109F5000FFF718FF6868800605D4FFF71AFF00288E
:109F600002D0012400E00124FF2028622046F2BD37
:109F700010B50C46DFF8A4110968DFF8A4211140E0
:109F80000A0CE2700A0A02F01F02627001F03F023E
:109F9000A270490B01F00701217000280BD1E07875
:109FA00000F0D1F8E070607800F0CDF86070A07833
:109FB00000F0C9F8A07010BDDFF85411CA22CA61C0
:109FC0005322CA610A68D208D2000A600A681043A4
:109FD0000860FF20C8617047DFF84811CA220A6193
:109FE00053220A610860FF2008617047DFF83401DE
:109FF000006880B2704781B000210091DFF8101135
:10A00000CA22CA615322CA610028086804D040F4F9
:10A0100080600860012012E020F4806008604868D9
:10A0200000F00400009A521C0092009AB2F5803FA2
:10A0300001D00028F3D04868800800F00100FF221A
:10A04000CA6101B0704781B000220092364A009286
:10A05000009A02EB800000900098016001B0704708
:10A0600081B00021009130490091009901EB8000FE
:10A0700000900098006801B07047254ACA23D36158
:10A080005323D36100F0040320F004000029116879
:10A0900005D008431060906B1843906305E021EAF7
:10A0A00000001060906B98439063FF20D061704770
:10A0B0000021184A12681D4B1A40024200D00121AB
:10A0C0000846704730B40021114A936B03F0040333
:10A0D00014680440050C45EAD0352B4023435268F0
:10A0E00002EA101002D0000400D00121084630BC62
:10A0F000704708490003000C40F080000A6802F035
:10A10000800262EA000008607047000000280040FA
:10A11000082800400C2800407F7F7F000428004072
:10A120003FFFFF0014280040502800407F7F0100BF
:10A13000002101E0491C0A38C0B20A28FADA40EAD4
:10A140000110C0B27047010901EB810200F00F005D
:10A1500000EB4200C0B270472DE9F04104460C21EB
:10A16000206990FBF1F202EB4201B0EB810144BFA8
:10A170000C31521E002A47D56069C2F10043984253
:10A180004ADB60691518284604F0AAF840F26D18F9
:10A1900008FB0500A168E56862682368DFF880C0F5
:10A1A000DFF87CE018274FF4B46691FBF7F7281826
:10A1B00092FBF6F6381893FBFCFC30186044194DFE
:10A1C000281807EB4705A1EBC5014FF4616569430A
:10A1D0000EFB00104FF4B46101FB1621C1EB01121C
:10A1E00000EB820018180EFB1C05226A2946204647
:10A1F00004F093F8206A0128A8BFA5F5616504F072
:10A2000033F9281ABDE8F081012ABADB6FF000406B
:10A210006369801A9842B4DA4FF0FF30BDE8F081EC
:10A2200080510100209CFFFF13F0004C03D55B42DE
:10A23000524263F100039CEA210C00F0178010B534
:10A24000644603D34942404261F1000100F00EF838
:10A25000640004D34942404261F10001244203D525
:10A260005B42524263F1000310BD00001B4213D158
:10A27000094236D12AB18446B0FBF2F002FB10C28B
:10A28000704704F03FB9FCD30022002370470B0055
:10A290000200002100207047904271EB030CF6D3BE
:10A2A00070B5B1FA81F4B3FA83F52C1BA340C4F165
:10A2B000200532FA05F63343A2405FF00046E6403F
:10A2C00002E05B085FEA3202841A71EB030524BFE7
:10A2D000204629467641F4D302000B0030000021CD
:10A2E00070BD012ACFD970B5140C20D0B1FA81F419
:10A2F000B2FA82F5C4F120046419B4F12006D6D371
:10A30000B2405FF00044F440002502E052085FEAEA
:10A310003303C61A71EB020E24BF30467146644106
:10A320006D41F3D302000B002000290070BD0C46E4
:10A33000B1FBF2F102FB11452D0445EA1045B5FBD6
:10A34000F2F402FB145580B240EA0545B5FBF2F089
:10A3500002FB105240EA044070BD000051EC100BAB
:10A3600000B500F003F841EC100B00BD40F2FF7C9B
:10A370000B0D4DD0634566D230B421EA035141F450
:10A38000801103F2FD3C5FEA5C0C01D300184941E7
:10A39000890041EA907180004FF440140023E202EA
:10A3A000D50AB1F5100107D46D081DD2091B641937
:10A3B00000184941491BF7D56D080AD20919641BD9
:10A3C00000184941491BEFD56D08F7D301E0520849
:10A3D00017D0C01861419B1AAC4100184941801A3E
:10A3E000A941F4D452080AD0C01AA1419B186C416B
:10A3F00000184941801AA941E9D45208F4D15B1CE4
:10A400006C4161084FEA330001EB0C5130BC7047DE
:10A4100050EA0103FBD030B4B1FA81F311B9B0FABC
:10A4200080F41B190B3BB3F120042FBF00FA04F199
:10A430009940C3F1200420FA04F438BF2143984026
:10A44000D3F101039DE76345E1D011F5801FDED80C
:10A4500050EA4101DBD0D94304F056B800206149ED
:10A460000860704738B52DED068BB0EE408AF0EEEF
:10A47000608AB0EE419A044620EE000A08EEA80A6F
:10A4800009EE090A10EE100AFBF73EF841EC100B3A
:10A49000FFF764FF51EC100BFBF700FA09EE900A8E
:10A4A0009FED4CABB0EE480A80EE290A10EE100A80
:10A4B000FBF72AF841EC100B00F036F953EC102BA7
:10A4C00051EC1A0BFBF7A4F8FBF7E8F908EE100AB9
:10A4D00088EEA90A10EE100AFBF716F841EC100BF3
:10A4E00000F022F953EC102B51EC1A0BFBF790F80B
:10A4F000FBF7D4F908EE900A89EE290A10EE100A4B
:10A50000FBF702F841EC100B00F00EF953EC102BA6
:10A5100051EC1A0BFBF77CF8FBF7C0F909EE100AB7
:10A52000002C06D1B2EE040AF0EE409A9FED2BAA61
:10A5300005E0B3EE040AF0EE409A9FED29AA10EE72
:10A54000100AFAF7E1FF02460B4614461D4618EEC4
:10A55000100AFAF7D9FF21F0004122462B46FBF7FB
:10A560003FF82AD219EE900AFAF7CEFF02460B46C0
:10A5700014461D4618EE900AFAF7C6FF21F0004176
:10A5800022462B46FBF72CF817D219EE100AFAF7E1
:10A59000BBFF21F0004102460B4614461D461AEE51
:10A5A000100AFAF7B1FF22462B46FBF719F804D23E
:10A5B0000C480168491C016002E00020094908605C
:10A5C00008480068152801DB012000E00020BDECF0
:10A5D000068B32BD46DF617EDCA54C400000A04208
:10A5E00000008C42B4710020B5EEC00AF1EE10FA02
:10A5F00002D4B1EEC00A70476FF0004C00EE10CAF2
:10A6000003F082BFD0B52DED048B82B041EC180B66
:10A610008DED008BDDE90023C3F30A5140F2FF7298
:10A62000914213D0002904BF190350EA113011D010
:10A6300051EC180B00220023FAF7D2FF3DBF81F046
:10A64000004141EC180B0824002409E0190350EAEA
:10A650001130EDD002B051EC180BBDEC048BD0BD25
:10A6600051EC180B2B4A2C4BFAF7BAFF1CD29FED7A
:10A670002C9B51EC190B53EC182BFDF735FF0646BC
:10A680000F4653EC182B51EC190BFBF793F832469D
:10A690003B46FAF7BDFFFFF769FE41EC100B51ECAA
:10A6A000180B53EC102B1EE001221C4BFAF798FFFD
:10A6B00023D29FED1B9B51EC190B53EC182BFDF78C
:10A6C00013FF06460F4653EC182B51EC190BFBF702
:10A6D00071F832463B46FAF79BFFFFF747FE84F0DE
:10A6E000020453EC182B03F015FF02B02246BDEC18
:10A6F000048BBDE8D04004F06BB804F061F921216F
:10A70000016002B04FF0FF30BDEC048B6FF00041F0
:10A71000D0BD0000CE3B7F669EA0E63F0000F03F2C
:10A72000000000000000F03F80B551EC100BFFF777
:10A7300069FF41EC100B01BD002848BF4042704743
:10A74000D54800F15C01016500210162C1614162EF
:10A75000C1648162817001700121417000210B464A
:10A7600003E000EB8102D362491C0729F9DB19469B
:10A7700041608160C16001614161816181644165C5
:10A780008165704738B50024C34D2878012801D170
:10A79000204632BDE869072806DBC01FE861A878BB
:10A7A000002801D10120A870DFEDB41A9FEDB42A72
:10A7B00060EE022A95ED013A43EE212AC5ED042A06
:10A7C00020EE823AD5ED023A03EEA13A85ED053A44
:10A7D00061EE020A95ED030A40EE210AC5ED060A74
:10A7E000C5ED012A85ED023AC5ED030A22EEA20A63
:10A7F00003EE030A00EEA00AFFF7F6FEE86905EB98
:10A80000800181ED0B0AA978002900F0CC80411C61
:10A81000072291FBF2F2C2EBC202891A05EB810119
:10A82000D1ED0B0A70EE600AB0EEE01ADFED951A7A
:10A83000B4EE611AF1EE10FA03D5296A491C2962B7
:10A8400006E0214629626978002901D10121697059
:10A85000296A652906DB2146697029626962E96413
:10A860006965A965A96C00290CD1B1EE001AF4EE56
:10A87000410AF1EE10FA41DB0121A964E96C491C9F
:10A88000E9643BE001290CD1E96C491CE9649FEDC6
:10A890007E1AF4EE410AF1EE10FA2FD50221A964D6
:10A8A0002CE002290CD1E96C491CE9649FED771A70
:10A8B000F4EE410AF1EE10FA20D50321A9641DE05F
:10A8C00003291BD1E96C491CE964B9EE001AF4EEC6
:10A8D000410AF1EE10FA11DB1F290CDA696A491CF2
:10A8E0006962022905DBAA6A142A02DA491E696232
:10A8F00001E02146A9622146A964E964E96C652961
:10A9000002DAA96A652903DB2146E964A964A96220
:10A91000696A012902DBAA6A521CAA62142902DBB5
:10A92000012421462970801D072190FBF1F1C1EB24
:10A93000C101401A05EB8000D0ED0B0A30EE600A31
:10A940008DED000A032200A9286D00F031F80322E2
:10A950001146286D00F040F8DFED4D0AB4EE600AB4
:10A96000F1EE10FA03D5686D401C686501E0002027
:10A970006865686DC92801DB0020A865B4EE600A2F
:10A98000F1EE10FA09DBDFED400AB4EE600AF1EEF9
:10A9900010FA02D5A86D401CA865A86DC92802DB75
:10A9A000012420462870E869401CE861204632BD39
:10A9B0000388934201D30023038003885B1C038038
:10A9C0009BB2934201D300220280028800EB8200F6
:10A9D00009684160012070472DE9F0412DED028B9F
:10A9E00004460D4616469FED2B8A0027B4F90080D9
:10A9F00000EE105AF8EEC08A00F022F880EE280A25
:10AA000004E0A6F101080FFA88F87F1C3FB2AF42BC
:10AA10000FDA04EB8800D0ED010A70EEC00A00EEF8
:10AA2000A08AB8F1010FECDBA8F101080FFA88F851
:10AA3000EBE788EE280ABDEC028BBDE8F081000050
:10AA400030B49FED140A0023B0F900400EE024B2A8
:10AA5000250006D400EB8505D5ED010A30EE200A6D
:10AA6000641E24B2002C00D5541E5B1C1BB28B420A
:10AA7000EDDB30BC7047084840787047D0CCCC3D07
:10AA80006666663FCDCCCC3D01008040FEFF7FC0B6
:10AA9000CDCCCC3E00000000286E002010B50FF297
:10AAA000EC40F9F7FBFDDFF8DC440022E42120460E
:10AAB000F7F794FC5020606010BD000030B4DFF860
:10AAC000C42492F8D83002EB8303C3F8981090EDB9
:10AAD000000A82ED200A0C2192F8D83011FB0323E2
:10AAE00083ED020A90ED010A02F1800383ED010A71
:10AAF00092F8D84011FB042484ED030A90ED020A79
:10AB000083ED020A92F8D80011FB002080ED040AC0
:10AB100092F8D800401C82F8D80002F1D804C0B2E4
:10AB20000A2804DB002082F8D800012060709FED25
:10AB3000D10ADFEDD00A9FEDCF1A00206478012CF6
:10AB40002ED1044613E011FB0425D5ED021A30EE98
:10AB5000210AD5ED031A70EEA10AD5ED041A31EEE3
:10AB6000211A02EB8405D5F898502818641C0A2C89
:10AB7000E9DBF2EE041A80EE210A83ED030AB2EE5D
:10AB8000040A80EE800A83ED040AB2EE040A81EE24
:10AB9000000A83ED050A0A21B0FBF1F0186403E016
:10ABA000D86018615861186430BC7047DFF8D4036E
:10ABB00090F8D9007047000030B400219FEDAD0A35
:10ABC000DFEDAC0A9FEDAB1A0A46DFF8B83303F1AC
:10ABD0008C051CE002EB420403EB8404D4ED021A62
:10ABE00093ED232A71EEC21A01EEA10AD4ED031AE5
:10ABF00095ED012A71EEC21A41EEA10AD4ED041AB4
:10AC000095ED022A71EEC21A01EEA11A521C0A2A0F
:10AC1000E0DBF2EE041A81EE211ADFEDC51AB2EE86
:10AC2000042A80EE020AB4EE610AF1EE10FA19D598
:10AC3000B2EE040A80EE800AB4EE610AF1EE10FA78
:10AC400010D5B4EE611AF1EE10FA0BD5A96B5A6863
:10AC50005118A963814203D30020A863022104E0B4
:10AC6000012102E008462A469063084630BC70473E
:10AC7000C44800F18001D0F8800088644868C86446
:10AC8000886808657047000010B52DED048B00241E
:10AC9000BC4901F1800090ED120AD1ED200A30EE9E
:10ACA000608A90ED130AD0ED010A70EE608A90ED93
:10ACB000140AD0ED020A30EE609A00F02FF8DFEDB2
:10ACC000A80A20EE200ADFEDA70AC0EE209A28EE9F
:10ACD000080A08EEA80A09EE090A10EE100AFAF7A7
:10ACE00013FC41EC100BFFF739FB51EC100BFAF79A
:10ACF000D5FD00EE100ADFED9C0AB4EE600AF1EE1D
:10AD000010FA07DB9FED990AF4EE409AF1EE10FA83
:10AD100000DB01242046BDEC048B10BD10B52DEDE9
:10AD2000068B04469FED538A964800F1C801D1ED89
:10AD3000028A91ED019AD0ED329A29EEA90A09EE24
:10AD4000090A08EEA80AFFF74FFCB0EE40AAD4EDBE
:10AD5000020A94ED011A94ED000A20EE000A01EEB9
:10AD6000010A00EEA00AFFF73FFCD4ED000A69EEED
:10AD7000A00A94ED011A49EE010A94ED021A48EE78
:10AD8000810A2AEE000A80EE800ADFED790AB4EE2D
:10AD9000600AF1EE10FA1EDADFED760AB4EE600A10
:10ADA000F1EE10FA02D59FED748A14E0DFED730A1C
:10ADB000B4EE600AF1EE10FA0DDAFFEE000AB4EE1E
:10ADC000600AF1EE10FA02D59FED6B8A03E003F002
:10ADD000FDFDB0EE408AB0EE480ABDEC068B10BD1A
:10ADE00080B52DED028B674800F1800191ED028A5C
:10ADF000D1ED010A90ED200A20EE000A00EEA00A33
:10AE000008EE080AFFF7F0FB88EE000A03F010FED8
:10AE1000DFED5B0A20EE200ABDEEC00A10EE100A3C
:10AE2000BDEC028B02BD80B5FFF7DAFF10F1460FD3
:10AE300003DA54490860012002BD002002BD80B53C
:10AE4000FFF7CEFF4F4909680A1A00D5421A4E484B
:10AE5000282A03DB0168491C016001E00021016030
:10AE60000168032903DB00210160012002BD0020ED
:10AE700002BD000000000000F0B58BB000A80FF28A
:10AE800018112822F7F7E8FA00243E4D05F1C00614
:10AE9000707E002801D1642048E0012000E0401CC1
:10AEA00005280DDAD5F8C01000AA52F830209142DA
:10AEB000F5D300AA02EBC00252688A42EFD30446DF
:10AEC00095F8E00005F1E007E4B2A04207D17978F7
:10AED000A14204D0F06969680818F06114E0A0424A
:10AEE00012D0042C02D179788C4201D1002807D1EC
:10AEF000D5F8C02079780FF2C800F9F7CFFB7C7045
:10AF00000020F06185F8E040F06947F23051884256
:10AF100009D395F8E02079780FF2BC00F9F7BEFB71
:10AF20000020F0617C7078786430C0B20BB0F0BD66
:10AF30009A99993E0020134901F1C002D1F8C0301E
:10AF40000A2B04D353694968C918516101E00146CD
:10AF500051615169B1F57A7F01D350610120704789
:10AF60000000B443D80FC9400100E0400100704127
:10AF70006766663F666666BFD80F49400100803F3E
:10AF8000E42E6542E8690020B0710020234450435C
:10AF90004D20494E495400009CFFFFFFFFFFFFFF7B
:10AFA000000000000200000003000000320000006A
:10AFB000330000006400000065000000FFFFFF7F19
:10AFC0004450434D20627269676874207570202573
:10AFD00064202564000000004450434D204C7578E7
:10AFE000206368616E6765642025642D3E256400DA
:10AFF0001EF0040F0CBFEFF30880EFF3098000F0A0
:10B000003DB870471EF0040F0CBFEFF30880EFF35C
:10B01000098000F033B8FEE71EF0040F0CBFEFF319
:10B020000880EFF3098000F029B870471EF0040F84
:10B030000CBFEFF30880EFF3098000F01FB87047F2
:10B040001EF0040F0CBFEFF30880EFF3098000F04F
:10B0500015B870471EF0040F0CBFEFF30880EFF334
:10B06000098000F00BB870471EF0040F0CBFEFF31F
:10B070000880EFF3098000F001B87047F9F7CFBA04
:10B0800038B50C46DFF8A8552968C90706D52968E0
:10B090004908490029602968C907FCD400220146F3
:10B0A000284600F0D3FCDFF88C15284600F0EBFCB6
:10B0B000214628464160C04601212846BDE834406B
:10B0C00000F0AEBCF8B5DFF870452078401C207069
:10B0D000DFF868552878401C2870FCF7EFFC68788A
:10B0E000F021084202D09920FCF7A4F9FCF718FAE5
:10B0F0006878401C687002F027FF6878F0210842E9
:10B1000002D09920FCF796F96878401E6870C0B2AA
:10B11000002801D1FCF7FEF9012003F0EFFC012823
:10B1200040F08C80012003F0F1FCDFF8140500787A
:10B1300000281CD1FCF7F4F92078411E217000286A
:10B1400002D19820FCF776F92878012804D16868A4
:10B15000002801D0FCF7DAF92878401E2870FCF7A7
:10B16000D9F90FF20050BDE8F240F9F7E8B800262F
:10B170000121DFF8D00400F079FB002853D0DFF87C
:10B18000C864DFF8AC74384600F066FC002825D0AF
:10B190003046461E0028F6D10021DFF8B00400F04A
:10B1A0003FFC0021384600F03BFC0FF2C040F9F7AD
:10B1B00075FAFDF775F9FCF7B3F92078411E217097
:10B1C000002802D19820FCF735F92878012847D1CA
:10B1D0006868002844D0FCF799F941E04FF48051A9
:10B1E000DFF86C0400F042FB002812D0FCF798F95D
:10B1F0002078411E2170002802D19820FCF71AF90E
:10B20000287801282CD16868002829D0FCF77EF91D
:10B2100026E0DFF84014DFF8400403F07FFC064628
:10B22000FDF73EF904E0DFF834140220FAF7EAFDF6
:10B23000002E03D00FF23C40F9F781F8FCF770F9CB
:10B240002078411E2170002802D19820FCF7F2F8E6
:10B250002878012804D16868002801D0FCF756F945
:10B260002878401E2870BDE8F140FCF753B938B586
:10B27000DFF8C4432078401C2070DFF8C0532878E2
:10B28000401C2870FCF71AFC6878F021084202D0B4
:10B290009920FCF7CFF8FCF743F96878401C6870F8
:10B2A00002F052FE6878F021084202D09920FCF7A3
:10B2B000C1F86878401E6870C0B2002801D1FCF760
:10B2C00029F9042003F01AFC002827D0042003F0F9
:10B2D0001DFCDB48007800281CD1FCF721F9207800
:10B2E000411E2170002802D19820FCF7A3F828788D
:10B2F000012804D16868002801D0FCF707F92878F4
:10B30000401E2870FCF706F90FF27830BDE8324095
:10B31000F9F715B8D2491020FAF774FDFCF700F9D7
:10B320002078411E2170002802D19820FCF782F875
:10B330002878012804D16868002801D0FCF7E6F8D5
:10B340002878401E2870BDE83140FCF7E3B838B5D6
:10B35000B94C2078401C2070B84D2878401C2870CB
:10B36000FCF7ACFB6878F021084202D09920FCF78A
:10B3700061F8FCF7D5F86878401C687002F0E4FDCD
:10B380006878F021084202D09920FCF753F86878D9
:10B39000401E6870C0B2002801D1FCF7BBF808203D
:10B3A00003F0ACFB002827D0082003F0AFFBA44833
:10B3B000007800281CD1FCF7B3F82078411E2170DA
:10B3C000002802D19820FCF735F82878012804D10C
:10B3D0006868002801D0FCF799F82878401E28708A
:10B3E000FCF798F80FF2A420BDE83240F8F7A7BFA9
:10B3F0009B490820FAF706FDFCF792F82078411ED9
:10B400002170002802D19820FCF714F82878012830
:10B4100004D16868002801D0FCF778F82878401E2D
:10B420002870BDE83140FCF775B838B5824C2078FB
:10B43000401C2070814D2878401C2870FCF73EFB92
:10B440006878F021084202D09920FBF7F3FFFCF75F
:10B4500067F86878401C687002F076FD6878F02123
:10B46000084202D09920FBF7E5FF6878401E68701B
:10B47000C0B2002801D1FCF74DF84FF48050FEF720
:10B4800021FE00282ED06E48007800284FF480500E
:10B4900022D1FEF72EFE4FF4003003F037FBFCF70D
:10B4A0003FF82078411E2170002802D19820FBF738
:10B4B000C1FF2878012804D16868002801D0FCF772
:10B4C00025F82878401E2870FCF724F80FF2C410E5
:10B4D000BDE83240F8F733BFFEF70BFE4FF4003003
:10B4E00003F014FBFCF71CF82078411E21700028A3
:10B4F00002D19820FBF79EFF2878012804D16868C4
:10B50000002801D0FCF702F82878401E2870BDE81A
:10B510003140FBF7FFBFF0B585B0474C2078401CA9
:10B520002070464D2878401C2870FCF7C7FA02208E
:10B5300003F002FC002862D00021022003F0DFFBB0
:10B54000022003F001FC002003F02EFB00A90020E4
:10B55000FEF793FC012003F023FC01214FF480202F
:10B5600003F08BFB0F20FEF77BFD06461020FEF755
:10B5700077FD0746012003F07DFB002003F07AFBF6
:10B5800031460F20FEF75FFD39461020FEF75BFDC8
:10B5900000214FF4802003F070FB012003F0F4FA47
:10B5A00001214FF0805003F073FB4FF4807003F0E3
:10B5B0004BFB3F20029040F2FF10039000200190CF
:10B5C00001A8FEF79DFB00A90020FEF703FC012067
:10B5D00003F04DFBFEF7DDFB0320FEF7EDFC4FF41F
:10B5E0008040FEF786FD4FF4800003F08FFA0121C2
:10B5F0004FF48040FEF741FD022003F0A5FBFBF76E
:10B600008FFF2078411E2170002802D19820FBF77F
:10B6100011FF2878012804D16868002801D0FBF7C1
:10B6200075FF2878401E2870FBF774FF05B0F0BD49
:10B630001064024020000010F9710020501F00200B
:10B64000F771002000000240809698005864024084
:10B6500000040240146F0020203F0020584A0020C0
:10B660003037002045585449302D52004558544930
:10B67000300000004D534720426F782046756C6CB7
:10B680000000000045585449352D52004558544992
:10B69000322D5200525443414C2D520080B54B493B
:10B6A000884209D10121084603F008FB002101204E
:10B6B000BDE8044003F002BB4549884209D101219D
:10B6C000022003F0FBFA00210220BDE8044003F051
:10B6D000F5BA4049884209D10121042003F0EEFA6D
:10B6E00000210420BDE8044003F0E8BA3A4988424A
:10B6F00009D10121082003F0E1FA00210820BDE86A
:10B70000044003F0DBBA3549884209D101211020F9
:10B7100003F0D4FA00211020BDE8044003F0CEBAB3
:10B720002F49884209D10121202003F0C7FA0021C6
:10B730002020BDE8044003F0C1BA2A49884209D15B
:10B740000121402003F0BAFA00214020BDE8044066
:10B7500003F0B4BA2449884209D10121802003F0C2
:10B76000ADFA00218020BDE8044003F0A7BA1F49CC
:10B7700088420BD101214FF4807003F09FFA002121
:10B780004FF48070BDE8044003F098BA184988422D
:10B790000BD101214FF4007003F090FA00214FF417
:10B7A0000070BDE8044003F089BA124988420BD109
:10B7B00001214FF4806003F081FA00214FF4806092
:10B7C000BDE8044003F07ABA01BD00000000024069
:10B7D0000004024000080240000C02400010024039
:10B7E0000014024000180240001C024000200240E9
:10B7F0000024024000280240F0B4002232E001237D
:10B8000093400C681C409C422BD154000325A5405A
:10B81000ED4306682E40066006680F79A7403E4358
:10B8200006600E79012E01D0022E11D186682E40BD
:10B83000866086684F79A7403E438660466826EA60
:10B840000303436043688E799640B6B23343436046
:10B85000C3682B40C360C368CD7905FA04F4234361
:10B86000C360521C102ACAD3F0BC70470022006982
:10B87000084200D00122104670470183704741837F
:10B88000704710B4CB1000EB830001F00701890072
:10B89000036A0F248C40A3430362036A02FA01F196
:10B8A0001943016210BC70470168490849000160F2
:10B8B0000021016041608160C1600161212141611D
:10B8C0009D49884203D13D209C49086070479C49AE
:10B8D000884204D14FF474609849086070479949D0
:10B8E000884204D14FF47410944908607047964917
:10B8F000884204D14FF074609049086070479349C2
:10B90000884203D192488D494860704791498842E6
:10B9100003D191488949486070479049884203D1D2
:10B920008F488649486070478E49884204D14FF05D
:10B930003D508249486070478B49884203D13D2081
:10B940008A49086070478A49884204D14FF474607C
:10B950008649086070478749884204D14FF47410C3
:10B960008249086070478449884204D14FF074606E
:10B970007E49086070478149884203D174487B49F9
:10B98000486070477E49884203D1734877494860D0
:10B9900070477C49884203D17148744948607047B8
:10B9A0007949884203D14FF03D5070494860704753
:10B9B0000268764B1A400B681A43CB681A434B69EE
:10B9C0001A438B691A43CB691A430B6A1A434B6AB1
:10B9D0001A438B6A1A434B6B1A438B6B1A430260F0
:10B9E0004269D208CB6A53EAC2020B6B1A43426126
:10B9F0000A6942604A6882608968C16070470021B4
:10BA0000016041608160C160016141618161C1612A
:10BA1000016241628162C162016341638163704777
:10BA20000029016803D041F0010101607047490815
:10BA30004900016070470029016803D041F480216A
:10BA40000160704721F4802101607047002A01D015
:10BA500001617047C1607047006800F001007047E5
:10BA60000022414B984201D2494800E049488B00EE
:10BA700001D5406800E0006808404749084200D00E
:10BA8000012210467047384A904201D2404800E0F7
:10BA90004048414A0A40890001D5C260704782602F
:10BAA00070470B0609D5002A436903D043F0800391
:10BAB000436102E023F08003436180290AD001F052
:10BAC0001E01002A026802D011430160704722EA79
:10BAD00001010160704710B40022234B984201D24B
:10BAE0002B4B00E02B4B2D4C214205D0006800EA87
:10BAF000D12000F01E0002E0406900F080008C00C0
:10BB000001D55B6800E01B681940234B194202D045
:10BB1000002800D00122104610BC7047124A904203
:10BB200001D21B4800E01B481B4A0A40890001D58E
:10BB3000C260704782607047106002400860024037
:10BB4000286002404060024058600240706002403D
:10BB50003D00002088600240400F0020A0600240AD
:10BB600000003D20B86002401064024008640240BA
:10BB700028640240406402405864024070640240FD
:10BB800088640240A0640240B86402403F801CF018
:10BB900000600240006402407D0F7D0F3C0F3C0FAF
:10BBA00010B504001F480078002802D0A120FBF740
:10BBB00041FCFBF75EFF1C480078401C1A490870E6
:10BBC000802080F3118800BF00BF1748806880691B
:10BBD000204209D114488068C46113488068082154
:10BBE00001741148FBF77FFC0F48806884690E4898
:10BBF0008068002181610C480078401E0A49087065
:10BC000009484078F021084202D09920FBF712FC45
:10BC100005484078002802D1002080F311882000D8
:10BC200010BD00BFFB710020501F002038B504007C
:10BC30000D0016480078401C14490870144800781C
:10BC4000002802D0A120FBF7F5FBFBF712FFA07E36
:10BC5000662802D08220FBF7EDFB802080F311885C
:10BC600000BF00BF08E04021200001F08FF98020D4
:10BC700080F3118800BF00BFE0680028F3D02900DE
:10BC8000200001F0D2F9FBF735FF31BD501F002035
:10BC9000FB7100202DE9F04104000D0016001F008B
:10BCA000802080F3118800BF00BF2248D0F80080B8
:10BCB00006E0A04502D1AC20FBF7BCFBD8F804801D
:10BCC000B8F1000FF5D11C484078F021084202D0AD
:10BCD0009920FBF7AFFB18484078002802D10020DC
:10BCE00080F31188FBF79DFE1C220021200001F04B
:10BCF00043F9A760266125836620A076802080F323
:10BD0000118800BF00BF0B480068606009480460EC
:10BD100009484078F021084202D09920FBF78AFBBD
:10BD200005484078002802D1002080F31188BDE842
:10BD3000F0810000D8710020501F00202DE9F84349
:10BD400004000E0017001D00DDF828802E48007842
:10BD5000002802D1A520FBF76DFBFBF78AFE2B48DC
:10BD6000D0F80C9006E0A14502D1AA20FBF762FBB7
:10BD7000D9F80090B9F1000FF5D15422002120002C
:10BD800001F0FAF8642084F850006761207C2049B3
:10BD900009780843207484F84580002E00D066623C
:10BDA000089EE662099FA7623A00CD21300001F0AB
:10BDB000E3F8BE19F608F600503E002030605FF050
:10BDC0008070706413483064F5647FF00200706224
:10BDD0001148F06211483063114870631148706077
:10BDE0001148B0601148F06011483061114870612D
:10BDF0001148B0611148F06111483062666020005E
:10BE0000FBF715FFBDE8F183FC710020501F0020F7
:10BE1000F8710020B37400080100CCCC0200CCCC37
:10BE20000300CCCC0400CCCC0500CCCC0600CCCCA0
:10BE30000700CCCC0800CCCC0900CCCC0A00CCCC80
:10BE40000B00CCCC80B53B4988420BD101214FF48B
:10BE5000805002F049FF00214FF48050BDE80440BB
:10BE600002F042BF344988420BD101214FF4804097
:10BE700002F02FFF00214FF48040BDE8044002F0A3
:10BE800028BF2E4988420BD101214FF4004002F017
:10BE900020FF00214FF40040BDE8044002F019BF2C
:10BEA000274988420BD101214FF4005002F01CFFBA
:10BEB00000214FF40050BDE8044002F015BF2149B5
:10BEC00088420BD101214FF4801002F00DFF0021B8
:10BED0004FF48010BDE8044002F006BF1A498842C2
:10BEE0000BD101214FF4001002F0FEFE00214FF4AF
:10BEF0000010BDE8044002F0F7BE01BD028802F464
:10BF000041520B881A434B881A438B881A43CB88BB
:10BF10001A430B891A434B891A438B891A43CB89DD
:10BF20001A430280828B4FF2FF731A408283098A80
:10BF3000018270470030014000380040003C004062
:10BF400000340140005001400054014000290188A4
:10BF500003D041F04001018070474FF6BF7211409D
:10BF600001807047002A828802D011438180704787
:10BF700022EA01018180704700220089084200D036
:10BF800001221046704700002DE9F04FA1B0824613
:10BF9000002017461D4602910B900DF1440B6FF0E7
:10BFA00000490AE017F8011B0298D04702900028C8
:10BFB00000F0A8820B98401C0B90387808B90B98B9
:10BFC000A2E22528EED10020059006900790089067
:10BFD00009900A9001E040F0010017F8011F2029A4
:10BFE000F9D023290DD02B2904D02D2906D03029B2
:10BFF0000AD00CE040F0020080B2EEE740F004000E
:10C00000FAE740F00800F7E740F01000F4E72A29CB
:10C010000ED12968296051F8042B2960002A0D925D
:10C0200004D5514240F004000D9180B27F1C11E014
:10C0300000210D9109E00D99494505D001EB8103DF
:10C0400002EB430130390D917F1C3A78A2F13001A7
:10C050000A29F0D339782E2903D04FF0FF310C9103
:10C060001DE017F8011F2A2907D1296829607F1CC4
:10C0700051F8042B29600C9211E000210C9109E089
:10C080000C99494505D001EB810302EB430130399E
:10C090000C917F1C3A78A2F130010A29F0D3ADF857
:10C0A00038000FF67440397802F084FE08B117F8B2
:10C0B000010B8DF83A009DF83A00682802BF3978E4
:10C0C0006829622005D06C2804BF38786C2803D119
:10C0D00071208DF83A007F1C11A8049017F8014BCD
:10C0E000B4F125002AD01C3800F0CC80001F0228B3
:10C0F00040F2C880133800F0EE80093800F0C280AA
:10C10000801E00F04F81401E00F02481401E022856
:10C1100040F2B880001F00F01D81401F00F08380B6
:10C12000401E00F0D880401E29D0C01E0CD0801EBA
:10C1300000F0D180C01E00F0CE803DE101200590CE
:10C1400025208DF8440043E12868286050F8044B0E
:10C1500028600394DDF83080B8F1000F04D5204644
:10C16000FBF74CF9804607E042460021204602F0EA
:10C170002DFE08B1A0EB0408CDF8188028E129684D
:10C1800029604FF03C0851F8040B29600021CDE9EB
:10C19000000111A80390DDE90001049C11B908B960
:10C1A0000C9AC2B10206120FA0EB02123032D2B2C8
:10C1B0003A2AA8BF27320009A8F1010340EA01701A
:10C1C00009091A5508BF0028984604D0039A08EBBD
:10C1D00004039A42E6D308EB04000390C8F13C0143
:10C1E0000C980691814209DA401A08904FF6EF71D7
:10C1F000BDF838000840ADF83800E9E0002840F10B
:10C20000E7809DF8380000F01400102840F0E0802E
:10C210000D98059A801A089A801A401A0128C0F2CF
:10C22000D7800890D4E09DF83A0062281AD0682898
:10C2300006D06A280CD06C281CD0712808D019E0D0
:10C240002868286050F8041B28600B980880BFE01D
:10C250002868286050F8042B28600B98C117C2E9A1
:10C260000001B5E02868286050F8041B28600B988E
:10C270000870ADE02868286050F8041B28600B980F
:10C280000860A5E02868C01D20F007022A60D2E9F6
:10C29000000108322A60CDE90001002903D5012000
:10C2A00005902D200CE0BDF83800810703D5012052
:10C2B00005902B2004E0C00704D501200590202024
:10C2C0008DF84400059911A808180390214600A88C
:10C2D00000F0D8F97CE09DF83A206C2A0DD0712A44
:10C2E00018BF6A2A09D12868C01D20F007032B60F7
:10C2F000D3E9000108332B6005E02968296051F873
:10C30000040B29600021CDE90001682A08BF80B232
:10C3100007D0622A08BFC0B203D0742A18BF7A2A95
:10C3200002D10021CDE900019DF83800000730D589
:10C33000DDE90001002908BF00282AD044F02000D0
:10C34000782826D130208DF844008BF80140022057
:10C3500005901EE09DF83A00294600F0D8F8CDE996
:10C360000001002904DA0598411C05912D210EE0F9
:10C37000BDF83800810704D50598411C05912B2193
:10C3800005E0C00705D50598411C0591202100F85E
:10C390000B10059911A808180390214600A800F079
:10C3A000EDF815E0012005902868286050F8041B7E
:10C3B00028608DF844100BE0012005902520002C0A
:10C3C0008DF8440004D00598411C059100F80B40FD
:10C3D0000D980599401A0899401A0699401A09992A
:10C3E000401A0799401A0A99A0EB01089DF83800F5
:10C3F00040070FD420208DF84000002408E00123DE
:10C4000010AA00A9504600F070FC00287AD1641CE4
:10C410004445F4DB059C11AE0AE016F8011B0298B6
:10C42000D047029000286DD00B98401C0B90641EE2
:10C43000002CF2D130208DF840000026089C08E046
:10C44000012310AA00A9504600F04FFC002859D142
:10C45000761CA642F4DB069C039E0AE016F8011B3C
:10C460000298D047029000284CD00B98401C0B90AB
:10C47000641E002CF2D130208DF840000026099C6B
:10C4800007E0012310AA00A9504600F02EFCC8BB0B
:10C49000761CA642F5DB03980699079C0E1809E066
:10C4A00016F8011B0298D047029058B30B98401C15
:10C4B0000B90641E002CF3D130208DF84000002634
:10C4C0000A9C07E0012310AA00A9504600F00DFCC9
:10C4D000C0B9761CA642F5DB9DF8380040077FF511
:10C4E0006CAD20208DF84000002400E0641C444521
:10C4F000BFF663AD012310AA00A9504600F0F5FB7A
:10C500000028F3D04FF0FF3021B0BDE8F08F622853
:10C5100026D068281DD06A2808D06C2827D071281A
:10C5200004D0742823D07A280CD020E00868C01DDD
:10C5300020F007000860D0E90023083008601946A1
:10C54000104670470A680A6052F8040B0A6000211E
:10C5500070470A680A6052F8040B0A6000B20BE0E8
:10C560000A680A6052F8040B0A6040B204E00A68E4
:10C570000A6052F8040B0A60C11770472DE9FA4EA1
:10C5800005460A462F696F2A08BF082405D041F0E6
:10C590002000782814BF0A2410243C26D5E9000185
:10C5A000642A18BF692A81468A4605D1002903DA20
:10C5B000D9F100096AEB4A0ABAF1000F08BFB9F1D4
:10C5C000000F0CD1286B50B9082C36D195F83800E3
:10C5D000000732D530203B2687F83B002DE0E317DB
:10C5E000484651462246FDF741FEA4FB0023A9EB35
:10C5F00002023032D2B2A6F1010B3A2A5E4603DBC8
:10C600009DF80030513B9A1881465FEA010A0BF809
:10C61000072008BFB9F1000F03D0E868F11988427C
:10C62000DDD3082C09D195F83800000705D5F05D59
:10C63000302802D0761E3020F055C6F13C00A861AB
:10C64000F119E960296B884208DA081A28624FF666
:10C65000EF71288F08402887BDE8F38E00290ED59A
:10C6600095F8381001F01401102908D1696B6A6936
:10C67000891A2A6A891A081A0128A8BF2862BDE8FF
:10C68000F38E00002DE9F24F04468EB0D4E900018C
:10C69000CDE9020104AF9DF8380040F0200BBBF15A
:10C6A000610F0AD0206B002848BF062004D408BFC1
:10C6B000BBF1670F01D1012020636168C1F30A500B
:10C6C00040F2FF7290421CD1080304BF206800288A
:10C6D00009D10320A0619DF8380061381A2836D3AB
:10C6E0000FF2486108E00320A0619DF8380061382E
:10C6F0001A2829D30FF22C61E0680322F5F79CFE7B
:10C70000BEE1012816DA204602F08CFB012811DB7D
:10C7100000250020BBF1610F20D1E168302201F833
:10C72000012B4A1CE2609DF83820612A0CBF782258
:10C7300058220FE0626840F2FE3161F31E52451A42
:10C7400062604FF0FF30E5E70FF2D451D4E70FF20B
:10C75000D851D1E70A706169891C616110B900265E
:10C76000002584E1BBF1610F40F09780206B002829
:10C770004CBF2126461CDDE90201D4E900AB0022B2
:10C780000023F8F72DFF36B23ABF8BF00040CDE919
:10C7900002A0CDE902AB06F101082D1F8DF8102093
:10C7A0000DF1110700E0C71DB8F1010F33DBDDE922
:10C7B000020100220023F9F7B9F82CD21C2102A8AB
:10C7C00002F052FBDDE90201F8F7DEFEA8F10708EE
:10C7D000B8F1010F814609DBF8F7BEFE02460B46B1
:10C7E000DDE90201FBF780FECDE90201F81D07211A
:10C7F00005E009F00F0200F8012D4FEA2919B9F1FF
:10C80000010F01DB491EF4D5491E5CBF002200F870
:10C81000012DF9D5C7E70DF11100391AB142B8BFA2
:10C820000E4636B230000DF111072FD4884206DAD9
:10C8300004A9411849780829A8BF0F2100DA00216E
:10C8400004AA821800E0761E12F80139401E8B42BD
:10C85000F9D00F2904D104A941184A78521C4A7012
:10C86000002802D504AF761C2D1D36B2701E0DD4E3
:10C87000C1190A783032D2B23A2A03DB9DF8383037
:10C880003A3B9A18401E01F80129F2D5206B002886
:10C8900040F1ED80701E2063E9E0DDE90201002235
:10C8A0000023F8F79DFE3CBF81F00041CDE9020175
:10C8B0002DB247F2975068434B49DFF8309190FB17
:10C8C000F1F52DB2C5F1070ABAF1010F90461CDB54
:10C8D000DDE902675FEACA7007D542464B4630463B
:10C8E0003946F8F795FE06460F464FEA6A0A404673
:10C8F000494642464B46F8F78BFEBAF1000F804698
:10C900008946E7D1CDE9026724E0CAF1000A002692
:10C91000374F14E05FEACA7007D542464B463046AF
:10C920003946F8F775FE06460F464FEA6A0A404652
:10C93000494642464B46F8F76BFE80468946BAF1B7
:10C94000000FE7D1DDE9020132463B4601F0E2FD8E
:10C95000CDE90201BBF1660F216BDFF898900CBFA7
:10C9600005F10A0006204618142EA8BF1326302011
:10C970008DF810000DF11107012E3DDBDDE90201FC
:10C98000F8F718FE07F1080104220A23B0FBF3F3BD
:10C9900003EB8307A0EB4700303001F8010D0A20BC
:10C9A000B3FBF0F000EB8007A3EB47033033521EDC
:10C9B00001F8013DE9D1083E012E01F10807DBDB5A
:10C9C000DDE90201F8F7F6FDF8F7D0FD02460B4667
:10C9D000DDE90201FBF788FD00224B46F8F718FE5F
:10C9E000CDE90201CAE700BFA08601000000244093
:10C9F0000000F03F84D797410DF11100381A0DF176
:10CA0000110702E0401E6D1E7F1C39783029F9D0D5
:10CA1000BBF1660F02D12DB2691C04E0BBF1650FBA
:10CA20000CBF01210021226B8E1836B2B042B8BF74
:10CA3000064636B231001AD4814204DAC85D352880
:10CA4000A8BF392000DA3020CA19521E00E0761E35
:10CA500012F80139491E8342F9D0392802D1C85D44
:10CA6000401CC855002902D57F1E761C6D1C2DB2B6
:10CA70009DF83810009533B23A46204600F003F88E
:10CA80000FB0BDE8F08F2DE9F043054685B01E4696
:10CA9000D5F83080012E8946174602DA01260FF2BA
:10CAA000902749F02000BDF93040662808BF641C7B
:10CAB00017D0672840F0828014F1040FC0F2848000
:10CAC000444580F2818095F83800641C000702D448
:10CAD0004645B8BFB04624B2B8EB040848BF4FF093
:10CAE000000824B2E868A969012C25DA4A1C302321
:10CAF0000B54B8F1010F03DA95F83810090702D585
:10CB00002E211154521C18EB040FB8BFC8F10004B9
:10CB100024B26142A044B045AA61B8BF46466962EA
:10CB200036B2EE613246AB6939461818F5F784FC27
:10CB3000A8EB0600A862C1E00818A64218DA32463F
:10CB40003946F5F779FCA9697118A01BA961B8F1FC
:10CB5000010F686203DA95F83800000705D5EA6826
:10CB60002E208854E869401CE861C5F82880A5E0BB
:10CB700022463946F5F760FCA8692018361BB8F143
:10CB8000010F03DA95F83810090703D5EA682E215A
:10CB90008154401CA86136B2B045B8BF4646E8682B
:10CBA000AB6936B23246E1191818F5F745FCA869A9
:10CBB0003018A861A8EB060068627FE0B9F1610F48
:10CBC00016D14FF0700918E0464504DA95F8381090
:10CBD000090758BFB046B8F1010848BF4FF0000838
:10CBE000B9F1670F14BF4FF045094FF0650904E034
:10CBF000B9F1410F08BF4FF05009A969E86817F86B
:10CC0000013B0B544A1CB8F1010F05DA95F83810B6
:10CC1000090758BFAA6117D52E211154531CB8F12A
:10CC2000010FAB6110DB761E36B2B045B8BF464689
:10CC300036B2324639461818F5F7FEFBA8693018A7
:10CC4000A861A8EB06006862E868A9690F182000CF
:10CC500007F8019B03D42B2007F8010B03E02D21DB
:10CC600007F8011B644200260DF1080808E00A22BB
:10CC700000A802F085F9019808F8010B761C009CC9
:10CC800021B20129F3DA022E06DA49F020006528E4
:10CC900004BF302007F8010B4EB9302007F8010B14
:10CCA00007E0761E02A8305C303007F8010B012E39
:10CCB000F7DAE868A9690818381AE86195F83800C1
:10CCC00000F0140010280DD16869A9690818696A74
:10CCD0000818E9690818A96A0818696B8842BCBF76
:10CCE000081A286205B0BDE8F083F8B504460D4681
:10CCF00016461F46002004E0E86A401CE8627F1EDA
:10CD0000002047B116F8011BA868A047A8600028BA
:10CD1000F2D14FF0FF30F2BD686A6C747A4C0000BB
:10CD20006E616E004E414E00696E6600494E4600CF
:10CD3000300000000CB41CB5044604A801900A465B
:10CD4000009401AB00A9074878441830FFF71CF99C
:10CD5000009A0021117000285CBF0098001B16BCCF
:10CD60005DF80CFB6B57FFFF0901002806D55C4AF4
:10CD700000F00F00801800F8041C7047594A8154D5
:10CD8000704710B5401EB0F1807F01D3012010BD67
:10CD9000554C60600F214FF0FF30FFF7E5FF00209A
:10CDA000A06007202060002010BD50480068704738
:10CDB0004F48006800F08060704738B54D4D2878C6
:10CDC000401C28704C4C2078401C2070FAF776FEEE
:10CDD00002F0DEF8FAF7A4FB2878411E297000283B
:10CDE00002D19820FAF726FB2078012804D1606848
:10CDF000002801D0FAF78AFB2078401E2070BDE899
:10CE00003140FAF787BB30B585B000A80FF20011AA
:10CE10001422F5F721FB394D28680090364C6078D4
:10CE2000F021084202D09920FAF704FBFAF778FBC8
:10CE30006078401C607002F03FF928684FF47A7106
:10CE4000B0FBF1F0FFF79DFF002800D0FEE72C4873
:10CE50002C4908600E214FF0FF30FFF785FF28684E
:10CE6000009000A802F09CF92748016841F0404179
:10CE700001606078F021084202D09920FAF7DAFACE
:10CE80006078401E6070C0B2002801D1FAF742FB02
:10CE900005B030BD80B501E0FBF7F6FA1B484168EC
:10CEA0000029FBD100680028F6D1FBF7EBFAF5E783
:10CEB00010B41148006A114909684FF47A72B1FB45
:10CEC000F2F10A4A1368CB1A094C2468640102D5AE
:10CED00012688B1A401C00FB013010BC7047000028
:10CEE00018ED00E000E400E010E000E018E000E0F1
:10CEF00004ED00E0F9710020501F002040250020C3
:10CF00000000000808ED00E034EF00E0A47100200C
:10CF100000000000E803000000000000ABCD0008A6
:10CF2000B1CD0008EFF30580002842F05B81704727
:10CF300080B5EFF3108072B60B49096851F47F0198
:10CF4000094A116080F310880848006810F4700FD7
:10CF500002D1A720FAF76EFA05485FF00071016070
:10CF600004480021016001BD20ED00E088ED00E0F3
:10CF70003CEF00E034EF00E010B5040010000A00C0
:10CF800001002000F5F7A8FA200010BD00B585B01B
:10CF9000029001900E4A92680392802282F31188D7
:10CFA00000BF00BF0268009200AA0260009800283B
:10CFB00002D0009800AA42600548806800AA8260FA
:10CFC000034880680174FAF775FE05B000BD00BF24
:10CFD000501F002038B5028BC3684469E318046908
:10CFE000A34201D304691B1B534384680D781D556C
:10CFF000491C5B1C521E002AF7D1C168491CC16044
:10D00000012902D101F030F90EE027484078F021E3
:10D01000084202D09920FAF70DFA234840780028F8
:10D0200002D1002080F3118831BD10B50400208B9F
:10D0300062694243A368D35C0B70521C491C401EBA
:10D040000028F7D16069401C60612169884201D3E2
:10D0500000206061E068411EE1602169884212D1D0
:10D0600011484078F021084202D09920FAF7E2F9FD
:10D070000D484078002802D1002080F3118820005C
:10D0800001F0F2F80EE008484078F021084202D0A2
:10D090009920FAF7CFF904484078002802D10020FF
:10D0A00080F3118810BD0000501F002009010028E6
:10D0B00007D5DFF8302B00F00F00801800F8041CB3
:10D0C0007047DFF8842C8154704710B5401EB0F1D2
:10D0D000807F01D3012010BDDFF8704C60600F210C
:10D0E0004FF0FF30FFF7E2FF0020A0600720206034
:10D0F000002010BDDFF8582C002803D04021104636
:10D10000FEF7BBBB40211046FEF7B9BBDFF8402C51
:10D1100000284FF48051104601D0FEF7AEBBFEF759
:10D12000AEBB1CB5DFF82C4C2046FEF7B7FA012148
:10D13000084601F0A2FD01208DF8040000208DF8C2
:10D140000500ADF806004FF4807120460183C0460B
:10D150004FF48070009000A92046FEF74DFB4FF47D
:10D1600080710020FBF792F913BDF0B583B0DFF8B2
:10D17000E04B2046FEF792FADFF8DC5B2846FEF72C
:10D180008DFADFF8D86B3046FEF788FA01210846A1
:10D1900001F073FD0121022001F06FFD0121042047
:10D1A00001F06BFD0121802001F067FD03208DF867
:10D1B000040001208DF8060000208DF807008DF88E
:10D1C000050049F6FF600090DFF8887B00A938462B
:10D1D000FEF712FB4FF6FF70009000A92046FEF705
:10D1E0000BFB00A92846FEF707FB00A93046FEF717
:10D1F00003FB0021012001F040FD0021022001F08D
:10D200003CFD0021042001F038FD0021802001F0C8
:10D2100034FD0121032001F030FD01208DF80400D0
:10D2200000208DF80500ADF806000121022001F074
:10D2300024FD402120460183C0464020009000A9E3
:10D240002046FEF7D9FA4FF4805120460183C046AC
:10D250004FF48055009500A92046FEF7CDFA2946E7
:10D2600038464183C046009500A93846FEF7C4FA07
:10D2700004220A212046FEF704FB0922032120464E
:10D28000FEF7FFFA02208DF8040001208DF805005A
:10D290008DF8060000208DF807004FF480600090A4
:10D2A00000A92046FEF7A8FA0820009000A9204611
:10D2B000FEF7A2FA042208212046FEF7E2FA042231
:10D2C00007212046FEF7DDFA02208DF80400012038
:10D2D0008DF805008DF8060000208DF807004FF44A
:10D2E0008070009000A92046FEF786FA802000900A
:10D2F00000A92046FEF780FAF7BD30B585B0DFF80B
:10D30000401C884235D0DFF83C1C88422FD14FF4B6
:10D3100080050C460121284601F0BAFC01210220BB
:10D3200001F0ABFC0121284601F0D3FC0021284686
:10D3300001F0CFFC0020ADF804004BF6FF70ADF813
:10D3400006004FF48060ADF80A004FF48040ADF85D
:10D350000C000A20ADF80800DFF8AC0C009000A922
:10D36000204601F088FF0121204601F0E7FF05B0CB
:10D3700030BD4FF400150C46CCE72DE9F04192B0DA
:10D3800001214FF4805001F08EFC0121032001F0B7
:10D3900074FC01214FF4800001F06FFCDFF8B44908
:10D3A000052211462046FEF76CFADFF8A459052243
:10D3B00011462846FEF765FA052204212846FEF7A5
:10D3C00060FA05220F212046FEF75BFA02208DF855
:10D3D000040001208DF805000020ADF80600202093
:10D3E000009000A92046FEF707FA2020009000A92F
:10D3F0002846FEF701FA1020009000A92846FEF703
:10D40000FBF94FF40040009000A92046FEF7F4F924
:10D41000DFF8F84B2046FEF715FDDFF8F45B00203F
:10D42000288068600120288100206881E86007204A
:10D43000288200206880DFF8DC6B3046FEF734FA83
:10D44000DFF8D47B3846FEF72FFA4FF48060069061
:10D4500000210D9103210E9100210F910A91089056
:10D46000DFF83C0C039008461090099007904FF4A9
:10D4700000300C9008460B904FF0C068CDF8088043
:10D48000402005900846049002A93046FEF790FA25
:10D4900000200B90CDF80880059005F11400049051
:10D4A00002A93846FEF784FA002068802946204603
:10D4B000FEF724FD012202212046FEF753FD012242
:10D4C00011462046FEF74EFD01212046FEF73EFDA7
:10D4D00000213046FEF7A4FA00213846FEF7A0FAF4
:10D4E00012B0BDE8F08130B589B001214FF0805015
:10D4F00001F0CEFB012001F053FC01214FF480200C
:10D5000001F0BBFB0F20FCF7ABFD04461020FCF73D
:10D51000A7FD0546012001F0ADFB002001F0AAFBAC
:10D5200021460F20FCF78FFD29461020FCF78BFDCC
:10D5300000214FF4802001F0A0FB042001F024FB27
:10D54000412001F0E7FB0028FAD04FF4807001F091
:10D550007BFB012001F018FB012001F088FBFCF7A8
:10D5600018FC0120069043F6FF70079000200590FC
:10D5700005A8FCF7C5FB0020029002A9FCF72AFCD5
:10D5800000208DF8070001208DF804008DF80500BB
:10D590008DF8060001A90020FCF799FC4FF48000EB
:10D5A00001F0B4FA4FF48000039000208DF81000D1
:10D5B00008208DF8110001208DF8120003A801F059
:10D5C00067FA03208DF800000D208DF8010000207F
:10D5D0008DF8020001208DF8030000A801F015FF6E
:10D5E0000320FCF7E9FC4FF48040FCF782FD4FF488
:10D5F000800001F08BFA01214FF48040FCF73DFDE3
:10D60000012009B030BD1FB50121084601F035FBEE
:10D6100001214FF4804001F046FB00208DF80C0002
:10D620008DF80F0001200290DFF8A04A02A92046E1
:10D63000FEF7E2F80420029002A92046FEF7DCF88B
:10D640000820029002A92046FEF7D6F800210846DD
:10D6500001F014FF0221002001F010FF032100203F
:10D6600001F00CFF00208DF8040001208DF8060069
:10D6700000900C208DF8050000A801F009FA0420A4
:10D6800000900C208DF8050000A801F001FA082098
:10D6900000908DF8050000A801F0FAF9012001F0D2
:10D6A00035FA042001F032FA082001F02FFA1FBDEC
:10D6B00000B585B00121084601F0DFFA01214FF4E1
:10D6C000804001F0F0FA00208DF810008DF8130072
:10D6D0000820039003A9DFF8F409FEF78DF8032171
:10D6E000002001F0CBFE00208DF8080001208DF80D
:10D6F0000A00082001908DF8090001A801F0C8F97E
:10D70000082001F003FA09208DF800000E208DF8A2
:10D71000010000208DF8020001208DF8030000A810
:10D7200001F073FE05B000BD00B585B001210846CB
:10D7300001F0A3FA01214FF4804001F0B4FA002077
:10D740008DF810008DF813000420039003A9DFF872
:10D750007C09FEF751F80221002001F08FFE002025
:10D760008DF8080001208DF80A00042001900C209B
:10D770008DF8090001A801F08BF9042001F0C6F929
:10D7800008208DF800000E208DF8010000208DF893
:10D79000020001208DF8030000A801F036FE05B05C
:10D7A00000BD38B5DFF828492078401C2070DFF82C
:10D7B00024592878401C2870FAF780F96878F021FD
:10D7C000084202D09920F9F735FEF9F7A9FE6878EA
:10D7D000401C687000F0B8FB6878F021084202D065
:10D7E0009920F9F727FE6878401E6870C0B20028BB
:10D7F00001D1F9F78FFE4FF48040FCF763FC00285D
:10D8000014D04FF48040FCF774FC4FF4800001F01A
:10D810007DF9F8F753FA009000A9DFF8BC0801F091
:10D820007DF9DFF8B8180420F8F7ECFAF9F778FE7C
:10D830002078411E2170002802D19820F9F7FAFDC6
:10D840002878012804D16868002801D0F9F75EFE25
:10D850002878401E2870F9F75DFE31BDDFF880089A
:10D860000068704738B50446012C38DB012001F010
:10D8700097FA0020FCF7BFFB4FF400550420FCF79B
:10D8800017FC012804D12846451E80B20028F5D196
:10D8900000EE104AB8EEC00ADFEDB50A80EE800A4D
:10D8A000F0EE000A20EE200ADFEDC20A80EE800AC8
:10D8B000BDEEC00A10EE100A401E80B2FCF78CFBD1
:10D8C0004FF48040FCF715FC4FF4800001F01EF986
:10D8D0000120FCF790FBDFF80808046031BD002050
:10D8E000DFF8FC170860012001F05AFA0020BDE8BB
:10D8F0003240FCF780BB000070B501240023DFF844
:10D90000E4171A468A608A6812F00C0FFBD1DFF820
:10D91000D82705460C2D4BD8DFE805F01D4A4A4AAA
:10D9200007181D2C31363B4045008D6845F08005B9
:10D930008D604FF4C065DFF8B46735600D6825F081
:10D9400080750D60DFF8A857156032E02346DFF8D8
:10D95000A45715602DE08D688D604FF4C065DFF829
:10D960008C6735600D6825F080750D60DFF888578D
:10D9700015601EE00223DFF88457156019E00323C9
:10D98000DFF87C57156014E00423DFF87857156042
:10D990000FE00523DFF8705715600AE00623DFF873
:10D9A0006C57156005E00723DFF86457156000E049
:10D9B0001C46002B4AD00FF6680503EBC3035B1926
:10D9C0008D688D600D6825F080750D600D6825F0FF
:10D9D00080650D609D781E8845EA8615DE7876089C
:10D9E000761E45EA06451E7945EA06654D60DD88E6
:10D9F0001E7A360746EA8515DFF8186735600D6828
:10DA000045F080750D600D68AD01FCD55B7943F480
:10DA1000C063DFF8D8562B608B688B608B688B6097
:10DA2000052804D1886840F09000886005E00B2844
:10DA300003D1886840F480508860886840F0020014
:10DA40008860886800F00C000828FAD11068DFF8B8
:10DA5000C816884207D2DFF8C406016821F44041A5
:10DA600041F48041016010684FF47A71B0FBF1F02D
:10DA7000FFF72BFB204670BD3EE7002800E0401E6C
:10DA8000FDD17047F0B583B00727DFF8B4148842A2
:10DA900003D14FF48074802502E04FF480640825A0
:10DAA00001208DF804008DF805008DF80600002097
:10DAB0008DF807000094DFF8686600A93046FDF78E
:10DAC0009BFE009500A93046FDF796FE21463046A4
:10DAD0004183C0460F20FFF7D0FF21463046018327
:10DAE000C0460F20FFF7C9FF3846471E80B2002806
:10DAF000ECD1009500A93046FDF77EFE2146304668
:10DB00004183C0460520FFF7B8FF29463046018310
:10DB1000C0460520FFF7B1FF214630460183C046CD
:10DB20000A20FFF7AAFF214630464183C046052060
:10DB3000FFF7A3FF294630464183C0460520FFF783
:10DB40009CFF02208DF8040001208DF805008DF85F
:10DB5000060000208DF80700009400A93046FDF76C
:10DB60004BFE009500A93046FDF746FEF7BD0000CC
:10DB700000007A4438B50024DFF8A8550121286850
:10DB800001F015FC286801F047FB2868FFF7B5FB9A
:10DB900005E02868FFF776FF2868FFF7AEFB4FF433
:10DBA0000031286801F00EFC002802D0641C032C10
:10DBB000EFDB31BD0000004730B40022838A008BC8
:10DBC000DFF86045656843EA00400840000255EA16
:10DBD000102060600840884200D10122104630BC0D
:10DBE0007047000018ED00E02DE9F84F04460D469F
:10DBF00016464FF080091F78DFF828854FF4003172
:10DC0000D8F8000001F0DEFB002808D04846A0F15B
:10DC100001090028F2D1FFF7ADFF00203EE0D8F85F
:10DC2000000001884FF6FF52114001800121D8F811
:10DC3000000001F08FFB4FF4007AD1460020C8F8B5
:10DC40000400D8F800B0DFF8E0145846FFF7B4FF3E
:10DC5000002806D14846A0F101090028F1D1002092
:10DC60001CE0D14600222146584601F08BFB0020E3
:10DC7000C8F80400D8F80040DFF8B0142046FFF7D9
:10DC80009BFF00280CD14846A0F101090028F1D1E2
:10DC90000121D8F8000001F069FB0020BDE8F28FF7
:10DCA0003146C9B220460182C046D1460020C8F89C
:10DCB0000400D8F80040DFF878142046FFF77CFF16
:10DCC000002805D14846A0F101090028F1D1DFE77D
:10DCD000012F15D1297820460182C046D146002067
:10DCE000C8F80400DFF84C14D8F80000FFF764FF10
:10DCF000002822D14846A0F101090028F2D1C7E747
:10DD00003846471EC0B2002817D015F8011BD8F8B6
:10DD100000000182C046D1460020C8F80400DFF8A8
:10DD20001414D8F80000FFF747FF0028E8D1484650
:10DD3000A0F101090028F2D1AAE70121D8F80000DA
:10DD400001F014FB0120A9E700E400E010E000E08E
:10DD5000000402400000024000080240001C024093
:10DD60002DE9F54F81B00D461E464FF080083778FB
:10DD7000DFF8B0434FF40031206801F023FB0028A6
:10DD800008D04046A0F101080028F3D1FFF7F2FEC9
:10DD9000002039E0206801884FF6FF5211400180D1
:10DDA0000121206801F0D6FA4FF40079C84600201E
:10DDB0006060DFF874A3D4F800B051465846FFF70E
:10DDC000FBFE002805D14046A0F101080028F2D151
:10DDD0006EE000229DF80410584601F0D3FAC846C0
:10DDE00000206060D4F800B0D0495846FFF7E4FE48
:10DDF00000280BD14046A0F101080028F2D10121F2
:10DE0000206801F0B3FA0020BDE8FE8FBDF80810CD
:10DE1000C9B258460182C046C846C749206801F0C9
:10DE2000D1FA002805D14046A0F101080028F4D11C
:10DE3000E5E70121206801F08DFAC8460020606006
:10DE4000D4F800B051465846FFF7B6FE002805D179
:10DE50004046A0F101080028F2D129E001229DF8F6
:10DE60000410584601F08EFA022FC84638DAB3493A
:10DE7000206801F0A7FA002805D14046A0F101086A
:10DE80000028F4D1BBE70021206801F084FA206863
:10DE9000018B012101F06AFAC846A949206801F006
:10DEA00091FA002806D14046A0F101080028F4D1DB
:10DEB0000020A9E72068008AC0B228703078401E90
:10DEC0003070C84620680188890505D54046A0F114
:10DED00001080028F6D192E7012101F05CFA29E05F
:10DEE0000020606097492068FFF766FE002805D192
:10DEF0004046A0F101080028F4D180E7012616E091
:10DF0000012F0CD1012E0AD100263146206801F0E4
:10DF100042FA2068818A018B012101F027FA2068EA
:10DF2000818A490603D5008A05F8010B7F1EFFB2DE
:10DF3000002FE5D10121206801F02DFA012063E7CF
:10DF400000540040005800407F48016808292FD144
:10DF500064490A6842F080720A604268B2F1806FD8
:10DF600003D10A6842F080620A600A689201FCD517
:10DF70008A6842F002028A608A6802F00C02082A6B
:10DF8000FAD14268B2F1806F02D10A681201FCD561
:10DF900055490968604A914206D260490A6822F4EC
:10DFA000404242F480420A600021016041607047B3
:10DFB0004168B1F1806F09D14A490A6842F0806234
:10DFC0000A600A681201FCD50021416070475F4871
:10DFD000016841F08051016050480168890889005A
:10DFE00041F0010101600FF23500594908607047A6
:10DFF0005848016821F00401016030BF016841F018
:10E00000040101607047000070F30500003001401A
:10E01000006F0020586402401064024010B5FAF707
:10E02000C3F9807A002803D0012000F0BCFE02E092
:10E03000002000F0B8FE474C80214748FDF79CFFC8
:10E0400000281FD172B627483F49826802F00C02AF
:10E050000A60006800F080604860206840F00400BA
:10E060002060FBF7C3FFB0F5704F02D90220FBF729
:10E07000B3FF30BF62B6206820F004002060BDE826
:10E08000104061E7206820F00400206030BF206865
:10E0900040F00400206010BD2D48006800470000DB
:10E0A0000C3001400949401E05280DD8DFE800F07A
:10E0B000030507090C0B1A4906E0284904E0284922
:10E0C00002E0284900E02849084670470000024065
:10E0D000F9710020501F0020F42E0020303700205E
:10E0E000BC7100200038024040250020003C024066
:10E0F00000127A00809698000024F40000366E0129
:10E100000048E801005A6202006CDC0280F0FA026A
:10E1100000BD0105843802400190D003007000402A
:10E1200000040240C0250020010003008200070017
:10E1300080000700840007000400001002000010A7
:10E1400040000010020003008471002040380240AB
:10E15000C071002010ED00E00030014000080240D6
:10E16000000C024000100240001C024010B50C469A
:10E17000FFF798FF214689B2BDE81040FDF77DBB4F
:10E1800010B50C46FFF78EFF214689B2BDE810405E
:10E19000FDF775BBE0B5002A03D10C228DF80920EC
:10E1A00002E008228DF8092000281CD0012802D0A6
:10E1B000032821D007BD0120019010208DF809000F
:10E1C00006208DF800000E208DF8010000208DF84B
:10E1D00008008DF80200002917D001208DF80A00F0
:10E1E0008DF8030015E00420019008208DF8000050
:10E1F0000E208DF80100E9E70820019009208DF834
:10E2000000000E208DF80100E0E78DF80A008DF87F
:10E21000030001A800F03CFC00A801F0F6F807BDDF
:10E22000200110040F03020103F00010060F010289
:10E230000103C00010080F01020103C00010060F07
:10E2400001020103F00010060F0102010360000843
:10E25000040F02020103C80010040F02020103A808
:10E260000010020F0302010310B5040003E0206850
:10E27000C068F9F77FFC802080F3118800BF00BFE1
:10E2800020680028F3D108484078F021084202D0E5
:10E290009920F9F7CFF804484078002802D10020EF
:10E2A00080F3118810BD00BF501F0020012001F035
:10E2B000F9B800000749086808B10020704706480F
:10E2C000C008C00008600549C908C900091A0160F2
:10E2D000704700BFEC7100204F0800204818002054
:10E2E000012804DB421E531002EB937205E010F18B
:10E2F000030F04DA421000EB9272921000E0002249
:10E3000010F0030F00D110B90FF2441001E00FF22A
:10E31000281030F91100801870472DE9F84F044695
:10E3200042484018154600901CB9414801F0C4F815
:10E33000044625624FF461650098DFF8F8A00FF2FB
:10E3400010160FF2F4076FF0020840F26D1902E0A8
:10E35000009800F561605146B0FBF1F14B1C4FF0A5
:10E36000070C93FBFCFCCCEBCC0CA3EB0C03A361E4
:10E370004B4691FBF3F300E05B1E012B05DB5A1EBD
:10E380004FEA620E02EB9E7204E0434505DA5A1032
:10E3900003EB92724FEAA20C01E04FF0000C13F075
:10E3A000030F02D10BB1BE4600E0B646BEF9002015
:10E3B000944409FB03CC6145DEDBA1EB0C026361F5
:10E3C00013F0030FE26100D10BB9334600E03B4686
:10E3D0004FF00C0C03F1180E3EF902BD5A45ACF19A
:10E3E000010CF9DBC4F810C00AFB110033F91C3032
:10E3F000D21A521C2946E260B0FBF1F1A16005FB84
:10E4000011003C21B0FBF1F1C1EB01126160A0EB06
:10E4100082002060206A002805D5204601F05AF8C5
:10E420000128206294DA2046BDE8F28F807EAA831C
:10E430000C0000208051010000001F003C005B0028
:10E4400079009800B600D500F400120131014F01A7
:10E4500000001F003B005A0078009700B500D40070
:10E46000F300110130014E01F0B5244E83B0304667
:10E4700001F022F80446224D284601F01DF80068FC
:10E4800008B901F0C1F8284601F016F80546301D1C
:10E4900001F012F8064628682168814228D00078E9
:10E4A00010B901F0C7F82860286800AA022101F01D
:10E4B000C6F8074600230A2201A901F0E1F83060FE
:10E4C0000199009AC91B914205D100F2135040F600
:10E4D0002721884201D3002030606421306890FBFE
:10E4E000F1F101EB8102C0EBC200306028682060CE
:10E4F0003068A0EB0011880003B0F0BD04000020DC
:10E500003C000020704700001FB500F059FA21219F
:10E5100001601FBDF0B540F2FF7581EA030C0CF0FD
:10E52000004C15EA11541DBF15EA1357AC42AF4217
:10E53000E5E0BC41C1F31301C3F31303801A994111
:10E5400043F4801304D2641E4000494180185941AD
:10E55000C90241EA5051B1FBF3F603FB1611A2FBCD
:10E560000675D7EBC020A94102D2761E801859410A
:10E57000C90241EA5051B1FBF3FE03FB1E11A2FB9D
:10E580000E75D7EBC020A94103D2AEF1010E801861
:10E590005941890241EA9051760546EA8E2EB1FB37
:10E5A000F3F603FB1611A2FB0675D7EB8020A941F9
:10E5B00002D2761E80185941C90241EA50514EEAF2
:10E5C000060EB1FBF3F603FB1611A2FB0675D7EBA3
:10E5D000C020A94102D2761E80185941C90241EAE1
:10E5E0005051B1FBF3F703FB1711A2FB0735D3EB37
:10E5F000C020A94167F100070CBF004247F00107A6
:10E6000066F3D5274FEA1E31B80814F5806412DD91
:10E61000BD0775F1004250EB0E5051EB045111F55E
:10E62000801F5CBF41EA0C01F0BD4CF07F6141F0FE
:10E63000E0410020F0BDBD076D0840EA0E5041F4F6
:10E640008011D4F10104B4F120060ADAC4F12006E5
:10E650000200E04001FA06F3E1401843B2401543DE
:10E660000EE0342C13DCC6F1200445EA40056D08A9
:10E6700020FA06F2154321FA06F0A1400D430021CD
:10E6800075F1004250F1000051EB0C01F0BD00208B
:10E690005FEA0C01F0BDCFB992185B41B3FA83F782
:10E6A00004BFB2FA82F6BF190B3FB7F120062FBFA5
:10E6B00002FA06F3BB40C7F1200622FA06F638BF7D
:10E6C0003343BA401CB1E419641E33E77F4231F092
:10E6D0000041B1FA81F404BFB0FA80F6A4190B3CF2
:10E6E000B4F120062FBF00FA06F1A140C4F12006C4
:10E6F00020FA06F638BF3143A0403C1B1AE7AC4273
:10E700001ABF05EA1357AF4212E050EA41061CBF98
:10E7100052EA4306BFE750EA4107304661461CBF54
:10E7200041EA0551F0BD52EA430C08BFC143F0BDB8
:10E7300000204FF4001616EB410F98BF16EB430F65
:10E7400008BF16EB410F24BFC14305E016EB430F92
:10E750000CBF61464CEA0551F0BD000080B51A4877
:10E7600000688047002801D0012002BD002002BDC2
:10E7700080B5154949688847002801D0012002BDAD
:10E78000002002BD0020704780B50F49C968884746
:10E79000002801D1012002BD002002BD00207047E9
:10E7A000002070470949C1611C2101700521417099
:10E7B000002181700121C17000210182418281828A
:10E7C000C1828161084670475C24002074240020C7
:10E7D000D0B51446544A554BF7F7A8F82DED048BE5
:10E7E00041EC180B1DD89FED529B53EC182B51ECAC
:10E7F000190BF6F70DFF00224F4BF6F7DBFF06462D
:10E800000F4653EC182B51EC190BF6F7D3FF0246C9
:10E810000B4630463946FFF77DFE41EC180B44F0BD
:10E82000010451EC180B0022444BF6F7D9FE05D336
:10E8300001224FF07953F7F779F851D853EC182BA0
:10E84000F6F7E6FE41EC190B53EC182BF6F7E0FE59
:10E8500006460F4653EC192B39483A49F6F7D8FECD
:10E86000394A3A4BF6F7A6FF53EC192BF6F7D0FED0
:10E87000374A384BF6F79EFF32463B46F6F7C8FE5E
:10E8800053EC182BF6F796FF06460F4653EC192B60
:10E8900031483249F6F7BCFE314A324BF6F78AFF6F
:10E8A00053EC192BF6F7B4FE2F4A304BF6F782FFE4
:10E8B00053EC192BF6F7ACFE2D4A2E4BF6F77AFFE8
:10E8C00053EC192BF6F7A4FE2B4B0022F6F772FF40
:10E8D00002460B4630463946FFF71CFE41EC180B4A
:10E8E000A00705D551EC180B81F0004141EC180B45
:10E8F00014F007020BD00FF2880303EBC20251ECB5
:10E90000180B53681268F6F755FF41EC180B2007F7
:10E9100005D551EC180B81F0004141EC180B51EC7E
:10E92000180BBDEC048BD0BD57CD9E5E1426D13F95
:10E93000AA4C58E87AB6FB3F0000F0BF000040BE8A
:10E94000845D57134B57B03FB2934C19ED5EE43FD3
:10E95000BEDE02B90240F83FDE39028FC7C0743F05
:10E960008AAB1283000CC83F24D7E508B6D8F03F25
:10E970000F34580E5895FD3F0000F03F0000000096
:10E98000000000000000000066732D3852C1E03F17
:10E99000182D4454FB21F93F66732D3852C1F03FC6
:10E9A000182D4454FB21F93F66732D3852C10040A5
:10E9B000182D4454FB2109403FD038C6A6F104402D
:10E9C000014800F079BD00000000002010EE101A90
:10E9D00004204FF07E5C01EE90CA49004FEA5101DD
:10E9E00000EE101A88BF0820B1F17E5F13D871EED7
:10E9F000C00ADFF838C031EE801A61EE200AF1EE6D
:10EA0000E00A614586BF80F0040080EE800A80EE57
:10EA1000200A00F079BE490011F1807F9CBF6FF0A1
:10EA2000004100EE101A7FF66FAD7047F404353FD9
:10EA300010EE101A4FF07E5C01EE90CAC80F31F054
:10EA4000004122D000EE101AB1F17E5F13D871EEB2
:10EA5000C00ADFF838C031EE801A61EE200AF1EE0C
:10EA6000E00A614586BF80F0040080EE800A80EEF7
:10EA7000200A00F049BE490011F1807F9CBF6FF071
:10EA8000004100EE101A7FF63FAD7047F404353FA9
:10EA900030B40168CB431F498279002A27D00A4647
:10EAA00014682340136053680468A34353600379D8
:10EAB000CC18236805682B43236093680468A3433C
:10EAC0009360D3680468A343D36043790568102B2F
:10EAD00007D1916829439160D16800680843D060EC
:10EAE0000AE051FA83F420682843206004E00079AA
:10EAF0000C1820681840206030BC70470021064A7E
:10EB00001268024200D0012108467047024908609D
:10EB100070470000003C0140143C014070B5040007
:10EB20000D000126A07E662802D08220F8F782FC24
:10EB3000F8F777FF13480078401C124908708020CE
:10EB400080F3118800BF00BFE0682169884204D2C9
:10EB500029002000FEF73EFA00260A484078F021FE
:10EB6000084202D09920F8F765FC06484078002852
:10EB700002D1002080F31188F8F7BCFF3000C0B24A
:10EB800070BD00BF501F0020DFF8C81100220A70BE
:10EB90000A70012802D0042803D0704701200870B1
:10EBA0007047052008707047DFF8AC1108607047A7
:10EBB00030B46A494A6802F00C02042A02D0082ADA
:10EBC00003D022E0674A026021E00A68C2F3805263
:10EBD0000B6803F03F03002A07D0624AB2FBF3F24E
:10EBE0000B68C3F388135A4306E05F4AB2FBF3F2A3
:10EBF0000B68C3F388135A430B68C3F301435B1CD0
:10EC00005B00B2FBF3F2026001E0574A02604A681F
:10EC100002F0F003554A1B099B5C05682C46DC405A
:10EC200044604B6803F4E0539B0A9B5C2546DD403F
:10EC30008560496801F46041490B895C426813466C
:10EC4000CB40C36030BC7047454900F44072B2F518
:10EC5000407F06D10A6822F4F812454B03401A435C
:10EC60000A608A6E000552EA105088667047414972
:10EC700008607047404908607047404A00291168A1
:10EC800002D008431060704721EA0000106070470E
:10EC90003B4A0029116802D008431060704721EAFE
:10ECA000000010607047374A0029116802D00843FD
:10ECB0001060704721EA000010607047324A002956
:10ECC000116802D008431060704721EA000010600C
:10ECD00070472E4A0029116802D00843106070471F
:10ECE00021EA000010607047294A0029116802D00B
:10ECF00008431060704721EA000010607047254A01
:10ED00000029117802D008431070704721EA0000F2
:10ED10001070704741090E4A012901D1116804E0C1
:10ED2000022901D1116F00E0516F00F01F000A4667
:10ED3000C24002F0010070470021174A12680242E7
:10ED400000D0012108467047144908707047000040
:10ED50000038024070380240800E474204380240BA
:10ED60000838024040787D010024F400642500202A
:10ED7000FFFCFF0F3C0E4742400E47423038024036
:10ED800040380240443802401038024020380240E7
:10ED9000243802400D3802400C3802400E38024040
:10EDA00002490860704702490860704720000E421F
:10EDB00024000E420278C9B28A421AB11CBF10F870
:10EDC000012FF9E718BF002070470000C9B2830780
:10EDD00006D0521E22D310F8013B9942F7D11FE012
:10EDE000083A13D302F1040241EA012141EA014148
:10EDF00050F8043B121F21BF4B40A3F1013C2CEA09
:10EE0000030C1CF0803FF3D0C9B2001F083210F889
:10EE1000013B521E28BF91EA030FF8D818BF01200A
:10EE2000401E704730B4436803F0004201211B03C9
:10EE30001B0B436004BF0368002B08D10DE003687F
:10EE4000DD0F45EA440444605B000360491E4468EA
:10EE5000E302F4D523031B0B436043681A4342606B
:10EE6000084630BC7047000070B504460D46606827
:10EE7000C0F30A5040F2FF71884207D16068000376
:10EE800004BF2068002817D0022070BD20B920469A
:10EE9000FFF7C8FF012868DA012D0FDB40F2FF7190
:10EEA000091A8D420AD3606800284CBF9FED300BD1
:10EEB0009FED310B84ED000B012070BD4142A94252
:10EEC000616806DA6FF31E51401941EA0050606034
:10EED00042E0401E63684519012205F1350062F3E6
:10EEE0001F53352801F00041636003D361600020A7
:10EEF000206070BD002215F11F0F04DA2268236024
:10EF0000002020356060684214D0521E256892416E
:10EF1000C0F12003D2439D4045EAD272256825FA0C
:10EF200000F6656805FA03F333432360636823FA48
:10EF300000F5656060680843B2F1004F606003D877
:10EF40000DD12078C0070AD52068401C20602068B9
:10EF500028B96068401C60604FF0FF3070BD606889
:10EF6000884204BF20680028F6D1002070BD00BF91
:10EF7000000000000000F0FF000000000000F07F33
:10EF800091FBF2F303FB1211C0E90031704700005E
:10EF900010B522480078002802D1A220F8F74AFADA
:10EFA0001F48406B002807D01D48012180F8381009
:10EFB0001B480121417127E01948006A401C18498B
:10EFC00008621749D1E90A23521C53F1000314497E
:10EFD000C1E90A231249496A401A002802D410489C
:10EFE000012141710E4890F8300000280CD00C48E7
:10EFF00090F83000401E0A4981F83000C0B2002865
:10F0000002D10748012101710648046802E06068E6
:10F0100080472468002CFAD110BD00BFF971002090
:10F02000501F0020DC710020BFF34F8F494801685A
:10F0300001F4E061484A11430160BFF34F8F00BF04
:10F04000FDE710B5454C606C40F480406064444876
:10F05000016801F0070101290CD10168C908C90044
:10F060000160006800F00700012803D1FFF7DCFF12
:10F0700000BFFDE74FF4407000F0C2F93948016865
:10F0800041F470010160206840F001002060002020
:10F09000A0602068344908402060344860602068DF
:10F0A00020F4802020600020E06000F039F84FF06C
:10F0B00000602F49086010BD00212E48426802F010
:10F0C0000C02042A02D0082A04D01CE02A492B4A48
:10F0D00011611BE00268C2F38052036803F03F0332
:10F0E000002A06D12649B1FBF3F10268C2F3881267
:10F0F00051430268C2F30142521C5200B1FBF2F1CB
:10F100001E4A116102E01E491C4A11614068114605
:10F11000C0F30310405C0A691346C3400B6170479B
:10F120001448C16B41F08051C16316490A6822F44A
:10F13000404242F480420A60416841604168416057
:10F1400041684160082101604FF4C0600E490860C9
:10F15000704700000CED00E00400FA0500380240A2
:10F160000038014088ED00E0FFFFF6FE103000247B
:10F1700008ED00E00438024040787D013025002091
:10F180000024F40000700040003C024005E0B0FBA9
:10F19000F1F201FB1202080011000029F7D17047BB
:10F1A00038B501000E481422F3F756F90C480068F0
:10F1B0000B494968B0FBF1F0094948614FF47A7492
:10F1C0000748456929002000FFF7E0FFB4FBF0F194
:10F1D000034A9161B5FBF0F00149C86131BD0000FF
:10F1E000787000200021102806DB103800F1604103
:10F1F00011F56441097806E00E2801D1042007E0EA
:10F200000449001F415C802901DA022000E001204E
:10F21000704700BF18ED00E080B5434988420BD12C
:10F2200001214FF40010FFF754FD00214FF40010AE
:10F23000BDE80440FFF74DBD3C4988420BD1012198
:10F240004FF48000FFF745FD00214FF48000BDE83A
:10F250000440FFF73EBD364988420BD101214FF4EF
:10F260000000FFF736FD00214FF40000BDE8044028
:10F27000FFF72FBD01BD7FB504460D46A68800A847
:10F28000FFF796FC02992B48B1FBF0F04FF6C072E5
:10F2900032400243A28022884FF6FE731A40228039
:10F2A0002A68254B9A420AD25200B1FBF2F10A4673
:10F2B00092B2042A00DA0421401C208421E0EB8869
:10F2C0004BF6FF76B34204D102EB4202B1FBF2F1FE
:10F2D00006E019235A43B1FBF2F141F4804189B2AF
:10F2E0000A0502D141F0010189B241F4004180B226
:10F2F0004FF4967250434FF47A7290FBF2F0401C38
:10F300002084A183208840F00100208020884FF6CF
:10F31000F5310840A9880843698908432080A889F5
:10F320002989084320817FBD0054004000580040D7
:10F33000005C004040420F00A186010000290188C6
:10F3400003D041F00101018070474FF6FE72114079
:10F35000018070470029018803D041F48071018049
:10F3600070474FF6FF621140018070470029018805
:10F3700003D041F40071018070474FF6FF521140F5
:10F3800001807047002A02D041F0010101E001F044
:10F39000FE01018270470029018803D041F4806199
:10F3A000018070474FF6FF321140018070470029FD
:10F3B000018803D041F40041018070474904490CA1
:10F3C0000180704782B002460020034601930093FB
:10F3D00000920A0F01920902090A019A002A03D039
:10F3E000009A1432009203E0090C009A183200923D
:10F3F000009A12680A4200D0012002B07047000053
:10F4000019490843194908607047F0B403781A464F
:10F410000121C478002C1DD0144B1B6803F4E06359
:10F42000C3F5E0631B0A4478C3F10405AC4085785A
:10F430000F2637461F4107EA050323431B010C4CE7
:10F440001355007800F01F0291400A4A401142F81B
:10F45000201007E003F01F0001FA00F006495211E6
:10F4600041F82200F0BC70470000FA050CED00E006
:10F4700000E400E000E100E080E100E030B401F0F1
:10F480000302920021F00301054BCC580F25954053
:10F49000AC43CC50CC5890402043C85030BC70474F
:10F4A0000838014080B5C046C046024A1100182005
:10F4B000ABBEFBE72600020004490968002900D121
:10F4C0000349034A801A411808007047E071002080
:10F4D000000000202DE9F84304464748FFF7ECFF01
:10F4E00080464648FFF7E8FF454F05463846FFF798
:10F4F000E3FF006808B900F087F83846FFF7DCFF43
:10F5000006464048FFF7D8FFD8F80010074638688D
:10F51000814220D0007878B93068007810B900F0C6
:10F5200089F83060306800AA032100F088F838605C
:10F53000017809B1401E3860386800F04BF90600C8
:10F5400008BF4FF0FF3054D02868FAF74CF92E600E
:10F550003868C8F800004FF0000960690021FEF724
:10F56000BFFE8046E169A0682D6801EB410200EB17
:10F57000C207606940F26D1101FB0080401C072149
:10F5800090FBF1F1C1EBC101401A00F10E0600E061
:10F590006D1D2878FF282BD0606929798842F7DB18
:10F5A000E978FEF79DFEA978A0EB080008182978F5
:10F5B00071B13218521A072392FBF3F3C3EBC30362
:10F5C000D21A18BFC2F1070210180829B8BFC01F0D
:10F5D00000EB4001687800EBC100874208DB287926
:10F5E000697A88420CBF89F001094FF00009CFE722
:10F5F0004846BDE8F28300BF4400002038000020E8
:10F600003C0000204000002038B5084C2046FFF7A1
:10F6100053FF006848B90FF218052046FFF74CFF6A
:10F620000560201DFFF748FF056031BD3C0000204C
:10F63000000000000FF20400704700003A00F8B527
:10F6400004460D462078002816460CBF002714F803
:10F65000017B01E06D1E441C39462046FFF7AAFBE2
:10F6600018B92046F7F7CAFE0019012D03DA001B6E
:10F6700030602046F2BD01780029EBD13160F2BD47
:10F680002DE9F04182B080460E001D4608BF00AE55
:10F69000474600E07F1C3878A0F109010529F9D31D
:10F6A0002028F7D02D2816BF2B2817F8014B2B2424
:10F6B0003146384600F02CF931688F4208BFC6F851
:10F6C00000803168884514D120B92D2C16D1B0F1B5
:10F6D000004F15D9FFF774F9222101600DB1012007
:10F6E00028602D2C14BF6FF000404FF00040BDE8A3
:10F6F000F6812B2CE9D1B0F1004FEBD2BDE8F681B9
:10F700004042BDE8F68100001AA210EE101ADFF8A0
:10F7100060C0F2EC060A614509DB00EE803A70EE4B
:10F72000800A83EE200A40F0020010EE101A21F049
:10F73000004CDCF1665C0BD860EE000A20EE203A4B
:10F7400003EE010A01EEA02A42EE202A80EE220AF0
:10F75000400810F0020F18BFB1EE400A02EB800221
:10F76000D2ED000A30EE200A28BFB1EE400A704701
:10F77000A430893ED7B3DD3F6AD5033F2B94A93D22
:10F78000B82A593F0000803F000080BF0000000001
:10F79000920A063FDB0FC93F920A863FDB0FC93F43
:10F7A000920A0640DB0F4940368D274000220AE0CE
:10F7B0000378303B0A2B09D202EB820310F8012BAD
:10F7C00002EB4302303A491EF2D501E04FF0FF321E
:10F7D000104670472DE9F843054615F8018BB8F13E
:10F7E000000F00F092802846022601E0401C761CA3
:10F7F0004146FFF7DFFA0028F8D106EB8600F9F75B
:10F8000092FE060000F08180002734464FF0FF3959
:10F8100000E0641D287828280BD10421681CFFF71C
:10F82000C5FFA0F26C77002F6CD46879292869D1C4
:10F83000AD1D277102212846FFF7B8FF401EE0707A
:10F84000AD1C0220294600220AE00B78303B0A2B2F
:10F8500009D202EB820311F8012B02EB4302303A8A
:10F86000401EF2D500E04A46501EA07015F8021F57
:10F8700030390A2928BF002316D202212A46002344
:10F880000DE092F800C0ACF1300CBCF10A0F09D2C7
:10F8900003EB830C12F8013B03EB4C03303B491E96
:10F8A000EFD500E04B46AD1C6370E1780C29BFBF7B
:10F8B000C0B264286078642824DA28782B2818BF1E
:10F8C0002D2802D00020207010E06878A0F13001CF
:10F8D000072917D230280CBF07203038207028782D
:10F8E0002B2802D12078C01D2070AD1C287828B9A3
:10F8F000FF20607167723046BDE8F28315F8010B96
:10F90000404586D03046F9F76EFF0020BDE8F2830F
:10F910002DE9F04F85B004461E000D4690461CBFF1
:10F9200000203060A14601E009F1010999F80000CA
:10F93000A0F109010529F7D32028F5D02D2816BFFD
:10F940002B2819F8017B2B27B8F1000F57D4B8F1F9
:10F95000010F54D0B8F1250F51DAB8F1010F0DDBCA
:10F96000B8F1100F04BF99F80000302802BF99F8D1
:10F97000010040F02000782814D10EE099F8000032
:10F98000302818BF4FF00A080CD199F8010040F058
:10F990002000782804D14FF0100809F1020901E095
:10F9A0004FF00808CDF8109001E009F1010999F82D
:10F9B00000003028F9D00FF2A00B4FF0000ACDF86C
:10F9C0000C908DF808B00AE09DF80810CDF804A05E
:10F9D000401AC0B2009008FB0A0A09F1010999F81F
:10F9E0000010A1F141001A2838BF20314246584684
:10F9F000FFF7ECF90028E7D10498484503D105B199
:10FA00002C60002025E00FF27801039818F801100F
:10FA1000A9EB0000401A14D4012808DA0098BAEBC8
:10FA2000000004D30199B0FBF8F0884209D0FEF73A
:10FA3000C7FF222101600EB1012030604FF0FF3A74
:10FA400003E02D2F08BFCAF1000A0DB1C5F80090E0
:10FA5000504605B0BDE8F08F30313233343536379B
:10FA600038396162636465666768696A6B6C6D6E7C
:10FA70006F707172737475767778797A0000000010
:10FA800000002115110E0D0C0B0B0A0A09090909BA
:10FA900009080808080808080707070707070707ED
:10FAA0000707070707000000F0B583B004460D46BE
:10FAB00016461F460020ADF806008DF80400012010
:10FAC000009001AB2A467221204601F054F9010052
:10FAD00015D18DF806509DF80400B04338438DF8D9
:10FAE00004009DF804008DF8070002230DF10602C2
:10FAF0007221204601F0E1F8010000D10020FEBD96
:10FB000070B582B004460020ADF80000DFF8805DDB
:10FB10002878062818DB002600E0761C032E11D278
:10FB2000701900798DF800007019007A8DF80100C5
:10FB3000022300AA7221204601F0BFF80100ECD098
:10FB4000297076BD0020287076BD1CB504460020C3
:10FB5000ADF806008DF804002046012807D00428DF
:10FB600005D0102803D0402801D0802846D100239A
:10FB7000022280210520FFF797FF010047D10120D5
:10FB8000009001AB90227221052001F0F4F80100F1
:10FB90003DD19DF8040000F0FC008DF80400012C1C
:10FBA0000AD0042C04D0102C1ED0402C21D025E0EB
:10FBB00040F001008DF8040090208DF806009DF8BB
:10FBC00004008DF807009DF8040000F00300DFF842
:10FBD000C41C487002230DF106027221052001F0B9
:10FBE0006CF801000CD016BD40F002008DF8040046
:10FBF000E2E740F003008DF80400DDE7012016BDC8
:10FC000002231A4680210520FFF74EFF002016BD73
:10FC100010B582B00020ADF8000082208DF8000001
:10FC200000AC38206070022300AA7221082001F085
:10FC300044F801001FD18E208DF8000096206070DE
:10FC4000022300AA7221082001F037F8010012D126
:10FC50008F208DF8000008206070022300AA722116
:10FC600001F02BF8010006D108231A46D9211046CD
:10FC7000FFF71AFF002016BD38B50022ADF80020AE
:10FC8000DFF8104CA28A002902D01043A08202E0C3
:10FC900022EA0000A082A08A002805D002284BD0CA
:10FCA0001FD3032848D01AE0DD208DF8000000ADF6
:10FCB00000206870022300AA7221052000F0FDFFD9
:10FCC00001000DD180208DF8000000206870022313
:10FCD00000AA7221052000F0F0FF010000D10020F1
:10FCE00032BD81208DF8000000AD11206870022324
:10FCF00000AA7221052000F0E0FF0100F0D1687831
:10FD00002070DD208DF8000000206870022300AA1A
:10FD10007221052000F0D1FF0100E1D180208DF893
:10FD2000000003206870022300AA7221052000F061
:10FD3000C4FF0100D4D1D2E781208DF8000000ADCE
:10FD400011206870022300AA7221052000F0B5FF7F
:10FD50000100C5D168782070FFF75AFF0100BED0BE
:10FD600032BD2DE9FE4F82468B4616461C460027C3
:10FD7000B846DFF8205B0FF250106978085C2978EC
:10FD8000491C10FB01F240F6DC235A43029289021F
:10FD9000B1F5803F01D34FF6FF71C9000A22B1FBD4
:10FDA000F2F1102808D18C4206D34FF001084046EA
:10FDB000FFF7CBFE074619E0102808D1642C06DABD
:10FDC0004FF001084020FFF7C0FE07460EE0402834
:10FDD00002D164398C4203D2012807D1642C05DAA0
:10FDE0004FF001081020FFF7B0FE0746B8F1000FF2
:10FDF0000BD06A7839460FF63C30F4F74FFC002FF1
:10FE000001D101205EE038465CE0AA69D3172046A4
:10FE1000A0FB028900FB0399CDE90089E869C117BD
:10FE2000D046A8FB002308FB0133DDE90001801860
:10FE30005941CDE900012A6AD3175846A0FB02892F
:10FE400000FB0399DDE9000110EB080841EB09090B
:10FE5000686AC117A6FB002306FB013340464946EA
:10FE60008018594132461AFA8BF3D3181B1B03EB47
:10FE7000D3735B101BB2AAEB0306D41A002903DC70
:10FE800000DB01D200200146002E00D10126D5F86A
:10FE900028804FEAE879A8FB002308FB013309FB1F
:10FEA000003310461946029AD317FAF7BDF90C9998
:10FEB0000860E86A604390FBF6F0296B08180D991A
:10FEC00008600020BDE8FE8F0104104000B585B039
:10FED000DFF8C019CA6902600A6A42604A6A826031
:10FEE0008A69C2608A6A0261CA6A4261096B816179
:10FEF00003914169029101690191C1680091836890
:10FF0000426801680FF64420F4F7C8FB1C2005B0D6
:10FF100000BD00B585B01C2806D001460FF6502064
:10FF2000F4F7BCFB01201FE0DFF868090A68C26132
:10FF30004A6802628A684262CA6882610A698262A9
:10FF40004A69C2628A6902638869039048690290BB
:10FF500008690190C86800908B684A6809680FF6C4
:10FF60002C20F4F79BFB002005B000BD1CB5044617
:10FF700000208DF80400ADF806000120009001ABD0
:10FF800093227221082000F0F6FE002811D1932060
:10FF90008DF806009DF8040020438DF80700022329
:10FFA0000DF106027221082000F087FE010000D149
:10FFB000002016BD10B582B00020ADF800000FF68D
:10FFC000F010F4F76BFBDFF8D0080221C1720021BA
:10FFD00041730123072280210820FFF765FD0028D7
:10FFE00022D1DD208DF8000000AC082060700223D3
:10FFF00000AA722100F061FE010015D16023E02209
:020000021000EC
:10000000D9210820FFF750FD00280DD1D7208DF809
:10001000000001206070022300AA7221082000F075
:100020004CFE010000D1002016BD70B582B0002545
:100030002C462146ADF80010042801DB012076BDD6
:10004000002805D0022810D008D3032814D017E0C8
:10005000DFF8440801720478457811E0DFF83808C9
:10006000012101728478C5780AE0DFF82C080221AA
:1000700001720479457903E06424DFF81C084579AE
:10008000224629460FF64410F4F708FB88208DF825
:10009000000000AE7470022300AA7221082000F054
:1000A0000CFE01000CD18A208DF80000757002232F
:1000B00000AA7221082000F000FE010000D10020FB
:1000C00076BD00002DE9FC41044600200190064663
:1000D000DFF8C477787B002805D10FF60410F4F719
:1000E000DDFA0320C4E00120009001AB9C227221C4
:1000F000082000F040FE002840F0BA809DF80480FF
:1001000040466070387A042800F2AC80DFE800F0E6
:10011000030F2EAA400041460FF6D400F4F7BEFAB2
:100120000120FFF782FF010040F0A2807AE0F8781A
:1001300040450BDA41460FF6C800F4F7AFFA02204B
:10014000FFF773FF010040F093808BE0B8788045A3
:1001500080F2888041460FF6BC00F4F79FFA3046E3
:10016000FFF763FF010040F083800DE041460FF68A
:10017000B800F4F793FAFFF71DFF010078D130467D
:10018000FFF753FF010073D101260020207069E0C2
:1001900041460FF6A400F4F781FA0220009001AB6B
:1001A000C0227221082000F0E6FD002860D19DF8F1
:1001B00004309DF80520002A03D0184645422DB290
:1001C00000E01D4629460FF68400F4F767FAFB2D80
:1001D0002CDBC0208DF806000DF1060628462838D5
:1001E000707002230DF106027221082000F065FDF7
:1001F00001003DD171780FF67000F4F74FFAC1207D
:100200008DF806000020707002230DF106027221A5
:10021000082000F052FD01002AD10320FFF705FF5E
:10022000010025D10126304620701BE0F8784045BA
:1002300005DA0220FFF7F9FE010019D107E078780E
:10024000404507DA0120FFF7F0FE010010D1012040
:10025000207006E03046FFF7E8FE010008D1304686
:1002600020700126A5702DB22812E07086F00100E2
:10027000BDE8F68180B5042806D001460FF2FC7077
:10028000F4F70CFA012002BD0878002808D04A785B
:10029000002A05D08A78002A02D0CA78002A05D11F
:1002A0000FF2F470F4F7FAF9012002BDDFF8E82547
:1002B0005070487890708878D070C8781071C8787D
:1002C00000908B784A7809780FF2D870F4F7E6F945
:1002D000002002BD1CB504460020ADF80400022039
:1002E000009001ABC0227221082000F044FD0028DC
:1002F00001D0002016BD9DF8041001A84278002A04
:1003000000D049429DF8042022704378637022781F
:1003100009B20FF2A870F4F7C1F9022016BD70B54A
:1003200082B004465E25002600E040365E2E18DAD4
:10033000C6F15E00402801DB402000E080B2C0B280
:10034000009033193046A0F18002D2B27221082009
:1003500000F011FD0028E8D00FF27870F4F79EF954
:100360000025284676BD38B50C460125012806D063
:1003700001460FF27070F4F791F9002032BD284663
:100380000090134622787221082000F0F4FC002827
:1003900005D021780FF26C70F4F780F9002528461B
:1003A00032BD80B5022806D001460FF27C70F4F70A
:1003B00075F9012002BD02230A467221082000F0CF
:1003C0007CFC010000D1002002BD00B583B00121FA
:1003D000009101AB9222722100F0CDFC01000AD104
:1003E0009DF80410E42905D00FF25C70F4F756F97B
:1003F00001200EBD00200EBD38B50020ADF8000074
:100400000520FFF77DFB40B2014601292CDADFF819
:10041000844440F29D30A062DFF88004E06140F245
:100420004C402062DFF8780460624FF47A70A0617B
:1004300040F6C150E06240F62F002063002500E046
:100440006D1C052D12D2281900798DF8000028198D
:10045000007B8DF80100022300AA7221052000F024
:100460002CFC40B20100EBD0C0B232BD002032BD46
:1004700080B50520FFF7A9FF4020FFF766FBDFF8F6
:100480001404002181700321C17001210846FFF787
:10049000F3FB40B2010001D0C0B202BD002002BD9A
:1004A00080B500210120FFF7E7FB40B2010001D039
:1004B000C0B202BD002002BD2DE9F04389B0044660
:1004C00007A800210A4606C00846059006900820A5
:1004D000009007AB94227221052000F04CFC00280C
:1004E00053D19DF81C00A07307A84178E17381786F
:1004F0002172C17861720179A1724079E0729DF830
:10050000220020739DF823006073DFF88853287859
:10051000207468786074607A217A41EA0026E07A73
:10052000A17A41EA0027607B217B41EA0028E07B39
:10053000A17B41EA002906A8019005A800904B463E
:10054000424639463046FFF70CFC01001DD10598A4
:100550002060069860600120A870E878002813D019
:100560000120049005980390687802902878019003
:10057000CDF8009043463A4631460FF2EC50F4F77E
:100580008DF8E878401EE870002009B0BDE8F083DF
:1005900030B404460D4611461A4600201C2C06D0E5
:1005A0001D2C07D0222C08D1104630BC8EE41046FA
:1005B00030BCB4E6284630BCD5E630BC704780B5C8
:1005C0000B4611461D2805D0222806D11846FFF7F4
:1005D000A0FC02E01846FFF7E4FE002002BD10B5C3
:1005E00082B00020ADF8000004460820FFF788FA2A
:1005F000010015D100E0641C032C10D2A948215C35
:100600008DF80010201800798DF80100022300AA4F
:100610007221082000F051FB0100ECD016BD002033
:1006200016BD38B50020ADF800009B4C04202072A8
:10063000002060738C208DF8000000AD30206870C1
:10064000022300AA7221082000F037FB01002BD101
:100650000120207301460220FFF70EFB010023D189
:1006600088208DF80000FF206870022300AA722104
:10067000082000F022FB010016D18A208DF800002E
:1006800000206870022300AA7221082000F015FBE8
:10069000010009D1FFF78EFC010005D12020FFF7F2
:1006A00065FC010000D1002032BD10B588B003A860
:1006B00000210A4606C00FF2E8410CC90CC0002414
:1006C000754821460173407B002822D100E0641C5C
:1006D000062C0CDA0120009003A8231805A8225C40
:1006E0007221082000F047FB0028F0D01DE003A88D
:1006F0009DF8111002919DF8101001919DF80F10B6
:100700000091837842789DF80C100FF29C40F3F72B
:10071000C5FF00210220FFF7AFFA010005D120201C
:10072000FFF724FC010000D1002008B010BDFEB589
:10073000044600200190ADF8080006460546012059
:10074000009001AB93227221082000F014FB0028D6
:1007500040F09D80012000900DF10503DC22722104
:10076000082000F008FB002840F09180FF20FFF7F0
:10077000FDFB010040F08B80474F9DF804004007CF
:100780000CD5387B002809D00FF25C40F3F786FFC8
:10079000FFF710FC01007AD10120FEBD9DF8040096
:1007A000000747D5387B002844D001231A46DC21B6
:1007B0000820FFF779F9002869D106231A4680211D
:1007C0000820FFF771F9010061D1DD208DF80800E4
:1007D00024208DF80900022302AA7221082000F0CB
:1007E0006CFA010053D19DF805100FF21040F3F799
:1007F00055FF0FF22040F3F751FF012078730220DC
:1008000000900DF10603C0227221082000F0B3FA17
:1008100000283CD19DF806109DF80720002A00D042
:1008200049429DF8063009B20FF22020F3F736FF57
:100830000120FEBD9DF80400800609D50126204652
:10084000FFF740FC002803D1387B002800D0354654
:100850009DF80400C021084200D00126002E09D1D5
:100860003869411C39619DF804200FF2C430F3F758
:1008700015FF01E00020386138691E2805D30FF20A
:10088000C830F3F70BFF0020386185F00100FEBD92
:100890009C250020C82000201C250020C2FCFFFF52
:1008A00064FBFFFFC82500201CB504460020ADF8FE
:1008B00004000220009001ABC0227221082000F049
:1008C0005AFA00280DD10120009001AB9C22722120
:1008D000082000F050FA002803D19DF80400207091
:1008E000002016BD30B404460D4611461A460020BD
:1008F0001C2C06D01D2C07D0212C08D1104630BC52
:10090000E8E4104630BC0AE5284630BC2BE530BC94
:10091000704780B50B4611461D2805D01E2806D10C
:100920001846FFF7A7FC02E01846FFF73AFD002043
:1009300002BD0000233E206761696E206368616725
:100940006E6564282564292025640000233E6C2000
:1009500067657420434F4546202564202564202583
:10096000642025642025642025642025640000007F
:10097000233E6C20636F6566206C656E677468202B
:100980006572726F7228256429000000233E6C2076
:1009900073657420434F4546202564202564202537
:1009A000642025642025642025642025640000003F
:1009B000233E702063616C6962726174696F6E209E
:1009C000537461727420212121000000233E7020A5
:1009D0004849202564204C4F572025642000000002
:1009E000233E7020647572696E672063616C00003D
:1009F000233E7020444554454354202564000000A4
:100A0000233E70204445544543545F48494748209D
:100A100025640000233E702044482052454C454147
:100A20005345202564000000233E702052454C456C
:100A30004153452025640000233E70204E4F4E4513
:100A40005F4D4F444520256400000000233E702088
:100A50006F666673657420256420307825782C20B5
:100A60003078257800000000233E702057726974AA
:100A700065206F666673657420256400233E7020D0
:100A8000746864206C656E677468206572726F723A
:100A90002825642900000000233E7020746864202B
:100AA0003D203000233E70207468736574202575E6
:100AB000202575202575202575000000233E702017
:100AC0006F66667365742025642030782578203041
:100AD00078257800233E2064756D70206661696C0E
:100AE00065640000233E2067657420726567207688
:100AF000616C206C656E677468206572726F722815
:100B000025642900233E206765742072656720767E
:100B1000616C206661696C65642861646472203070
:100B20007825782900000000233E20736574207228
:100B300065672076616C206C656E677468206572ED
:100B4000726F722825642900746D64333732352042
:100B50006465766963652069642028307825782982
:100B6000206661696C656400233E723D25642067E0
:100B70003D256420623D256420633D256420617429
:100B8000696D653D256420616761696E3D2564205E
:100B90006C75783D25752072656164793D2564002A
:100BA00080888A93D7DD0000233E72454E41424C37
:100BB000453D2564207250494C543D2564207250B7
:100BC0004948543D256420725354415455533D25A2
:100BD00064207243414C49423D25642072494E5481
:100BE000454E41423D256400233E7020726561649C
:100BF0002053545F5A494E5400000000233E702099
:100C00007243414C494253544154203D2030782591
:100C100078000000233E702043616C696272617449
:100C2000696F6E2046696E69736865642000000014
:100C3000233E20696E7620696E74202564207374CB
:100C40006174757320257800233E20726573657486
:100C500052510000052803D0082801D01D2803D1D7
:100C60007848794908607047784877490860704744
:100C700010B50446F7F798FBD0E94423104619460F
:100C8000224600F001F900F0010011F0000101D14D
:100C900000280DD06E4C2068401C20601E2807D311
:100CA0000FF2B810F3F7FAFCFCF764FF00202060A5
:100CB00010BD00206649086070472DE9F8430546DD
:100CC0000E4617464FF00208624C6078F021084249
:100CD00002D09920F6F7AEFBF6F722FC6078401CB4
:100CE00060709DF80000401E8DF8000017F9019B10
:100CF000284640B2FFF7AEFF00AB4A4692B23946F3
:100D00003046FCF771FF002812D06078F0210842CD
:100D100002D09920F6F78EFB6078401E6070C0B25A
:100D2000002801D1F6F7F6FBFFF7C3FF002020E013
:100D30004FFA88F8424629460FF23410F3F7AEFC1A
:100D40004046A0F101080028D6D16078F021084281
:100D500002D09920F6F76EFB6078401E6070C0B23A
:100D6000002801D1F6F7D6FB284640B2FFF780FFF6
:100D70000120BDE8F2832DE9F04704460D461646F2
:100D80001F46DFF8D480089888F80000DFF8C49088
:100D900099F80100F021084202D09920F6F74AFBA9
:100DA000F6F7BEFB99F80100401C89F801002046C7
:100DB00040B2FFF74FFF4FF0020A43463246394632
:100DC0002846FCF7CDFF002815D099F80100F02146
:100DD000084202D09920F6F72DFB99F80100401E39
:100DE00089F80100C0B2002801D1F6F793FBFFF7A4
:100DF00060FF002023E04FFA8AFA524621460FF2A4
:100E00007C00F3F74BFC5046A0F1010A0028D4D136
:100E100099F80100F021084202D09920F6F70AFB68
:100E200099F80100401E89F80100C0B2002801D1E4
:100E3000F6F770FB204640B2FFF71AFF0120BDE82D
:100E4000F087000000540040C025002000580040FA
:100E5000B8710020501F0020F5710020233E496E1C
:100E60006974696C61697A65204932430000000049
:100E7000495745202564202564000000495245203B
:100E80002564202564000000D2B2203A22BF21FA56
:100E900002F0002170472032D141D04048409140BB
:100EA000D14048407047000080B500920B46024692
:100EB000D6210120FFF75FFF02BD70B5A0B0064646
:100EC0000D46144600A88021F1F7FEFA204680283E
:100ED00001DB012012E08DF80060002105E04A5D91
:100EE00000ABCB185A70491CC9B28142F7DB631CB6
:100EF000DBB200AAD6210120FFF7DFFE20B070BDD3
:100F000080B500920B460246D6210420FFF733FF3E
:100F100002BD70B5A0B006460D46144600A880215B
:100F2000F1F7D2FA2046802801DB012012E08DF88B
:100F30000060002105E04A5D00ABCB185A70491CE7
:100F4000C9B28142F7DB631CDBB200AAD6210420C0
:100F5000FFF7B3FE20B070BD70B582B004460D46F9
:100F600016460020ADF80000012200A92046FFF738
:100F7000C7FF00280BD19DF80000A84330438DF82F
:100F8000010001220DF101012046FFF7C2FF76BDED
:100F900080B5DFF8B00A4178807840EA0102FE218E
:100FA0001120FFF7D9FF401E8041C043C00F00D180
:100FB000002002BD80B5DFF8901A0A78521C0A7032
:100FC00080B2F7F727FABDE80140F6F793BD38B5D0
:100FD0000420F2F74AFF006A00283FD0C0684FF4AF
:100FE000C871002804D04FF47A7191FBF0F109B276
:100FF00000254800DFF84C4A00E06D1C082D05DA9A
:1010000004EB4502B2F920209042F6DA082D00D117
:1010100007252819007C6178884220D06070FFF78E
:10102000B7FF00281AD1607810281ED020281CD0C5
:1010300030281AD060281BD0702819D0802817D0EB
:101040000220207394F90C2004EB4500B0F9201025
:101050000FF64830BDE83840F3F720BB31BD0FF63E
:101060002C30BDE83240F3F719BB01202073E9E7CB
:1010700008202073E6E780B500208DF8000080226C
:1010800011460920FFF768FF00283FD15C208DF84A
:1010900000000246FE211120FFF75EFF002835D137
:1010A000002240211220FFF757FF00282ED1832075
:1010B0008DF80000012200A90620FFF72AFF002872
:1010C00024D1012207210846FFF746FF00281DD141
:1010D00008208DF80000012200A9FFF71AFF002860
:1010E00014D100208DF80000012200A90920FFF78B
:1010F00010FF00280AD129208DF80000012200A944
:101100000A20FFF706FF002800D1002002BD2DE9CC
:10111000F04788B005460E4604A8002101600F463E
:1011200002A80A4606C000A806C005A80B460EC0C5
:10113000FFF7A1FF8146B9F1000F05D00FF674202B
:10114000F3F7ACFA484608E1C820FFF733FF4FF445
:101150004070F4F703FC04000FD10220FDE00127EA
:101160000020059005A84FF0000CC0F804C0C0F89E
:1011700008C0ADF800E04A808B80002207210A20D9
:10118000FFF7EAFE8146B9F1000F04D00FF62C20DC
:10119000F3F784FADBE06420FFF70CFF012207215C
:1011A0000A20FFF7D9FE8146B9F1000F04D00FF6EF
:1011B0001420F3F773FACAE06420FFF7FBFE4FF444
:1011C000C0786420FFF7F6FE042204A93A20FFF756
:1011D00097FE002810D19DF81100000602D54FF0AF
:1011E000000812E0A8F101080FFA88F8B8F1000F22
:1011F000E7D14FF00109AAE00FF6D010F3F74EFA4D
:101200004FF00109A3E008F10108B8F5C07F0EDA3C
:10121000022204EB48013E20FFF772FE8146B9F13D
:10122000000FF0D00FF6AC10F3F738FA8FE0002083
:101230003060804602A901E008F10308B8F5C07FDC
:101240003BDA3068401C306034F81800ADF8080014
:1012500004EB4800B0F90290A1F80290B0F904A0A4
:10126000A1F804A00598BDF9082000FA82F00590C5
:1012700005A8426802FA89F24260826802FA8AF29C
:101280008260002000E0401C0328D5DA02AA32F96F
:101290001020002A00D55242B2F50F6FF3DD0FF691
:1012A0003C10F3F7FBF9BDF808002880A5F8029080
:1012B000A5F804A04FF0010949E04FF0000805A887
:1012C0000CE050F8281040318A1101EB5261C9112D
:1012D00040F8281025F8181008F10108B8F1030F9C
:1012E000EFDBB5F90430B5F90220B5F900E000A94B
:1012F000012F7FF434AFBDF80000A0EB0E00ADF875
:1013000000004888801A48808888C01A88804FF07A
:10131000000801E008F10108B8F1030F0EDA00A897
:1013200030F91800002800D540424928F2DB0FF6BA
:10133000B400F3F7B3F94FF0010908E00022FE21F1
:101340001120FFF709FE8146B9F1000F04D1002CEE
:1013500002D02046F4F71AFB484608B0BDE8F087F3
:1013600010B584B000A80FF684011CC91CC00A2265
:1013700000A91020FFF7CDFD002807D1002207218A
:101380000A20FFF7E9FD002800D1002004B010BDBD
:10139000F0B587B004460D4600208DF8000001A886
:1013A00000210A4606C00E46084604E045F826001D
:1013B00044F82600761C032EF8DBFFF7D1FF002847
:1013C00040F0E780C820FFF7F5FD0A270520FFF76A
:1013D000F1FD012200A91E20FFF792FD002840F038
:1013E000D8807F1E03D09DF800008007EED506222E
:1013F00001A92220FFF784FD002840F0CA800026C2
:101400002DE00A270520FFF7D5FD012200A91E20A7
:10141000FFF776FD002840F0BC807F1E03D09DF8CA
:1014200000008007EED5062201A92220FFF768FD03
:10143000002840F0AE80012E10DB2068BDF90410BA
:1014400000FA81F0206001A86168B0F902208918D3
:101450006160A168B0F904000818A060761C062E2F
:10146000CFDB2068052190FBF1F02060606890FBE5
:10147000F1F06060A06890FBF1F0A06004220C2104
:101480001420FFF769FD002840F083803220FFF729
:1014900091FD0A270520FFF78DFD012200A91E20DE
:1014A000FFF72EFD002874D17F1E03D09DF80000A9
:1014B0008007EFD5062201A92220FFF721FD002891
:1014C00067D100262BE00A270520FFF773FD0122D4
:1014D00000A91E20FFF714FD00285AD17F1E03D05B
:1014E0009DF800008007EFD5062201A92220FFF712
:1014F00007FD00284DD1012E10DB2868BDF904102E
:1015000000FA81F0286001A86968B0F90220891802
:101510006960A968B0F904000818A860761C062E56
:10152000D1DB2868052190FBF1F02860686890FB0A
:10153000F1F06860A86890FBF1F0A8600022FF213C
:101540001120FFF709FD002823D100220C211420CF
:10155000FFF702FD00281CD100273E460AE003A940
:1015600041F82600A0F65E0041F6B361884200D340
:101570007F1C761C032E07DA54F8262055F8261017
:10158000881AECD5501AEAE7012F01DB012000E0B0
:10159000002007B0F0BD70B594B004460020ADF84F
:1015A00014000FA800210A4606C00B460EC003A86F
:1015B00006C001A806C00CA80EC009A80EC006A847
:1015C0000EC008460090012205A90F20FFF798FCE5
:1015D000002840F0EC809DF814006A2840F0E78075
:1015E0000FF21460F3F75AF805220FA90620FFF74F
:1015F00087FC060006D10A2211A91020FFF780FC03
:10160000060005D00FF2F850F3F748F83046D0E066
:1016100000A903A8FFF77BFD002821D00FF2E850B6
:10162000F3F73CF8BDF80C00ADF8040001A803A9DD
:101630004A8842808988818005220FA90620FFF709
:1016400068FC060006D10A2211A91020FFF761FCF0
:10165000060043D00FF2C850F3F720F83046A8E058
:101660000A20FFF7A7FC00A903A8FFF750FD0028F8
:101670000ED00FF29C50F3F711F8BDF80C00ADF846
:10168000040001A803A94A88428089888180D3E7A1
:1016900009A90CA8FFF77CFE002805D00FF27850AE
:1016A000F2F7FCFF002500E0012500200AE0891A7E
:1016B00001AA22F8101003A931F9101006AA42F865
:1016C0002010401C0328B7DA0CA951F8202009A9E2
:1016D00051F820108B1AEAD5511AE9E70120207041
:1016E000BDF804006070BDF904000012A07001A8EC
:1016F000B0F90210E17009122171B0F904006071B3
:101700000012A071E57100982072009800126072BA
:1017100000980014A07200980016E07206982073DA
:1017200006980012607306980014A07306980016BD
:10173000E07306A8416821740A1262740A14A27444
:101740000916E17480682075011261750114A17594
:101750000016E0750C9820760CA8B0F90000001275
:1017600060760CA94868A076B1F904000012E07612
:1017700088682077B1F90800001260770998A0778F
:1017800009A8B0F900000012E07709A9486884F8B8
:101790002000B1F90400001284F82100886884F860
:1017A0002200B1F90800001284F8230000E00126AD
:1017B000304614B070BDF8B504460020ADF8000006
:1017C0000420F2F752FB054605F11C06307B002889
:1017D00006D10020E969496888473220FFF7EAFB13
:1017E000012200A91E20FFF78BFB0028F8D19DF8ED
:1017F00000004007F4D5022200A92020FFF780FB5B
:101800000746307B002803D10020E969C968884772
:101810009DF801009DF8001041EA002000B2C110BF
:1018200000EB1170001119302070002060703846F4
:10183000F2BD8648704710B5824C062204F11801AB
:101840002220FFF75DFB002805D00FF2DC30F2F715
:1018500025FF012010BD1020F2F707FB417804F1AD
:10186000180000F057FA94F90C00002809D0401E27
:101870002073062204F1300104F11800F0F7ECFDAA
:1018800006E0062204F1180104F13000F0F7E4FD4F
:10189000002010BD10B50A46D2B201460020FFF765
:1018A00003FB040005D00FF28830F2F7F7FE204664
:1018B00010BD0FF28C30F2F7F1FE002010BD10B514
:1018C0000122FFF7F1FA040005D00FF2A430F2F77D
:1018D000E5FE204610BD40F231320FF274310FF2B6
:1018E0009C30F2F7DBFE002010BD10B50122411C38
:1018F0000078FFF7E2FA040005D00FF2A830F2F703
:10190000CDFE204610BD4FF450720FF278310FF229
:101910006C30F2F7C3FE002010BD10B582B000207D
:10192000ADF80000474C2070602060700820A07067
:10193000474860600020A060012200A90F20FFF747
:10194000DFFA002822D19DF800106A2905D00FF295
:101950006030F2F7A3FE012016BD4422114612208A
:10196000FFF7FAFA002240211320FFF7F5FA0022D0
:1019700080211620FFF7F0FAA0788DF801000122EF
:101980000DF101011120FFF7C4FA002016BD10B5BA
:101990002C4CA06800060BD5002240211320FFF735
:1019A000DBFA00280BD1A06820F08000A06005E0E1
:1019B000FFF7EEFA002802D101202070002010BDB0
:1019C00010B586B0044602A800210A460B460EC098
:1019D00000A806C0FFF72FFF02A94220F2F7FDFA88
:1019E0001848018B029A891AADF80010418B039AAE
:1019F000891AADF80210808B0499401AADF80400E2
:101A0000062200A92046F0F717FD002006B010BD01
:101A100010B5002240211320FFF79EFA00280FD1B5
:101A200000F0C6FF074CA06820F08000A0600022F4
:101A3000F0211120FFF790FA002801D1002020703A
:101A400010BD00005C200020501F002074200020EA
:101A5000295C0F3D70B5A8B001A90FF2AC2370CB83
:101A600070C18DF806000024182806D01C2829D043
:101A70001D2837D0262810D044E01EA82421F0F7D6
:101A800023FD1EA8FFF787FD04462420ADF80700BC
:101A90001EA901A8F5F7F5FA34E02046ADF80000DC
:101AA00000A8FFF788FE04469DF800100FF21820EA
:101AB000F2F7F4FD0220ADF8070000A901A8F5F740
:101AC000E0FA1FE004A86821F0F7FEFC652104A8F5
:101AD000FFF7E0FE6520ADF8070004A901A8F5F7BF
:101AE000D0FA0FE020468DF802000DF102011078C7
:101AF000FFF7E5FE0120ADF807000DF1020101A896
:101B0000F5F7BFFA204628B070BD10B584B0144672
:101B10001A2806D01D2830D0232812D02E2830D0E5
:101B200031E021780FF2B010F2F7B8FD0420F2F79F
:101B30009CF9217841701020F2F797F921784170D3
:101B400021E06078217841EA002000B20090E0783E
:101B5000A17841EA002212B201926079217941EA2A
:101B600000231BB2029300990FF27C10F2F796FD4E
:101B700000A94220F2F786F905E02046FFF7B5FEFE
:101B800001E0FFF724FA002004B010BD736B697008
:101B9000206779726F206F64722121006779726FFC
:101BA000206F64723A25642C20736B69703A256447
:101BB000000000004746462D310000004746462DF4
:101BC000320000004746462D330000004746462DB0
:101BD000340000004753462D350000004753462D82
:101BE000360000004753462D37000000005C4400DB
:101BF00000000000003800004759524F2D530000EC
:101C00004753462D313100004753462D464631009B
